:020000040800F2
:100000000000022011C20008A96E0008E56E000879
:10001000F96E0008FD6E0008016F00080000000086
:10002000000000000000000000000000714B00080C
:10003000056F000800000000014C0008096F00086F
:1000400065C2000865C2000865C2000865C20008F4
:1000500065C2000865C20008D170000865C20008CA
:10006000D9700008E1700008E97000080D6F000801
:1000700065C20008196F000865C20008256F0008F6
:10008000316F000865C20008E16F00083D6F00088D
:10009000496F00084D6F0008516F0008F1700008AB
:1000A00065C200089170000865C2000865C20008BA
:1000B00065C2000865C2000865C20008B970000882
:1000C000C570000865C2000865C2000865C2000866
:1000D00065C2000865C2000865C2000865C2000864
:1000E0001971000865C2000865C2000865C20008F1
:1000F000A5700008556F000865C2000865C20008B9
:1001000065C2000865C2000875700008716F0008BC
:100110007D6F000865C2000865C2000865C200085E
:1001200065C2000865C2000865C2000865C2000813
:1001300065C20008000000000000000065C2000861
:1001400065C2000865C2000865C20008896F000822
:1001500065C2000865C2000865C2000865C20008E3
:1001600065C2000865C2000865C2000865C20008D3
:1001700065C2000865C20008000000000000000021
:0801800065C2000865C2000819
:1001900010B5054C237833B9044B13B10448AFF3C1
:1001A00000800123237010BD08060020000000001D
:1001B000548E020808B5034B1BB103490348AFF343
:1001C000008008BD000000000C060020548E0208CC
:1001D00010F8012B11F8013B012A28BF9A42F7D0F1
:1001E000D01A7047034613F8012B002AFBD1181AC6
:1001F000013870470000000000000000000000000F
:1002000001F0FF01102A2BDB10F0070F08D010F8C7
:10021000013B013A8B422DD010F0070F42B3F6D1CB
:10022000F0B441EA012141EA014122F007047FF0E4
:1002300000070023F0E80256083C85EA010586EA3B
:10024000010685FA47F5A3FA87F586FA47F6A5FA77
:1002500087F68EB9EED1F0BC01F0FF0102F0070283
:1002600032B110F8013B013A83EA010313B1F8D12E
:100270000020704701387047002D06BF354603380F
:10028000073815F0010F07D1013015F4807F02BF48
:10029000013015F4C03F0130F0BC0138704700BF99
:1002A00081F0004102E000BF83F0004330B54FEA27
:1002B00041044FEA430594EA050F08BF90EA020F94
:1002C0001FBF54EA000C55EA020C7FEA645C7FEA27
:1002D000655C00F0E2804FEA5454D4EB5555B8BF4A
:1002E0006D420CDD2C4480EA020281EA030382EABB
:1002F000000083EA010180EA020281EA0303362D4D
:1003000088BF30BD11F0004F4FEA01314FF4801C1F
:100310004CEA113102D0404261EB410113F0004F31
:100320004FEA03334CEA133302D0524263EB4303E8
:1003300094EA050F00F0A780A4F10104D5F1200E86
:100340000DDB02FA0EFC22FA05F2801841F10001E1
:1003500003FA0EF2801843FA05F359410EE0A5F1B5
:1003600020050EF1200E012A03FA0EFC28BF4CF0E6
:10037000020C43FA05F3C01851EBE37101F000459C
:1003800007D54FF0000EDCF1000C7EEB00006EEBA9
:100390000101B1F5801F1BD3B1F5001F0CD3490833
:1003A0005FEA30004FEA3C0C04F101044FEA44528A
:1003B00012F5800F80F09A80BCF1004F08BF5FEA11
:1003C000500C50F1000041EB045141EA050130BDF1
:1003D0005FEA4C0C404141EB0101013C28BFB1F503
:1003E000801FE9D291F0000F04BF01460020B1FA4E
:1003F00081F308BF2033A3F10B03B3F120020CDA21
:100400000C3208DD02F1140CC2F10C0201FA0CF0FE
:1004100021FA02F10CE002F11402D8BFC2F1200C63
:1004200001FA02F120FA0CFCDCBF41EA0C01904019
:10043000E41AA2BF01EB0451294330BD6FEA040462
:100440001F3C1CDA0C340EDC04F11404C4F120024D
:1004500020FA04F001FA02F340EA030021FA04F35F
:1004600045EA030130BDC4F10C04C4F1200220FAB6
:1004700002F001FA04F340EA0300294630BD21FAF4
:1004800004F0294630BD94F0000F83F4801306BFBA
:1004900081F480110134013D4EE77FEA645C18BFAE
:1004A0007FEA655C29D094EA050F08BF90EA020F45
:1004B00005D054EA000C04BF1946104630BD91EA3D
:1004C000030F1EBF0021002030BD5FEA545C05D140
:1004D0004000494128BF41F0004130BD14F580047F
:1004E0003CBF01F5801130BD01F0004545F0FE41F3
:1004F00041F470014FF0000030BD7FEA645C1ABF28
:10050000194610467FEA655C1CBF0B46024650EA5E
:10051000013406BF52EA033591EA030F41F400218A
:1005200030BD00BF90F0000F04BF0021704730B510
:100530004FF4806404F132044FF000054FF00001E5
:1005400050E700BF90F0000F04BF0021704730B5A6
:100550004FF4806404F1320410F0004548BF40427B
:100560004FF000013EE700BF42004FEAE2014FEAD0
:1005700031014FEA02701FBF12F07F4393F07F4FAB
:1005800081F06051704732F07F4208BF704793F0AE
:100590007F4F04BF41F40021704730B54FF46074C1
:1005A00001F0004521F000411CE700BF50EA0102C4
:1005B00008BF704730B54FF000050AE050EA01026D
:1005C00008BF704730B511F0004502D5404261EBDD
:1005D00041014FF4806404F132045FEA915C3FF41E
:1005E000D8AE4FF003025FEADC0C18BF03325FEABB
:1005F000DC0C18BF033202EBDC02C2F1200300FA6C
:1006000003FC20FA02F001FA03FE40EA0E0021FA90
:1006100002F11444BDE600BF70B54FF0FF0C4CF47E
:10062000E06C1CEA11541DBF1CEA135594EA0C0F30
:1006300095EA0C0F00F0DEF82C4481EA030621EA6B
:100640004C5123EA4C5350EA013518BF52EA0335A6
:1006500041F4801143F4801338D0A0FB02CE4FF058
:100660000005E1FB02E506F00042E0FB03E54FF088
:100670000006E1FB03569CF0000F18BF4EF0010E80
:10068000A4F1FF04B6F5007F64F5407404D25FEA7C
:100690004E0E6D4146EB060642EAC62141EA55512F
:1006A0004FEAC52040EA5E504FEACE2EB4F1FD0C71
:1006B00088BFBCF5E06F1ED8BEF1004F08BF5FEAEF
:1006C000500E50F1000041EB045170BD06F00046A1
:1006D00046EA010140EA020081EA0301B4EB5C044E
:1006E000C2BFD4EB0C0541EA045170BD41F4801146
:1006F0004FF0000E013C00F3AB8014F1360FDEBF6B
:10070000002001F0004170BDC4F10004203C35DA46
:100710000C341BDC04F11404C4F1200500FA05F3C9
:1007200020FA04F001FA05F240EA020001F000426A
:1007300021F0004110EBD37021FA04F642EB0601E0
:100740005EEA430E08BF20EAD37070BDC4F10C040A
:10075000C4F1200500FA04F320FA05F001FA04F2CE
:1007600040EA020001F0004110EBD37041F10001BA
:100770005EEA430E08BF20EAD37070BDC4F12005C5
:1007800000FA05F24EEA020E20FA04F301FA05F22D
:1007900043EA020321FA04F001F0004121FA04F2D5
:1007A00020EA020000EBD3705EEA430E08BF20EAA5
:1007B000D37070BD94F0000F0FD101F000464000DF
:1007C00041EB010111F4801F08BF013CF7D041EA61
:1007D000060195F0000F18BF704703F00046520065
:1007E00043EB030313F4801F08BF013DF7D043EA36
:1007F0000603704794EA0C0F0CEA135518BF95EAEC
:100800000C0F0CD050EA410618BF52EA4306D1D172
:1008100081EA030101F000414FF0000070BD50EA91
:10082000410606BF1046194652EA430619D094EA1B
:100830000C0F02D150EA013613D195EA0C0F05D105
:1008400052EA03361CBF104619460AD181EA030159
:1008500001F0004141F0FE4141F470014FF0000011
:1008600070BD41F0FE4141F4780170BD70B54FF0AC
:10087000FF0C4CF4E06C1CEA11541DBF1CEA13552C
:1008800094EA0C0F95EA0C0F00F0A7F8A4EB05040E
:1008900081EA030E52EA03354FEA013100F0888005
:1008A0004FEA03334FF0805545EA131343EA1263CE
:1008B0004FEA022245EA111545EA10654FEA002683
:1008C0000EF000419D4208BF964244F1FD0404F53C
:1008D000407402D25B084FEA3202B61A65EB030598
:1008E0005B084FEA32024FF480104FF4002CB6EB55
:1008F000020E75EB030E22BFB61A754640EA0C00D5
:100900005B084FEA3202B6EB020E75EB030E22BF14
:10091000B61A754640EA5C005B084FEA3202B6EB55
:10092000020E75EB030E22BFB61A754640EA9C0014
:100930005B084FEA3202B6EB020E75EB030E22BFE4
:10094000B61A754640EADC0055EA060E18D04FEAA2
:10095000051545EA16754FEA06164FEAC30343EA42
:1009600052734FEAC2025FEA1C1CC0D111F4801F0F
:100970000BD141EA00014FF000004FF0004CB6E708
:1009800011F4801F04BF01430020B4F1FD0C88BFA7
:10099000BCF5E06F3FF6AFAEB5EB030C04BFB6EBB2
:1009A000020C5FEA500C50F1000041EB045170BDA5
:1009B0000EF0004E4EEA113114EB5C04C2BFD4EBD2
:1009C0000C0541EA045170BD41F480114FF0000E56
:1009D000013C90E645EA060E8DE60CEA135594EAD2
:1009E0000C0F08BF95EA0C0F3FF43BAF94EA0C0FD5
:1009F0000AD150EA01347FF434AF95EA0C0F7FF44A
:100A000025AF104619462CE795EA0C0F06D152EA9D
:100A100003353FF4FDAE1046194622E750EA410681
:100A200018BF52EA43067FF4C5AE50EA41047FF492
:100A30000DAF52EA43057FF4EBAE12E74FF0FF3CF7
:100A400006E000BF4FF0010C02E000BF4FF0010CC8
:100A50004DF804CD4FEA410C7FEA6C5C4FEA430C41
:100A600018BF7FEA6C5C1BD001B050EA410C0CBF90
:100A700052EA430C91EA030F02BF90EA020F0020F2
:100A8000704710F1000F91EA030F58BF994208BF59
:100A900090422CBFD8176FEAE37040F00100704716
:100AA0004FEA410C7FEA6C5C02D150EA013C07D16D
:100AB0004FEA430C7FEA6C5CD6D152EA033CD3D0B8
:100AC0005DF8040B704700BF8446104662468C46B2
:100AD0001946634600E000BF01B5FFF7B7FF0028E5
:100AE00048BF10F1000F01BD4DF808EDFFF7F4FF0E
:100AF0000CBF012000205DF808FB00BF4DF808ED99
:100B0000FFF7EAFF34BF012000205DF808FB00BFBB
:100B10004DF808EDFFF7E0FF94BF012000205DF8DD
:100B200008FB00BF4DF808EDFFF7CEFF94BF012092
:100B300000205DF808FB00BF4DF808EDFFF7C4FF8B
:100B400034BF012000205DF808FB00BF4FEA410CD4
:100B50007FEA6C5C02D150EA013C0AD14FEA430CB7
:100B60007FEA6C5C02D152EA033C02D14FF00000F4
:100B700070474FF0010070474FEA410212F5001232
:100B800015D211D56FF47873B3EB625212D94FEAD4
:100B9000C12343F0004343EA505311F0004F23FABE
:100BA00002F018BF404270474FF00000704750EA13
:100BB000013005D111F0004008BF6FF000407047D0
:100BC0004FF00000704700BF4A0011D212F500122A
:100BD00011D20DD56FF47873B3EB62520ED44FEA95
:100BE000C12343F0004343EA505323FA02F0704715
:100BF0004FF00000704750EA013002D14FF0FF3053
:100C000070474FF0000070474FEA4102B2F1E043F5
:100C100024BFB3F5001CDCF1FE5C0DD901F0004CE3
:100C20004FEAC0024CEA5070B2F1004F40EB830033
:100C300008BF20F00100704711F0804F21D113F15F
:100C40003872BCBF01F00040704741F480114FEA98
:100C50005252C2F11802C2F1200C10FA0CF320FA21
:100C600002F018BF40F001004FEAC1234FEAD3233E
:100C700003FA0CFC40EA0C0023FA02F34FEA4303A8
:100C8000CCE77FEA625307D150EA01331EBF4FF031
:100C9000FE4040F44000704701F0004040F0FE404C
:100CA00040F40000704700BF7BB972B90029BEBF95
:100CB00000204FF0004106E008BF00281CBF6FF085
:100CC00000414FF0FF3001F041B9ADF1080C6DE982
:100CD00004CE002909DB002B1ADB00F083F8DDF8D5
:100CE00004E0DDE9022304B07047404261EB4101BA
:100CF000002B1BDB00F076F8DDF804E0DDE90223D1
:100D000004B0404261EB4101524263EB4303704740
:100D1000524263EB430300F065F8DDF804E0DDE9DF
:100D2000022304B0404261EB41017047524263EB41
:100D3000430300F057F8DDF804E0DDE9022304B0D6
:100D4000524263EB4303704753B94AB9002908BFC5
:100D500000281CBF4FF0FF314FF0FF3001F0F6B814
:100D6000ADF1080C6DE904CE00F03CF8DDF804E0CC
:100D7000DDE9022304B0704738B5002200230446A1
:100D80000D46FFF7BBFE28B920462946BDE838408E
:100D900000F00AB8204605F1004100F005F8404295
:100DA00061EB410138BD00BFD0B50C4B00220646B7
:100DB0000F46FFF731FCFFF707FF0446FFF7B2FBD2
:100DC000074B0022FFF728FC02460B463046394607
:100DD000FFF76AFAFFF7F8FE2146D0BD0000F03DAC
:100DE0000000F0412DE9F047089D04468C46002B99
:100DF00040F083808A42174647D9B2FA82F242B164
:100E0000C2F1200024FA00F09140974040EA010C22
:100E100094404FEA1748230CBCFBF8F61FFA87FEF4
:100E200008FB16C143EA014306FB0EF1994209D9BA
:100E3000FB1806F1FF3080F01981994240F21681CB
:100E4000023E3B445B1AA4B2B3FBF8F008FB10333C
:100E500044EA034400FB0EFEA64509D93C1900F103
:100E6000FF3380F00581A64540F2028102383C4400
:100E700040EA0640A4EB0E0400261DB1D440002336
:100E8000C5E900433146BDE8F08702B9FFDEB2FA9A
:100E900082F2002A50D1CB1B4FEA174E1FFA87F877
:100EA0000126B3FBFEFC210C0EFB1C3341EA03417F
:100EB00008FB0CF38B4207D979180CF1FF3002D2F2
:100EC0008B4200F2E9808446C91AA3B2B1FBFEF05E
:100ED0000EFB101143EA014408FB00F8A04507D9B6
:100EE0003C1900F1FF3302D2A04500F2D980184628
:100EF000A4EB080440EA0C40BFE78B4209D9002D5F
:100F000000F0B1800026C5E9000130463146BDE859
:100F1000F087B3FA83F6002E4AD18B4202D3824285
:100F200000F2B880841A61EB030101208C46002D89
:100F3000A8D0C5E9004CA5E7C2F1200320FA03F6CA
:100F4000974001FA02F04FEA174ED9403043030CA4
:100F5000B1FBFEF61FFA87F80EFB161143EA0143B8
:100F600006FB08F1994204FA02F409D9FB1806F1CC
:100F7000FF3C80F08D80994240F28A80023E3B44E3
:100F80005B1A81B2B3FBFEF00EFB103341EA034162
:100F900000FB08F38B4207D9791800F1FF3C73D2AC
:100FA0008B4271D902383944CB1A40EA064678E7B9
:100FB000C6F1200C03FA06F422FA0CF31C4320FAC3
:100FC0000CF701FA06F34FEA144E21FA0CF11F4315
:100FD0003B0CB1FBFEF91FFA84F80EFB191143EA32
:100FE000014109FB08FA8A4502FA06F200FA06F303
:100FF00008D9611809F1FF3048D28A4546D9A9F1CC
:1010000002092144A1EB0A01BFB2B1FBFEF00EFBC5
:10101000101147EA014700FB08F8B84507D9E7195E
:1010200000F1FF312ED2B8452CD90238274440EACE
:101030000940A7EB0807A0FB02894F45C646494671
:101040001AD317D05DB1B3EB0E0267EB010707FAB5
:101050000CFCF2404CEA0202F740C5E900270026EA
:101060003146BDE8F0872E4628460BE70646E9E6FE
:101070001846FDE64345E5D2B8EB020E69EB0401E4
:101080000138DFE70846D2E760468DE78146B9E7D9
:10109000664675E730464AE7ACF1020C394413E77F
:1010A00002383C4424E700BF03685A004CBF43F0B9
:1010B000004323F000431844704700BF2DE9F84374
:1010C00029B34F1E044615463E464FF0000808EB74
:1010D000060101EBD171491004EBC1094846FFF745
:1010E000E3FF0346C80008308F42204409D0AB42DA
:1010F00009D8FFF7D9FF0138A8420AD201F1010847
:10110000E5E7AB4205D9884501D04E1EDFE74FF039
:1011100000094846BDE8F883012807D0022807D017
:10112000044B00280CBF1846002070470248704747
:1011300002487047DD170008E1170008E5170008AE
:1011400030B5234B83B004468D1E3BB301A928461E
:10115000AFF30080E8B101992A46FFF7AFFF0146DF
:10116000B8B1FFF7A1FF4B68A064012B2BD0002B77
:1011700001F1040023DBFFF797FF0023C4E9130309
:101180000368002B10DBFFF78FFF2061002003B006
:1011900030BD00230920236103B030BD0D490E4846
:1011A000091AC9100191D7E7C3F30360FFF7B4FF31
:1011B0000028206114BF0020092003B030BD0123A6
:1011C000C4E91303DCE7002323610520DFE700BF48
:1011D00000000000D47F0308D47503080368DA0711
:1011E00010B5044606D49B0700F1480009D500F06D
:1011F0004BFC2368590709D51A070ED5DB0613D512
:1012000010BD00F039FC23685907F5D404F1D00073
:1012100000F042FC23681A07F0D404F5A87000F02F
:1012200043FC2368DB06EBD404F5E870BDE810400E
:1012300000F07EBC0346006800B11844704700BF50
:1012400009207047704700BF70B504460E46316CE8
:101250002046FFF775FF054688B9336C6361324657
:1012600023692146012098470828F0D0072806D195
:101270002846316CFFF7E6FF301D00F0F1FB22F04D
:1012800007FD00BF2DE9F0470D1D064614460FCDA2
:10129000ADF5727D0DF10C0CACE80F000FCDACE894
:1012A0000F000FCDACE80F0095E80F0002ADF76816
:1012B000D6F818808CE80F0000232B6021E02B6CFF
:1012C00073614FF4F07229467AA822F053FD336916
:1012D0007AAA314650469847889BCDE90058214666
:1012E0006B648146334632460120B8470446E8B96C
:1012F0004FF4F0727AA9284622F03CFDB9F1080FAC
:101300001BD1296C3046FFF71BFF09345FFA84FAC2
:1013100081460028D3D0AB6B4AF01001CDE90058CC
:1013200032466B6401203346B84708B14FF00909D3
:1013300048460DF5727DBDE8F087B9F1070FF5D18C
:101340002046296CFFF77EFF03A800F089FB00BF51
:10135000406C7047F0B5CB6B0B640E1D0F46054615
:101360000FCEF9B001AC0FC40FCE0FC40FCE0FC417
:1013700096E80F004FF0FF3684E80F00009606E075
:101380002B696A46294698470828044608D11099CF
:101390002846FFF7D5FE0028F2D0092079B0F0BD2D
:1013A0006846FFF71BFF062CF7D139462846FFF7A2
:1013B0004BFF00BF30B4DD6BC160826119461D6414
:1013C000002230BC5EE700BF70B5C66843690B649D
:1013D000AEB903690A4604460D4601460220984705
:1013E000072805D008280FD129462046FFF72CFFF3
:1013F0003046296CFFF726FF281D00F031FB012243
:10140000FFF740FF22F044FC22F042FCC2681AB110
:10141000CA6B0A64002235E79CE700BF704700BF33
:10142000836801460BB1012018477047012912D08B
:1014300009D873B90F2A0CD800EB820218465368FA
:10144000009A136070470339012994BF01200220DC
:101450007047022070470846704700BF10B584B03F
:10146000002303AC0A4600941946FFF7DFFF0398F8
:1014700004B010BD012912D009D873B90F2A0CD8B5
:1014800000EB8200009A12684260184670470339E8
:10149000012994BF012002207047022070470846AE
:1014A000704700BF10B584B0002303AC03920094D2
:1014B0000A461946FFF7DEFF04B010BDF0B5D36B46
:1014C0001364151D8C4606460FCDADF50F7D17AC88
:1014D0000FC40FCD0FC40FCD0FC495E80F004FF010
:1014E000FF3784E80F006546169710E0FFF7DAFF34
:1014F000294616A8B047034616AA6946082083B9AC
:10150000049B9847052804460CD0092809D0269941
:101510006846FFF715FE03466A460C2116A8002B05
:10152000E4D0092416A8FFF759FE20460DF50F7DDB
:10153000F0BD00BF2DE9F04FCC6C89B00D4654F8DA
:10154000041B0694174600F003081E46002B79D0B2
:101550000B0CDAB209048DF81D30022304EB82046F
:1015600005918DF81C302B6DB8F1020F08BFAC6BE4
:1015700013F001030CD0384605A900F073FB18B92D
:10158000082009B0BDE8F08F092009B0BDE8F08F50
:10159000D4F800A0BAF1000FEDD0019300F00803D9
:1015A0000293022E4AD0B4F800A0B4F8029004349A
:1015B000AA6C29F0010B0F2138469344FFF74EFF28
:1015C000834539D82AF001025A44824294BF002050
:1015D00001204FEA490303F002030AF0010A43EA3B
:1015E0000A03012B49D0022B32D0002BCCD1B8F109
:1015F000000F02D0002840F0CD800434D4F800A0C1
:10160000BAF1000FCDD105A9384600F02BFB002818
:10161000BAD1019B002BB3D00F213846FFF71EFF34
:101620000E2102463846FFF73DFF38466A4A0F2131
:10163000FFF738FF0720A8E70020CAE7D4F8049096
:101640000834B5E7090203230591ADF81C308AE799
:10165000236823F0004BB8F1000F45D128B1029A5E
:10166000002A5CD0BBF1000F74D0002B00DA0434E8
:101670000BF1010B04EB8B04C0E7B8F1000F19D19B
:10168000B0B1D4E90023991C4FEAD2723FF47CAF89
:1016900005F158010133049100F09080201DFFF7FF
:1016A000C9FD04AB0146284621F0AAFA00285BD107
:1016B0000834A3E70D213846D5F82090FFF7CEFE79
:1016C0008145F5D1AB6A9C42F2D12046FFF7ECFC94
:1016D0000F2102463846FFF7E5FE38462A4600212C
:1016E000FFF7E0FE072050E70D213846D5F820909F
:1016F000FFF7B4FE814501D02368B6E7AB6A9C4290
:10170000FAD104220021C5E90B12A318C5F828B0AC
:101710006B6323688B4259DB01230193A8E705F132
:101720005803CDF80C8004F1040AB04691461E46D9
:101730000DE00496FFF77EFD04AB0146002228462B
:1017400021F05EFA09F101090AF1040AE8B9D94564
:101750005046EED138460D21FFF780FE049B2862EB
:10176000C5E90934062010E781460D213846FFF708
:1017700075FEB9F1020F286225D12B46049A43F871
:101780002C2F6B62AC620620FFE646462368DDF82C
:101790000C806AE72046FFF787FC04340246AC63FE
:1017A0002846144621F08AFA00283FF4EDAE384668
:1017B00022460F21FFF776FE0720E6E638460D2188
:1017C000FFF74CFE2862049B6B62DBE70BF1010024
:1017D00004EB80007AE700BF9D3802080023A9E6E9
:1017E0000123A7E60223A5E62DE9F0430646C3B090
:1017F00015461C46042900F2B980DFE801F09A532F
:10180000B7290300002C40F0B180102A00F2AE800E
:101810000368D80600F1F38020AF384600F092F953
:10182000B06B0023012404FA03F22A42014604D0DB
:1018300051F8042B47F8232008460133042BF2D13A
:10184000B063384600F074F9002043B0BDE8F0837F
:10185000032C40F08B8094B204EB1243102B4FEA20
:10186000124500F2838003681F0700F1D08020AF8B
:10187000384600F03BF907EBC501B56B54B10B4698
:10188000E81A01EBC401E4001A5843F8042B8B4218
:10189000FAD125443846B56300F006F9002043B07C
:1018A000BDE8F083012C4FEA124895B25AD0052CBE
:1018B0005CD108EB0509B9F1200F57D8B8F10F0F2B
:1018C00077D9A946002D40F08880B36B6DB320AF67
:1018D0004FF0000907EBC807043F03EBC50553F8B9
:1018E000041B47F8041FAB42F9D1B9F1000F0FD028
:1018F0006F464146102938BF102107EBC1018439DA
:1019000003EBC90553F8040B41F8040FAB42F9D1BE
:10191000012C00F08480B8F10F0FB56345D9B9F1FF
:10192000000F02D0684600F0B7F8002043B0BDE8D1
:10193000F083DCB9876B2346012094B206F1040CD6
:1019400000FA03F22242394604D051F8042B4CF835
:1019500023200F460133102BF2D115F40050E4D1AF
:10196000B76304E008EB0503102B03D9022043B052
:10197000BDE8F083B8F10F0FF8D83368DA0706D561
:10198000304623F0030340F8483B00F079F820AFDD
:10199000384600F075F8B36B002D99D11D4604351B
:1019A000B563384600F068F8BFE720A800F06CF88F
:1019B000B5E7B9F1100F40D9A9F110093368D9077B
:1019C00008D523F00103304643F0020340F8483BBA
:1019D00000F05EF8B9F1000F32D033685A0720D416
:1019E000B8F10F0F25D96F463846C8F1100500F041
:1019F00057F8002DB36B7FF77CAF20AF6AE723F079
:101A00001003336006F5E87000F09CF804E723F05B
:101A10000803036000F5A87000F068F827E720AF1E
:101A2000BDE7304623F0040340F8D03B00F038F81F
:101A3000D6E720A800F02CF8D5E74FF00009BDE765
:101A4000B8F10F0F3FF641AF20AF384600F020F855
:101A5000B36B002D7FF43CAF384600F015F864E717
:101A600000F1340191E838009C46A6464CF8045D2C
:101A700090E8FF0FE54600BD90EC210B704700BFDA
:101A800080EC210B704700BF90EC200B704700BF2B
:101A900080EC200B704700BFD0EC200B704700BFDC
:101AA000C0EC200B704700BFF0EC0201F0EC02111B
:101AB000F0EC0221F0EC0231F0EC0241F0EC0251CA
:101AC000F0EC0261F0EC0271F0EC0281F0EC0291BA
:101AD000F0EC02A1F0EC02B1F0EC02C1F0EC02D1AA
:101AE000F0EC02E1F0EC02F1704700BFE0EC020123
:101AF000E0EC0211E0EC0221E0EC0231E0EC02410A
:101B0000E0EC0251E0EC0261E0EC0271E0EC0281F9
:101B1000E0EC0291E0EC02A1E0EC02B1E0EC02C1E9
:101B2000E0EC02D1E0EC02E1E0EC02F1704700BF32
:101B3000B0FC0181B0FC0191B0FC01A1B0FC01B18D
:101B4000704700BFA0FC0181A0FC0191A0FC01A195
:101B5000A0FC01B1704700BFEC4600B52DE9005074
:101B60002DE9FF1F4FF000032DE90C0001A9FFF73D
:101B7000F1FBDDF840E012B0704700BFEC4600B565
:101B80002DE900502DE9FF1F4FF000032DE90C0057
:101B900001A9FFF719FCDDF840E012B0704700BF63
:101BA000EC4600B52DE900502DE9FF1F4FF0000372
:101BB0002DE90C0001A9FFF729FCDDF840E012B087
:101BC000704700BFEC4600B52DE900502DE9FF1F1E
:101BD0004FF000032DE90C0001ABFFF7EBFBDDF844
:101BE00040E012B0704700BFEC4600B52DE9005050
:101BF0002DE9FF1F4FF000032DE90C0001AAFFF7AC
:101C00005DFCDDF840E012B0704700BF027A7AB99F
:101C1000437AA3B14268013B10B4437213680321B5
:101C2000141D01721A024460026010BC180E704745
:101C30000368013A02721A020260180E7047B0205F
:101C4000704700BF00B585B003AA00230092194673
:101C50000C22FFF7EBFB039805B05DF804FB00BF17
:101C6000F0E700BF2DE9F043054685B00E464FF082
:101C700000083046FFF7CAFFB028044600F0B280E3
:101C8000070620D500F0F003802B4DD0902B36D0E6
:101C9000A02B60D0B02B74D0C02B00F08B8000F054
:101CA000F803D02B0BD100F00702013242F40022DE
:101CB000052301212846FFF797FD0028D9D00920E8
:101CC00005B0BDE8F0830DF10C090023194687002B
:101CD000CDF800900D222846FFF7A8FBFFB2039B2A
:101CE000CDF80090043760064CBFDF1BFF180023BF
:101CF00019460D2228460397FFF7BCFBB9E700F011
:101D00000D030D2BDBD003AF002300F00F021946AB
:101D100000972846FFF78AFB0023009719460D22FB
:101D20002846FFF7A7FBA4E73046FFF76FFF240222
:101D30002043B0F5004FC2D004010023A2B21946DF
:101D40002846FFF751FD0028B9D114F4004F18BF01
:101D50004FF001088DE7C24302F007034FF47F62A2
:101D60001A41010702F47F624FF0000348BF42F4BA
:101D7000804219462846FFF737FD00283FF479AF27
:101D80009DE7B12833D0B22800F08B80B32839D03A
:101D900000F0FC03B42B92D000F0070201320123C3
:101DA00042F4002219462846FFF71EFD00283FF4A2
:101DB00060AF84E7C62842D0C7284CD000F0F803B3
:101DC000C02B5BD0C82860D0C9287FF478AF3046DC
:101DD000FFF71CFF020300F00F0002F47022013035
:101DE000024365E7B8F1000F18D0002068E73046DD
:101DF000FFF70CFF024600283FF461AF10F0F0033C
:101E0000D0D05CE73046FFF701FF010300F00F0080
:101E100001F47021421C01230A43C3E703AC43468B
:101E20000E22414600942846FFF700FB0094284606
:101E300043460F224146FFF71DFB404640E7304630
:101E4000FFF7E4FE010300F00F0001F47021421CD3
:101E500003230A43A6E73046FFF7D8FE02460028D0
:101E60003FF42DAF10F0F0037FF429AF0421284692
:101E7000FFF7BAFC00283FF4FCAE20E700F00F02A9
:101E80000132032342F420228CE73046FFF7BEFEE6
:101E900000F0F00200F00F031032013343EA023287
:101EA00006E700230DF10C090D221946CDF800902C
:101EB0002846FFF7BBFA3046FFF7A8FE02064FF0B0
:101EC00002070CD5039B00F07F00B8400344304666
:101ED0000393FFF79BFE030607F10707F2D4039B6A
:101EE000CDF8009000F07F0403F50172BC400023A0
:101EF000144419460D2228460394FFF7BBFAB8E6AE
:101F000010B5C26C84B0536803248DF80C401B02DA
:101F100002F108040846D279019301A902948DF8D0
:101F20000D20FFF79FFE04B010BD00BF08B5FFF7FE
:101F300097FE806C08BD00BF08B5FFF791FEC06C2E
:101F4000C379023300EB830008BD00BF704700BFB8
:101F5000F1EE103A43F08073E1EE103A704700BFA3
:101F60000849CA6810B400024FF6FF04224000F48A
:101F7000E063134343F0BF6343F400335DF8044B65
:101F8000CB60704700ED00E0194BDB68C3F3022320
:101F900030B4C3F10705042D03F1040428BF042560
:101FA000062C19D9033B4FF0FF349C4022EA04026F
:101FB0004FF0FF34AC4021EA04019940002841EA87
:101FC00002010CDB00F1604000F561400901C9B27B
:101FD00080F8001330BC704700221346E8E7054B39
:101FE00000F00F0009010344C9B2197630BC7047F4
:101FF00000ED00E0FCEC00E000F01F01034A4009A6
:1020000001238B4042F82030704700BF00E100E020
:1020100043090549203300F01F00012202FA00F0B5
:1020200041F82300704700BF00E100E00138B0F143
:10203000807F0ED2084B10B4084C5860F02084F812
:1020400023000022072110469A605DF8044B1960B6
:1020500070470120704700BF10E000E000ED00E095
:10206000044A136804280CBF43F0040323F004035C
:102070001360704710E000E038B5134602250A46A9
:10208000C0E90633C0F8F451002102F02FFC002013
:1020900038BD00BF08B513460A46002102F026FCF1
:1020A000002008BD38B5134603250A46C0E942336F
:1020B000C0F8F451002102F027FC002038BD00BF19
:1020C00008B513460A46002102F01EFC002008BD98
:1020D00008B504220023C0F8F42119461A4602F07C
:1020E00005FC002008BD00BF08B505220023C0F88C
:1020F000F42119461A4602F007FC002008BD00BF73
:1021000030B5014689B000222D20FFF73DFF2D207C
:10211000FFF772FF0025164B02951A6C154C42F41E
:1021200080721A641B6C03F4807301A9029303A8E4
:10213000029B05F047FB05F025FB0F4A0F4925617F
:102140004300A2FB03239B0C013B40F2E7322046F5
:10215000C4E901352160E26008F0D4FA10B1012031
:1021600009B030BD204608F01FF809B030BD00BFEF
:1021700000380240B4C5002083DE1B43002000402D
:1021800000287CD038B590F820300446002B73D05E
:102190002268136823F00203136004F04DFD054626
:1021A00004E004F049FD431B0A2B5CD823685A68FD
:1021B0009107F6D41A6842F001021A6004F03CFD5F
:1021C000054604E004F038FD401B0A284BD823687C
:1021D0005A68D207F6D5227E012A1A680CBF42F04F
:1021E000800222F080021A60627E012A1A680CBF07
:1021F00042F0400222F040021A60A27E012A1A68D0
:102200000CBF42F0200222F020021A60E27E012A76
:102210001A680CBF22F0100242F010021A60227FEE
:10222000012A1A680CBF42F0080222F008021A6064
:10223000627F012A1A680CBF42F0040222F00402F5
:102240001A60D4E90221D4E904500A4361682A43A0
:10225000024301390A4301250021DA61616284F8F1
:102260002050084638BD636A052243F40033636298
:1022700084F82020012038BD04F0ACFF88E701205D
:10228000704700BF90F82030012B09D090F8203023
:10229000022B05D0436A43F4802343620120704738
:1022A0003B4BD3F8002242F00102F0B4C3F8002205
:1022B000D3F8002222F47C52C3F80022D3F8002283
:1022C000486A42EA0022C3F800224A69D3F81C4255
:1022D0000120904024EA0004C3F81C42CD69C443A5
:1022E000002D45D1D3F80C522540C3F80C52D20032
:1022F000CF688D888E680B8802F1804202F5C84253
:1023000045EA074543EA0643C2F84052C2F8443260
:102310008B691F4A33BBD2F804322340C2F804321F
:102320000B69C3B91A4BD3F814221440C3F81442F2
:102330000B6A012B05D1164AD2F81C321843C2F899
:102340001C02134AD2F8003223F001030020F0BC33
:10235000C2F8003270470E4AD2F814320343C2F872
:102360001432E5E7D2F804320343C2F80432D7E767
:10237000012DCDD1D3F80C520543C3F80C52D20035
:102380000F688D888E688B8902F18042B6E700BFA6
:102390000064004070B590F82030012B044606D050
:1023A000436A012643F400234362304670BD02684D
:1023B000DEB2022380F82030136823F0010313609B
:1023C00004F03AFC054604E004F036FC431B0A2BFB
:1023D00008D823685B6813F00103F5D11E466362D9
:1023E000304670BD636A052243F40033636284F8AB
:1023F0002020304670BD00BF38B590F82030022B49
:10240000044605D0436A43F480134362012038BD7B
:102410000268136843F00103136004F00DFC0546E5
:1024200004E004F009FC431B0A2B0CD823685A680B
:10243000D207F6D51A68012122F002021A6084F848
:102440002010002038BD636A052243F40033636224
:1024500084F82020012038BD70B490F82040012C71
:102460000AD090F82040022C06D0436A43F480231F
:10247000436270BC012070470468A5686D0105D4F3
:10248000A5682E0102D4A568ED0039D5A068012504
:10249000C0F3016085401D608B6843B3CD684E6812
:1024A0002B4300F118052D0143EAC603635104EBE9
:1024B00000130D69C3F88451097D01294FEA00100A
:1024C00005D1D3F8841141F48071C3F88411044418
:1024D0005168C4F88C111268C4F88821D3F880219F
:1024E00042F00102002070BCC3F8802170470E68E2
:1024F000CD6800F118031B0145EA4655E550D6E7C3
:10250000436A43F40013436270BC0120704700BF6C
:1025100090F82030012B05D090F82030022B01D00C
:1025200000207047036898689A689B681201C0F39E
:10253000806048BF0130DB00F3D50130704700BF39
:102540002DE9F04190F82050012D04460AD090F872
:102550002000022806D0636A43F4802363620120CE
:10256000BDE8F081256800295AD1E86886076CD05B
:1025700005EB01100F01D0F8B06106F0040696607B
:10258000002E58D1D0F8B061760D1660D0F8B0E1C9
:10259000D0F8B4C1D0F8B461D0F8B4013D44CEF362
:1025A000400ED5F8B881C6F307260CF00F05000CD5
:1025B000C2E903E5C2E9050683F8008022683A44CF
:1025C000D2F8B821120A5A7022683A44D2F8B821D7
:1025D000120C9A7022683A44D2F8B821120EDA70BE
:1025E00022683A44D2F8BC211A7122683A44D2F8DF
:1025F000BC21120A5A7122683A44D2F8BC21120C4A
:102600009A7122681744D7F8BC21120EDA71B9B951
:102610002268D36843F020030846D360BDE8F08108
:102620000129A5D128698007A2D1636A43F4001368
:102630000846636294E7D0F8B061F6085660A5E7F3
:10264000012909D00020BDE8F081636A43F400133A
:1026500063620120BDE8F0812268136943F0200322
:10266000136100207CE700BF90F82030012B05D0DB
:1026700090F82030022B01D000207047036819B970
:10268000D86800F003007047186900F00300704735
:1026900090F82030012B09D090F82030022B05D083
:1026A000436A43F480234362012070470268536900
:1026B000194351610020704790F82030012B09D058
:1026C00090F82030022B05D0436A43F48023436204
:1026D000012070470268536923EA0101516100201B
:1026E000704700BF2DE9F84F03685C69D3F8048098
:1026F0009F68D3F80CB0D3F810A0D3F8189014F05A
:10270000010605461ED017F0010653D1F8050BD57A
:102710002B684FF48072B9059A6000F1C0807A0589
:1027200040F1D88046F40056F8030BD52B684FF4DF
:102730008032B9039A6000F1AA807A0340F1CF8019
:1027400046F40046270702D51BF0100F6DD1600735
:1027500003D51BF0080F40F09380A10704D52B6828
:10276000DB689A0740F08880630602D51AF0100FE4
:1027700055D1A70602D51AF0080F64D1E00603D59B
:102780002B681B69990765D1A20302D518F0100FB9
:1027900064D1E30302D518F0080F66D1270405D5EC
:1027A00018F0040F14D12B6804225A60002E42D175
:1027B000BDE8F88F01229A60BB076CD47E0700F158
:1027C000868017F0080600F095804FF480569DE74C
:1027D000E00504D519F0010F18BF46F00106A10568
:1027E00004D519F0020F18BF46F00206620504D5A1
:1027F00019F0040F18BF46F004062305D3D519F0CD
:102800007009D0D0B9F1400F7FD04CD8B9F1200F6A
:102810006DD0B9F1300F54D146F020064BE02B6853
:10282000102246F480661A61A3E72B68102246F452
:102830000076DA608BE76B6A1E436E6228461FF0F3
:1028400087FEBDE8F88F2B6808221A6128461FF022
:1028500079FE93E728461FF073FE95E72B68102258
:102860005A6028461FF070FE93E72B6808225A60D2
:1028700028461FF06BFE91E728461FF053FE73E7D2
:102880002B680822DA6028461FF058FE65E72846C4
:102890001FF040FE56E71FF039FE002636E72846B7
:1028A0001FF036FE40E7B9F1500F1DD0B9F1600FAF
:1028B00008BF46F480762B689A6922F070029A610C
:1028C00072E7B9F1100FF6D146F00806F3E74FF4BE
:1028D00000661BE73B0514D546F4804624E73B031E
:1028E0000BD546F480362DE746F08006E3E746F048
:1028F0001006E0E71FF010FE08E728461FF010FE64
:1029000020E728461FF00AFE0EE746F04006D2E711
:10291000406A704790F82030012B09D090F82030A1
:10292000022B05D0436A43F48023436201207047A1
:1029300000234362184670470B4B01E0013B10D067
:102940000269002AFADA0369074A43F001030361C6
:1029500001E0013A05D0036913F00103F9D11846EB
:1029600070470320704700BF400D030084B070B56E
:102970000A9E05AD012E85E80E00044623D1836B27
:10298000119A23F480338363C36823F4840323F010
:102990004003C360C368012A23F44013C3601CD002
:1029A0002046FFF7C9FF089B012B07D1A36843F01E
:1029B0000603A360A36843F02003A360BDE8704052
:1029C000002004B07047C36843F04003C360FFF7C2
:1029D000B3FF4FF48033A363E5E7C36843F4801388
:1029E000C360DDE7034600209A6842F001029A6066
:1029F000704700BF034600209A6822F001029A60E7
:102A0000704700BF08B5C368012923F0C043C36005
:102A100009D019B9C36843F08043C360322004F081
:102A200011F9002008BDC36843F00053C360322091
:102A300004F008F9002008BD84B02DE9704307AC0C
:102A400084E80E00119C0A9D836B002C40F08B8063
:102A500043F4001383630023C0F8003E0C9BD0F8BE
:102A60000028C0F80028012B00F5006600F08E80D9
:102A7000D0F8003843F00303C0F800384FF4846303
:102A80000361494B01E0013B02D002699206FAD48E
:102A900010230361444B01E0013B02D00269D206DE
:102AA000FAD400224FF0FF3332617261B361F261F8
:102AB00091B3964600F510634FF090494FF0FF0830
:102AC000D3F800C00132BCF1000FB4BFC3F80090CE
:102AD000C3F800E08A42C3F810E0C3F8088003F1AD
:102AE0002003EDD10022964600F530634FF0904967
:102AF0004FF0FF08D3F800C00132BCF1000FB4BFA3
:102B0000C3F80090C3F800E08A42C3F810E0C3F8AD
:102B1000088003F12003EDD13369012D23F4807384
:102B2000336124D000226FF08043826143611DB97C
:102B3000836943F01003836181691C4B0D9A0B4339
:102B400083611AB1836943F008038361012C05D1C5
:102B5000836943F0804343F004038361BDE870431D
:102B6000002004B0704743F40023836373E7104BE5
:102B70003363336B43F4803343F003033363002246
:102B80006FF08043316B82614361D5E7099B23B9C4
:102B9000D0F80038C0F8003870E7D0F8003843F0BB
:102BA0000103C0F8003869E7400D030000383C809D
:102BB00000018000890141F02001064A016101E025
:102BC000013A05D0036913F02003F9D11846704784
:102BD00003207047400D030000F50063D0F808089B
:102BE00010F0060012D09A6802F00602022A0CD0F9
:102BF0009A6802F00602062A07D09B6803F00603D3
:102C0000042B14BF0020022070470320704700BF30
:102C100030B44B78012B20D00C78D0F81C584FF4EE
:102C2000803300F50062A34000F530602B4300EBD9
:102C30004410D36103681B040CD48B680468CA7801
:102C4000C3F30A03234343EA824343F0805343F42C
:102C500000430360002030BC70470A78D0F81C584D
:102C6000934000F500649BB200F510602B4300EB2D
:102C70004210E36103681C04ECD48B680468C978D3
:102C8000C3F30A03234343EA814343EA825343F0F5
:102C9000805343F40043036030BC0020704700BF02
:102CA00070B44B78012B28D00D782B4A00F5306199
:102CB00001EB45114FF000660B684FF0804423F4A0
:102CC00000430B600E600C6001E0013A41D08B685C
:102CD00013F01003F9D1D0F8044844F48064C0F82C
:102CE000044800F500624FF48030D169A84021EA21
:102CF000000170BC1846D16170470C78164B00F586
:102D0000106101EB44114FF000660A684FF08045F6
:102D100022F400420A600E600D6001E0013B18D011
:102D20008A685500FAD44FF4846303610A4B01E0CA
:102D3000013B02D002699206FAD40123D0F81C2884
:102D4000A3409BB222EA0303C0F81C3870BC0020E9
:102D50007047032070BC7047400D03002DE970439D
:102D60004C78012C49D00D784C6900F5306303EBA9
:102D700045131D69ED0CED041D611D6925F0FF551E
:102D800025F4C0151D616CB38D68654ED3F810C075
:102D90002C44013CB4FBF5F406EAC44646EA0C06B2
:102DA0001E61A4B205FB04F41D69C4F312042C4394
:102DB0001C61012A04BFCA685A61CA78012A0AD173
:102DC000D0F8082812F4807F1A680CBF42F0005235
:102DD00042F080521A601A6842F004421A600020E1
:102DE000BDE870838C681D69C4F312042C431C6118
:102DF0001C6944F400241C61DBE74D690E78DDB3E7
:102E000000F5106303EB4613D1F80890D3F8108057
:102E1000DFF80CC14FEAD8484FEAC848C3F8108021
:102E2000D3F8108028F0FF5828F4C018C3F8108099
:102E3000D3F8108005EB090E0EF1FF3EBEFBF9FE44
:102E40000CEACE4C4CEA080CC3F810C0D3F810E0E2
:102E5000C5F3120C4CEA0E0CC3F810C091F803C075
:102E6000BCF1010F4CD0012A57D0B440D0F83468DF
:102E70003443C0F83448AEE700F5106303EB461363
:102E8000012A1C6924F0FF5424F4C0141C611C693D
:102E900044F400241C611C694FEAD4444FEAC44442
:102EA0001C6191F803C024D0BCF1010F93D1D0F87C
:102EB000084814F4807F1C680CBF44F0005444F0B0
:102EC00080541C601C6844F004441C60002A86D1B5
:102ED000ADB20335AD0882D0CB6800F5805003EB6E
:102EE000850100EB063653F8042B32609942FAD183
:102EF00075E70C695C61BCF1010F7FF46CAFD6E73C
:102F00001C6924F0C0441C611C69012A44F000546F
:102F10001C61CCD10C695C61C9E70A695A615AE746
:102F20000000F81F4B78012B70B427D00B784C6948
:102F300000F5306000EB43100369DB0CDB04036138
:102F4000036923F0FF5323F4C01303618B689CB91A
:102F5000046944F4002404610469C3F312032343A5
:102F6000012A036104BFCB684361036843F0044353
:102F70000360002070BC70474B61E9E74C690E7834
:102F8000002C32D000F5106303EB4613D1F808C0D3
:102F90001D69ED0CED041D611D6925F0FF5525F43B
:102FA000C0151D611D69644545F4002588BFC1F841
:102FB00014C01D611D6988BF6446C4F312042C430C
:102FC0001C611C68012A44F004441C6027D04B6932
:102FD000002BCED0D0F83428012303FA06F616438E
:102FE000C0F83468002070BC704700F5106303EB34
:102FF0004613012A1C6924F0FF5424F4C0141C61F8
:103000001C6944F400241C611C694FEAD4444FEA53
:10301000C4441C611C6844F004441C60D7D10A6994
:103020005A61002070BC704710B49DF804406CB920
:1030300003339B080AD000F5805000EB023201EB0D
:10304000830351F8040B10608B42FAD100205DF825
:10305000044B7047033292080CD010B400F5805432
:1030600001EB8200236841F8043B8842FAD15DF805
:10307000044B7047084670474B78012B0B7810D0F3
:1030800000F5306000EB43100368002B03DB03689E
:1030900023F080430360036843F4001303600020BF
:1030A000704700F5106000EB43100368002BEEDA68
:1030B000F1E700BF4B78012B0B780CBF00F51060D7
:1030C00000F5306000EB4310036823F40013036045
:1030D000CB78023B012B03D8036843F08053036095
:1030E00000207047D0F8003823F4FE63C0F80038A1
:1030F000D0F80038090101F4FE611943C0F8001846
:103100000020704708B5D0F8042822F0020200F52C
:10311000006303205A6003F095FD002008BD00BF46
:1031200008B5D0F8042842F0020200F5006303203D
:103130005A6003F087FD002008BD00BF4269806926
:1031400010407047D0F8183800F50060C06918408A
:10315000000C7047D0F8183800F50060C0691840BE
:1031600080B2704700F5306303EB411100F5006059
:103170008A6840691040704710B4D0F81048D0F801
:10318000342800EB411000F5106022FA01F1CB0168
:103190008068DBB2234318405DF8044B704700BFE2
:1031A000406900F001007047D0F8003923F4FF6354
:1031B00023F0070300F50062C0F80039936803F0BC
:1031C0000603042B05D1D0F8003943F00303C0F8FF
:1031D0000039536843F4807353600020704700BF88
:1031E00010B40024C0F8104BD0F8104B44F4002465
:1031F000C0F8104BD0F8104B44F01804C0F8104B36
:10320000D0F8104B012944F0C044C0F8104B05D150
:103210004FF08021C0F8142BC0F8001B00205DF88F
:10322000044B704730B589B00023702501240C226F
:1032300001A9CDE90154CDE90333CDE90533079365
:1032400007F026FC09B030BD30B51848184B0360B4
:103250008DB04FF6FF72002301240325C26003A93D
:103260000422C0E9013303610493069308930A938F
:1032700003950594099407920B9207F0B3FA48B9A5
:1032800000230A4801A9CDE9013300F093FB30B9CE
:103290000DB030BD0748EA2101F0C0F9F0E705485C
:1032A000F12101F0BBF90DB030BD00BFA4C6002074
:1032B00000040040388F020830B51948194B0360EC
:1032C0008DB04FF6FF72002301240325C26003A9CD
:1032D0000422C0E9013303610493069308930A931F
:1032E00003950594099407920B9207F07BFA48B96D
:1032F00000230B4801A9CDE9013300F05BFB38B98D
:103300000DB030BD084840F20B1101F087F9EFE72E
:1033100005484FF4897101F081F90DB030BD00BF4F
:103320002CC6002000080040388F020810B5224843
:10333000224B036086B000234FF0FF32C0E9013317
:10334000C260036107F032FAE8B900231A486946FF
:10335000CDE9003300F02EFB40BB0A2201200024FF
:103360000F230292039002A913480822CDE90443D7
:1033700007F0C8FAA0B9104802A90C2207F0C2FA57
:1033800038B906B010BD0E4840F2231101F046F9DD
:10339000DBE70B484FF49C7101F040F906B010BD1B
:1033A000074840F2331101F039F9E4E704484FF4DB
:1033B000957101F033F9D0E768C60020000C004099
:1033C000388F02080A4808B50A4B036042F6031218
:1033D0000023C0E90133C260036107F093F900B92B
:1033E00008BDBDE80840044840F2851101F016B957
:1033F000E0C60020001C0040388F020800B51B4AC0
:103400000368934283B005D0194A934218D003B0A1
:103410005DF804FB0022174B0092596C41F001014A
:1034200059645B6C03F00103009311461920009B63
:10343000FEF7AAFD192003B05DF804EBFEF7DCBD32
:1034400000220C4B0192196C41F0800119641B6C35
:1034500003F08003019311462C20019BFEF794FD9D
:103460002C2003B05DF804EBFEF7C6BD0000014060
:10347000001C00400038024000B50368B3F1804FE3
:1034800083B005D0194A934212D003B05DF804FB13
:1034900003F50E33002200921A6C42F001021A6406
:1034A0001B6C03F001030093009B03B05DF804FB69
:1034B00000220F4B0192596C41F0020159645B6C80
:1034C00003F00203114601932C20019BFEF75CFDE3
:1034D0002C20FEF791FD002211462D20FEF754FD11
:1034E0002D2003B05DF804EBFEF786BD000401401B
:1034F0000038024030B51B4A0368934289B004D0BB
:10350000194A93421BD009B030BD02F50D32002399
:103510000193116C154841F002011164126C05937E
:1035200002F002020192019D3024022203A9CDE99A
:1035300003420693079207F079FD09B030BD02F50A
:103540000C3200230293116C084841F0040111640D
:10355000126C059302F004020292029DC024022222
:1035600003A9E4E700040040000800400004024012
:10357000144B02689A4200D0704730B587B00024DF
:1035800003F50B3300941A6C0F4842F008021A64DA
:103590001B6C039403F0080300930C22022301A97F
:1035A000CDE901230593009D049407F03FFD2246D9
:1035B00005213220FEF7E8FC3220FEF71DFD07B0A2
:1035C00030BD00BF000C00400000024070B5294A29
:1035D0000368934286B007D0B3F1804F1FD0264ACC
:1035E00093422CD006B070BD4FF46043234801A92C
:1035F000022600240125CDE90136CDE903440595D5
:1036000007F014FD1E4801A94FF4E063CDE9026400
:10361000CDE90445019307F009FD06B070BD002314
:103620000122164805924FF44065022401A9CDE914
:103630000154CDE9033307F0F9FC06B070BD8023D7
:1036400003250F48059501A902260024CDE901367E
:10365000CDE9034407F0EAFC0848059501A9CDE946
:103660000156CDE9034407F0E1FC064801A94FF4F7
:10367000E073CBE700000140000401400004024079
:10368000000002400008024030B55248524B03602F
:1036900095B00023602440F6AC510222C0E90241FB
:1036A00042614360036107F02DF800285BD14FF4BD
:1036B00080534848029302A906F04EFE002840F0CD
:1036C0008380444807F056F8002878D1414807F035
:1036D00035F800286ED1202200233E486946CDE906
:1036E000002300F067F900285FD1002270233948D9
:1036F000069306A9CDE90722CDE90922CDE90B22DF
:1037000007F0F6F900284BD13248042206A907F049
:10371000EFF900283FD12F48082206A907F0E8F961
:10372000002833D100232B48069306A90C2207F06A
:10373000AFF930BB4FF4006000234FF480651424D0
:103740004FF400520D900DA922481193CDE90E536C
:1037500013931094129200F053F948B91D48FFF7E3
:1037600035FF15B030BD1D48652100F057FF9EE7BD
:10377000A4211A4800F052FF1648FFF727FF15B0A2
:1037800030BD1648982100F049FFD3E71348922135
:1037900000F044FFC6E711488D2100F03FFFBAE773
:1037A0000E48882100F03AFFAEE70C487C2100F07B
:1037B00035FF9AE70948752100F030FF8BE707488D
:1037C000702100F02BFF81E704486B2100F026FFF9
:1037D00077E700BF1CC7002000000140388F0208B7
:1037E00010B5264800238AB04FF0804460214FF482
:1037F0008052C0E9021204604360036106F0BAFF20
:1038000020BB00231D4801A9CDE9013300F0D2F807
:1038100078BB702000230224039003A91748049367
:1038200008220793059407F063F9E8B941F201040F
:103830000023124803A90C22CDE9044307F058F9EC
:1038400048B90E48FFF7C2FE0AB010BD0C48B721B8
:1038500000F0E4FED5E7CE21094800F0DFFE07487E
:10386000FFF7B4FE0AB010BD0548C72100F0D6FE30
:10387000DCE70348BE2100F0D1FECAE758C70020AC
:10388000388F020830B53C483C4B036091B00023B0
:10389000602440F6AC510222C0E90241426143601B
:1038A000036106F067FF00283ED120220023324842
:1038B0006946CDE9002300F07DF8002856D10022AA
:1038C00070232D48029302A9CDE90322CDE90522F8
:1038D000CDE9072207F00CF9002841D1264804223F
:1038E00002A907F005F9002834D1234802A90822CB
:1038F00007F0FEF840BB4FF4006000234FF48065F2
:1039000014244FF40052099009A91B480D93CDE9E6
:103910000A530F930C940E9200F072F850B91648A7
:10392000FFF754FE11B030BD154840F24B1100F0C6
:1039300075FEBAE74FF4BA71114800F06FFE0E48F9
:10394000FFF744FE11B030BD0D484FF4B47100F0E4
:1039500065FED0E70A4840F2631100F05FFEC4E75D
:1039600007484FF4AF7100F059FEB7E704484FF431
:10397000A97100F053FEA2E7F0C500200004014049
:10398000388F020803680422186A02FA01F120EA5B
:10399000010018621A6A114319625A6C42F400421B
:1039A0005A641A6842F001021A600020704700BF92
:1039B000FFF7E8BF90F83830012B1ED002460220F6
:1039C000136870B482F839005C6824F07004D1E99F
:1039D00000565C60586828435860986820F0800062
:1039E00098609968002401253143996082F8395024
:1039F00082F83840204670BC70470220704700BFF4
:103A000090F83830012B22D030B4D1E9025304466B
:103A100023F44073D1E900202B4323F48063034354
:103A200023F40063D1E90450134323F480532B4360
:103A300023F4005389692268034323F440430B4372
:103A40000021536484F83810084630BC70470220C7
:103A5000704700BF704700BF704700BF30B40568B3
:103A60006B6A29B943EA0243AB62002030BC70475D
:103A7000A86A4C1E03EB10400CD0002319464031BD
:103A800005EB810101334968DBB2A34200EB114031
:103A90001946F4DB403405EB840440EA02406060E0
:103AA000002030BC704700BF036800205962704797
:103AB00000B583B01B4B00220092196B41F400113A
:103AC0001963196B01F40011009100990192196BAF
:103AD00041F4800119631B6B03F4800301930521FA
:103AE0000B20019BFEF750FA0B20FEF785FA00220F
:103AF00005210D20FEF748FA0D20FEF77DFA002281
:103B000005210F20FEF740FA0F20FEF775FA00227C
:103B100005211020FEF738FA102003B05DF804EB01
:103B2000FEF76ABA003802402DE9F04180460F46A0
:103B300016461D46D8F8003001E06A1C0AD19C6880
:103B400037EA04020CBF01240024A642F5D100206C
:103B5000BDE8F0813DB103F06FF8069BC01AA842A2
:103B6000E8D3D8F800305A68D8F8041022F0E00200
:103B7000B1F5827F5A6016D0D8F82820B2F5005FE0
:103B800007D00122002388F8512088F85030032004
:103B9000DEE71A684DF6FF710A401A601A6842F4AF
:103BA00000521A60EDE7D8F80820B2F5004F02D0B5
:103BB000B2F5806FE0D11A6822F040021A60DBE7AC
:103BC00000283BD070B590F851200023044602F045
:103BD000FF01836262B31846D4E90135D4E90321B9
:103BE0002B4313436269E569266A0B431343A269B9
:103BF00021682B43022584F85150334302F40075A9
:103C00000E682B43120C656A02F0040203432A4338
:103C100026F040060E600B604A60CB69002223F458
:103C200000630125CB61626584F85150104670BD78
:103C300080F8501000F0A6FEA06ACDE70120704782
:103C400090B10268022310B580F85130136823F058
:103C500040030446136000F01FFF0020606584F8F5
:103C6000500084F8510010BD012070472DE9F04349
:103C7000044690F85000012885B067D01D46012306
:103C800084F850300E46914602F0D6FF94F8513039
:103C9000012B07465FFA83F80BD04FF00208012290
:103CA0000023404684F8512084F8503005B0BDE828
:103CB000F083002EF3D0B9F1000FF0D0032384F885
:103CC0005130A268266300236365C4E91033A4F869
:103CD0003690A363E387A3872368A4F83490B2F5F2
:103CE000004F02BF1A6842F480421A601A685206F6
:103CF00003D41A6842F040021A60E268B2F5006F1D
:103D0000626829D0002A4CD0E28E92B2012A48D0B3
:103D1000E38E9BB25BB94CE016F8012B1A73E38E6D
:103D2000013B9BB2E386E28E92B2002A41D0236827
:103D30009A689207F0D435B16B1CF4D002F07CFF86
:103D4000C01BA842EFD34FF00308A8E74FF00208CA
:103D5000404605B0BDE8F083002A4BD136F8022B6F
:103D6000DA60E28E013A92B2E286E28E92B25AB9FB
:103D70001FE036F8022BDA60E38E013B9BB2E3864C
:103D8000E38E9BB2ABB123689A689007F1D4002D03
:103D9000D9D0691CF4D002F04FFFC01BA842EFD36A
:103DA000D1E716F8012B1A73E38E013B9BB2E38631
:103DB000AEE700972B46012202212046FFF7B4FE12
:103DC0000028C0D1024600972B4680212046FFF7ED
:103DD000ABFEA0B9A36833B922680393D3680393F9
:103DE00093680393039B636DB3F1000818BF4FF012
:103DF000010854E7E28E92B2012AB6D1AEE7636DB4
:103E0000202213436365626549E700BF2DE9F04353
:103E1000044690F8500085B001280C9F00F0858082
:103E20009946012384F850300E46154602F004FFEF
:103E300094F851206368012A8046D1B211D0B3F5BD
:103E4000827F09D002200122002384F8512084F8C7
:103E5000503005B0BDE8F083A268002AF2D10429F1
:103E6000F0D1002E65D0002D63D0B9F1000F60D0E5
:103E700094F851202168012A04BF052284F85120BA
:103E800000226265A4F83E90A4F836900868A56305
:103E9000C4E910224206A4F83C902663A4F83490AA
:103EA00003D40A6842F040020A60E268B2F5006F8B
:103EB00041D0002B70D0E38E9BB2012B6CD04FF021
:103EC0000109E38E9BB21BB9E38F9BB2002B43D059
:103ED000B9F1000F0FD0E38E9BB263B123689A68EB
:103EE000920708D516F8012B1A73E38E013B9BB29B
:103EF0004FF00009E386E38F9BB263B121688B68C2
:103F000013F0010307D0CA6805F8012BE18F0139CE
:103F100089B29946E1877B1CD3D002F08DFEA0EBDD
:103F20000800B842CDD303208DE7022005B0BDE8DC
:103F3000F083012087E7002B62D136F8023BCB608B
:103F4000E38E013B9BB2E3864FF00109E38E9BB207
:103F500053BBE38F9BB23BBBCDF800803B460122B5
:103F600002212046FFF7E0FD0028DCD10246CDF813
:103F700000803B4680212046FFF7D6FD002844D133
:103F8000A368002B7FF45FAF23680390DA68039285
:103F90009B680393039B56E716F8013B0B73E38E74
:103FA000013B9BB2E3868AE7B9F1000F0FD0E38EA5
:103FB0009BB263B123689A68900708D536F8022B44
:103FC000DA60E38E013B9BB2E3864FF00009E38F9A
:103FD0009BB263B12268936813F0010307D0D268E3
:103FE00025F8022BE28F013A92B29946E287791CBA
:103FF000ACD002F021FEA0EB0800B842A6D392E7B5
:10400000E38E9BB2012B9FD197E7636D2022134370
:1040100063650120626516E770B5044690F85000AC
:10402000012865D094F851000125A842C6B284F851
:1040300050500DD06068B0F5827F04D0022000237C
:1040400084F8503070BDA0680028F7D1042EF5D157
:1040500000294BD0002A49D0002B47D094F85100BA
:104060002163012804BF052084F851000020606509
:10407000E386E38794F85150A386042DA387C4E90F
:10408000100007BF1B491C4B1C491D4BE06CA26371
:104090001C4DC0E90F31E38F2168C56400259BB238
:1040A0000C31056501F090F92268A06C5368216B12
:1040B00043F001035360E38E05640C329BB2C0E908
:1040C0001355C56301F080F923681A68520603D4BA
:1040D0001A6842F040021A605A6842F020025A60A0
:1040E0005A6842F002025A600020A8E70120A6E7C1
:1040F000022070BD1141000855410008214100080F
:10410000A541000831410008704700BF704700BF5B
:1041100008B5806BFFF7FAFF08BD00BF704700BF0E
:1041200008B5806BFFF7FAFF08BD00BF704700BFFE
:10413000806B026808B5536823F003035360436D36
:10414000012143F01003436580F85110FFF7EEFFA3
:1041500008BD00BF08B50368806B1B68DB050FD482
:10416000D0E900215368B1F5827F23F00303536047
:1041700009D001230022C28780F85130436D73B902
:10418000FFF7C2FF08BD8368B3F5004F02D0B3F557
:10419000806FEED1136823F040031360E9E7FFF767
:1041A000C5FF08BD30B5054683B0846B02F044FD01
:1041B0002B681A6812F4807213D100906423802156
:1041C0002046FFF7B1FC88B921684B68002223F034
:1041D000030301204B60E286E28784F85100636D9F
:1041E0006BB9204609F0DCFA03B030BD636D43F0D3
:1041F00020036365636D43F020036365E4E72046B5
:10420000FFF794FF03B030BD026830B55168936882
:1042100003F04105012D85B0044656D09D0701D518
:10422000080659D413F4B07F4DD08D064BD55806EF
:104230000ED594F85100032854D0606D002540F04D
:10424000040060650095D068009090680090009828
:104250009D060CD5606D002540F00100606502955B
:1042600090680290106820F0400010600298D80515
:1042700008D5636D002043F00803636503909368DD
:104280000393039B636DF3B1536823F0E003536022
:1042900001208B0784F8510012D05368E06C23F0A2
:1042A0000303536018B1134B036501F017F9A06CB9
:1042B00048B1104B036505B0BDE8304001F00EB9C0
:1042C0002046FFF733FF05B030BD4D06A6D5036C81
:1042D00005B0BDE830401847636C204605B0BDE826
:1042E0003040184700230193D368019393680193EA
:1042F000019BE8E7F942000808B5806B0023C387FB
:10430000C386FFF713FF08BD38B5084C084D206879
:104310004FF0FF3104F05AFB0028F8D1284601F095
:10432000CFFB4320FDF768FEF1E700BFA4C70020E4
:10433000B0C7002008B502F00BFF0DF0A5FD034B40
:104340001868BDE8084005F0F5B800BF94C7002024
:1043500030B5074D0FCD87B001AC0FC42B6823607B
:10436000002101A804F056FA024B186007B030BDD6
:10437000708E0208A8C7002070B58AB00024012101
:104380006846009404F00CFB1E4B1F4E186021463B
:1043900004F01CFB012101A8019404F001FB1B4B5C
:1043A00002940246012102A81A6004F0F9FA184B9F
:1043B0002146186004F00AFB012103A8039404F0CD
:1043C000EFFA144B04940246012104A81A6004F089
:1043D000E7FA114B2146186004F0F8FAFFF7B8FF2E
:1043E0000EF014FA0DF0DAFA0FCE05AD0FC53368F2
:1043F0002B60214605A804F00DFA084B18600AB09E
:1044000070BD00BFA4C70020848E020898C700209A
:10441000A0C700209CC70020ACC7002094C7002084
:1044200010B5144C144A2368934205D0134A9342A2
:1044300006D02A2B0ED110BD114B00BF013BFCD181
:10444000104B2360104B83F30888104B1B68984770
:104450002368EEE72A232360BFF34F8F0C490D4BEF
:10446000CA6802F4E0621343CB60BFF34F8F00BF12
:10447000FDE700BF0406002075FEADDEEFBEADDE39
:1044800000A86100EDFEFECA000002200400FF1F2C
:1044900000ED00E00400FA0570B594B0294A2A4BFB
:1044A00000200190116C41F080511164126C02F0F7
:1044B00080520192019A02901A6842F480421A6076
:1044C0001B6803F48043029309224FF480330120D8
:1044D00002244FF48001042508920993A82207239F
:1044E0000D9008A8CDE90F15029E0E94129411921A
:1044F000139302F0B7FE00B1FEE74FF4A0524FF461
:10450000805305900F26052103A80494CDE90623C6
:10451000039603F097F8044600B1FEE703F02CF988
:104520000A4AA2FB00239809FDF780FD2846FDF703
:1045300097FD224631464FF0FF30FDF725FD14B0C0
:1045400070BD00BF0038024000700040D34D6210C3
:104550002549264B264A1B685288264870B50C68A8
:104560002549264D234442EA03421B0CC0E900239F
:1045700001F10C040846C3F303361B01AE5D00F8DD
:10458000016BA04243EA12734FEA0212F3D10023F7
:104590000B7302F02BFBFFF77FFF04F0F7FCFFF734
:1045A00087FA01F0CBFE01F01BFFFFF76DF8FFF774
:1045B00069F9FEF749FEFEF77FFE00F0B9F901F058
:1045C00063FFFFF70DF900F01FFCFEF7AFFEFEF7EB
:1045D000F9FE0B48FEF726FE0A48FEF723FEFFF71A
:1045E000CBFE04F009F9FEE7187AFF1F107AFF1FCF
:1045F000147AFF1F98BE0020A0BE0020708F020812
:104600001CC70020F0C50020034B02689A4200D06E
:10461000704702F005BB00BF00200040FEE700BF6E
:104620000368B3F1A04F00D0704730B587B04FF4A6
:10463000C050002403220A2301A90190022510483A
:10464000CDE90423CDE9025406F0F0FC0D4B5A6B82
:1046500042F080025A6300945A6C42F480425A64D9
:104660005B6C03F480432246009305214320009BAA
:10467000FDF78AFC4320FDF7BFFC07B030BD00BF4B
:10468000000002400038024070B5D0F8EC5382B010
:1046900005F5027600F56F7104463046019102F08F
:1046A000C7F995F80832019903F06003402B03D154
:1046B00095F80932502B06D0D4F8EC0302B0BDE8CF
:1046C000704000F09BBCD5F81432B5F80E229B6800
:1046D000C5F8F82101223146C5F8F421284698474B
:1046E000B5F80E3203B908B102B070BD284602B069
:1046F000BDE87040FDF7ECBCC1EBC10300EB8303E8
:10470000D0F8EC03D3F8042200F0A8BCC1EBC1033D
:1047100000EB8303D0F8EC035A6C00F0D3BC00BF6D
:10472000D0F8EC0300F05ABD10B5C168044600395A
:10473000D0F8EC0318BF012100F03AFDD4F8EC03E7
:10474000BDE8104000F014BD10B50446D0F8EC03ED
:1047500000F032FD2268D2F8003E43F00103C2F8B7
:10476000003E236A23B1034A136943F00603136131
:1047700010BD00BF00ED00E0D0F8EC0300F026BD56
:10478000D0F8EC0300F03ABDD0F8EC0300F034BDF3
:10479000D0F8EC0300F034BDD0F8EC0300F032BDEB
:1047A00002780AB10020704738B5194B0221C3F8CE
:1047B000EC034FF0A0450624C0F820321846C3E9A8
:1047C0000422C3E90722C3E90B22C3E900545A6259
:1047D000D960996101F0F2F8A0B980210C48FFF787
:1047E00063F9402200210A48FFF738F940220121ED
:1047F0000748FFF733F9402203210548FFF72EF958
:10480000002038BD03484FF4AC71FFF707FFE4E721
:10481000B0C70020848F020808B5D0F8200201F04C
:1048200039F9032896BF024B0220185C08BD00BF6F
:10483000A08F020810B51446D0F820021A4623466D
:1048400001F05EFC032896BF014B0220185C10BDEE
:10485000A08F020808B5D0F8200201F091FC0328CF
:1048600096BF024B0220185C08BD00BFA08F020853
:1048700008B5D0F8200201F009FD032896BF024BCD
:104880000220185C08BD00BFA08F020808B5D0F850
:10489000200201F02BFD032896BF024B0220185C7A
:1048A00008BD00BFA08F02080A06D0F8203206D447
:1048B000C1EBC10103EB810191F8FA01704701F0EE
:1048C0007F01C1EBC10103EB810191F83A00704710
:1048D00008B5D0F8200201F001FC032896BF024B76
:1048E0000220185C08BD00BFA08F020808B5D0F8F0
:1048F000200201F0A7FC032896BF024B0220185C9F
:1049000008BD00BFA08F020808B5D0F8200201F052
:1049100067FC032896BF024B0220185C08BD00BF4D
:10492000A08F020808B5D0F8200201F081FC08BD74
:10493000114838B5114B03604FF4827201234FF4D4
:1049400000654FF400741821426043610A2200237D
:10495000C0E90641C0E90833C560C26283600361F3
:104960008362FFF72DF900B938BDBDE8384004482F
:104970005221FFF753BE00BFA0CB0020003C0040F7
:10498000A48F02083D4B02689A4200D0704770B570
:1049900086B0002503F5FE3300951A6C384E42F4BC
:1049A00000421A641B6C03F4004300934FF4E0537D
:1049B0000446022201930123324800990292039394
:1049C0000322062301A90492059306F02FFBE36856
:1049D0002D48756040214FF48062F5603060B16011
:1049E0003261002B32D1C6E9053300234FF4803207
:1049F0002348F361C6E9082300F010FC002838D1F1
:104A0000224DE2682248A66400234FF48061C5E984
:104A10000133B46328602961EB60F2B9C5E905226E
:104A200000234FF480321948EB61C5E9082300F0F8
:104A3000F5FBC8B900220521E5643320AC63FDF71E
:104A4000A3FA3320FDF7D8FA06B070BD4FF4006228
:104A50004FF40053C6E90523C7E74FF400624FF453
:104A60000053C5E90523DBE70A489B21FFF7D6FD84
:104A7000E0E708488421FFF7D1FDC1E7003C004092
:104A8000F8CB0020000802408860024058CC00208B
:104A900010600240A48F02080D4B02689A4200D0B9
:104AA00070470C4A136C10B523F40043044613649A
:104AB0004FF4E051084806F0E1FBA06C00F048FC20
:104AC000E06C00F045FCBDE810403320FDF7A0BAD3
:104AD000003C004000380240000802400A4B1B68BE
:104AE000013308D04FF0500383F31188BFF36F8F69
:104AF000BFF34F8FFEE74FF0500383F31188BFF3EE
:104B00006F8FBFF34F8FFEE700000020064800685C
:104B1000006880F3088862B661B6BFF34F8FBFF3B9
:104B20006F8F00DF00BF000008ED00E0DFF80C0031
:104B3000016841F4700101607047000088ED00E0F9
:104B400030B421F00101094C40F80C4C4FF0807555
:104B50006FF0020340F8045C40F8081C40F8202C79
:104B600040F8243C30BC4438704700BFDD4A0008A0
:104B7000074B19680868B0E8F04F80F30988BFF365
:104B80006F8F4FF0000080F311887047AFF3008003
:104B9000EC0600204FF0500383F31188BFF36F8FB2
:104BA000BFF34F8F0A4A13680133012B136000D003
:104BB0007047084B1B6813F0FF0FF9D04FF05003FC
:104BC00083F31188BFF36F8FBFF34F8FFEE700BFF2
:104BD0000000002004ED00E0084A136843B94FF0DC
:104BE000500383F31188BFF36F8FBFF34F8FFEE73E
:104BF000013B13600BB983F311887047000000205C
:104C0000EFF30980BFF36F8F154B1A681EF0100F7A
:104C100008BF20ED108A20E9F04F10604DF8043DE8
:104C20004FF0500080F31188BFF34F8FBFF36F8FA9
:104C300004F0FEFE4FF0000080F3118808BC1968F4
:104C40000868B0E8F04F1EF0100F08BFB0EC108AF3
:104C500080F30988BFF36F8F704700BFAFF3008008
:104C6000EC06002008B54FF0500383F31188BFF322
:104C70006F8FBFF34F8F04F02FFD18B1034B4FF030
:104C800080521A60002383F3118808BD04ED00E010
:104C9000064B07491B680748074AA1FB03139B09FA
:104CA000013B072103601160704700BFF401002041
:104CB000D34D621014E000E010E000E0324B334AC4
:104CC0001968914256D01A68314B9A4249D010B5B2
:104CD000304B314C1A78314982B0D2B2FF20019268
:104CE00018701B78DBB28DF803309DF803309DF807
:104CF000032003F0500307202370140608600ED52C
:104D000006229DF803305B00DBB28DF803309DF87E
:104D100003000006134602F1FF32F2D40B600B6869
:104D200001981C4C1E4A1B02C0B203F4E0630B60E6
:104D30002070136843F470031360136843F07043EA
:104D40001360FFF7A5FF174B00221A60FFF7EEFE76
:104D5000154A136843F040431360FFF7D7FEFFF78F
:104D6000BDFE4FF0500383F31188BFF36F8FBFF385
:104D70004F8FFEE74FF0500383F31188BFF36F8F1F
:104D8000BFF34F8FFEE700BF00ED00E071C20F419F
:104D900070C20F4100E400E0240600202806002035
:104DA00020ED00E00000002034EF00E0EFF3058389
:104DB0000F2B0ED91049114A5B5C12789A4208D920
:104DC0004FF0500383F31188BFF36F8FBFF34F8F02
:104DD000FEE70B4B0B4A1B68126803F4E063934237
:104DE00008D94FF0500383F31188BFF36F8FBFF3DF
:104DF0004F8FFEE7704700BFF0E300E0240600207D
:104E00000CED00E0280600200C4808B50C4B0360B0
:104E10004FF4E13100230C22C0E90233C0E906332C
:104E200041604261036102F04BFE00B908BDBDE87C
:104E3000084004484E21FFF7F1BB00BF18CD002009
:104E4000004C0040B88F0208394B02689A4200D0EB
:104E500070472DE9F04387B0002503F5F633009540
:104E60001A6C344E42F400221A641B6C03F40023C3
:104E700000930227012301A94FF003094FF008080E
:104E800004462D48009A0193CDE90277CDE90498B4
:104E900006F0CCF8CDE901772748284FCDF81480EB
:104EA00001A9CDE9035906F0C1F84FF000614FF4B4
:104EB00080624FF480733046C6E90555C6E908554F
:104EC000C6E90071B560F5603261F36100F0A6F9E2
:104ED00020BB1B4D1B4866634FF0006340214FF41D
:104EE000806228606B6028460023C5E90332C5E96B
:104EF0000533C5E90733B463A9606B6200F08EF92E
:104F000088B92563002205213420AC63FDF73CF805
:104F10003420FDF771F807B0BDE8F0830A487F211F
:104F2000FFF77CFBD5E708489121FFF777FBE8E71F
:104F3000004C0040B8CC002000000240406002401D
:104F400058CD002070600240B88F02080D4B0268F7
:104F50009A4200D070470C4A136C10B523F400231A
:104F6000044613640321094806F088F9606B00F0D9
:104F7000EFF9206B00F0ECF9BDE810403420FDF7AC
:104F800047B800BF004C004000380240000002401B
:104F900088B108B5D0F8143213B10023C0F8143228
:104FA00009B1C0F810120123027080F8FC31FFF73C
:104FB000F7FB002008BD0220704700BF19B1C0F800
:104FC0001412002070470220704700BF08B5FFF799
:104FD00023FC002008BD00BF08B5D0F814321BB177
:104FE0001B68984700B908BD022008BD08B5D0F875
:104FF00014325B689847002008BD00BF38B50446EE
:1050000000F50275284601F013FD94F80812B4F873
:105010000E32C4F8F831012201F01F039342C4F8A4
:10502000F42109D0022B13D063B101F08001204696
:10503000FFF71EFC002038BD2946204601F06EFC1B
:10504000002038BD2946204601F016FB002038BD5F
:105050002946204601F080FC002038BD10B50446EA
:1050600031B91346D0F8F421032A0DD0002010BD29
:10507000D0F814329B69002BF8D090F8FC21032A59
:10508000F4D19847002010BDD0E9431291420DD8C9
:10509000D0F814321B6923B190F8FC21032A00D107
:1050A00098472046FDF714F8002010BD891A8A425F
:1050B00028BF0A4692B2C0F80C111946FDF700F855
:1050C000D4E700BF70B5044651B91346D0F8F421B7
:1050D000022A16D094F80032012B0DD0002070BDAA
:1050E000D0F814325B69002BF8D090F8FC21032A29
:1050F000F4D19847002070BD002384F800320020CE
:1051000070BDD0E90726B24221D88369B3FBF6F51A
:1051100006FB15355DB99E4209D8D0F8F8219342B7
:1051200005D22A46FCF7B6FFC4F8F85116E0D4F8C9
:105130001432DB681BB194F8FC21032A15D02046F9
:10514000FCF7D2FF94F80032012BC7D1D4E7921BB1
:105150000D46C261194692B2FCF79CFF2B462A46C7
:1051600029462046FFF7D0FBB4E720469847E6E7FC
:1051700038B50022044640231D461146FFF75AFB6E
:105180002B460022C4F8105120468021FFF752FB25
:10519000D4F818322562012284F8FC212BB1D4F80E
:1051A000143221795B6820469847002038BD00BF43
:1051B00001740020704700BF90F8FC2180F8FD21A9
:1051C000042380F8FC310020704700BF0346002014
:1051D00093F8FD2183F8FC21704700BF90F8FC2173
:1051E000032A01D00020704708B5D0F81432DB69DB
:1051F00003B19847002008BD002070470020704789
:105200000020704708B5D0F81422012180F8FC1165
:10521000526801799047002008BD00BFF8B50446E8
:1052200001F00AFD002C54D023680222002184F8EA
:10523000341084F835201A6822F0010205461A60FD
:1052400005E001F0F9FC431B052B3BD823681A68E5
:10525000D107F6D4D4E90126D4E903503243616979
:105260001F682A43D4E9066502430A43206A354988
:1052700032432A430243606A3940042841EA02016A
:1052800029D019605A6922F007021043DAB22E4978
:105290005861103AA1FB020109092C4823F47F73DD
:1052A000415CE16523F003035F2A88BF04333F229A
:1052B0008A4001250021A3659A60616584F8355014
:1052C0000846F8BD03232022626584F8353018466D
:1052D000F8BD0120F8BDD4E90B5028430143A26A70
:1052E0001960586920F00700104340F00400002DB9
:1052F000CCD07EB1B6F5005F12D0022A03D9032AC2
:10530000C4D1EA01C2D501234022626584F8353058
:105310001846F8BD012A11D032F00202B6D1F0E7EA
:10532000032AB3D801A151F822F000BF07530008A7
:1053300003530008075300083D530008B5F1C07F30
:10534000A4D1E0E73F8010F0ABAAAAAAD08F020850
:1053500030B400282FD090F83530022BDCB227D0A3
:105360000368174A1C68174DD9B21039A2FB01C255
:10537000120924F001041C60AD5C212400221A6093
:105380005A609A60DA601A615C6123F47F7323F0DB
:1053900003035F2988BF04333F210022A940C5656C
:1053A000836514469960426580F8342080F8352082
:1053B000204630BC70470124204630BC704700BFF7
:1053C000ABAAAAAAD08F0208F0B490F83440866D38
:1053D000012C38D090F835400125AC4280F834508B
:1053E00005D0002380F83430F0BC022070470468F8
:1053F0000227002580F8357045652568876825F403
:105400008025402F256063600ABFA260A160E16033
:10541000C16D18BFE2603F238B40026CB36023680C
:1054200043F016032360636943F0800363611AB19C
:10543000236843F008032360236843F001032360DB
:105440000020F0BC70470220F0BC704770B50446E5
:10545000866D01F0F1FB94F83530022B06D0002365
:10546000802284F834306265012070BD2368216C8D
:105470001A6822F016021A605A6922F08002054664
:105480005A6131B31A6822F008021A601A6822F0D1
:1054900001021A6005E001F0CFFB431B052B0FD87A
:1054A00023681B6813F00103F5D1E16D3F228A40A8
:1054B0000121B26084F8343084F83510184670BD8C
:1054C000202200230320626584F8343084F83500FC
:1054D00070BDA26C002AD5D1D8E700BF90F8353056
:1054E000022B03D080234365012070470268052307
:1054F00080F83530136823F00103136000207047F3
:105500002DE9F04182B00023866D0193C36D3468AC
:10551000714908229A4022420D68804604D00168F1
:105520000F68780700F18A8001229A40224204D055
:10553000D8F800104969090678D404229A4022421A
:1055400004D0D8F8001009688F0767D410229A4059
:10555000224204D0D8F800100F68380749D420221E
:105560009A40224217D0D8F800100C68E00612D5F5
:10557000B26098F83520052A73D00B6813F4802F99
:105580000B6800F09080190340F19B80D8F83C3004
:105590000BB140469847D8F854303BB3D8F8543054
:1055A000DA071BD5D8F800204C49052388F8353098
:1055B0001368A1FB051523F001031360AD0A02E097
:1055C0001368DB0704D5019B0133AB420193F7D984
:1055D0000022012388F8342088F83530D8F84C3080
:1055E00023B1404602B0BDE8F041184702B0BDE823
:1055F000F081B2600A6812F4802F0A682AD1D705B8
:1056000003D40A6822F008020A60D8F84020002A71
:10561000A5D040469047D8F85C30A0E7B260D8F8F3
:10562000542042F00402C8F854208FE7B260D8F842
:10563000542042F00202C8F854207EE70F6827F099
:1056400004070F60B260D8F8542042F00102C8F895
:10565000542069E71203D8D5D8F84820002AD8D1B9
:105660007DE70A68D8F8404022F016020A604A69CD
:1056700022F080024A6154B30A6822F008020A60EC
:105680003F22D8F8501002FA03F300240122B3603D
:1056900088F8344088F835200029A7D0404602B069
:1056A000BDE8F041084713F480737FF46FAF0A68D8
:1056B000012422F010020A6088F8343088F835405E
:1056C00064E7D8F84430002B7FF463AF63E7D8F881
:1056D0004820002AD0D1D3E7F4010020B5814E1B29
:1056E00010B4154B1A461B688342FBD351685418FB
:1056F000A0420AD041684418A3420DD090420360F2
:105700005DF8044B18BF10607047406801441046B4
:105710004418A3425160F1D1084C2468A342EDD053
:10572000D3E9003490422144036041605DF8044BAA
:1057300018BF1060704700BF3C0600202C060020F8
:105740002DE9F041404F044603F0B0FF3B68002BC9
:1057500039D03E4B1D682C422FD174B304F108039D
:1057600061071CBF23F00703083333B3DFF8EC8075
:10577000D8F800609E4220D335490C6803E02068C9
:1057800020B12146044662689A42F8D33868A042A4
:1057900013D020680F680860D11A102907F1080794
:1057A00039D9E018420731D04FF0500383F3118804
:1057B000BFF36F8FBFF34F8FFEE704F03DF8002774
:1057C0003846BDE8F081234B234E214D580714BFC6
:1057D000DA1D1A4603F58033A3F1080323F007030B
:1057E0001E483B6018BF22F0070211469A1A326029
:1057F0000260164E0020C3E9000068604A604FF066
:1058000000420B60326029601546A4E74160636086
:10581000FFF766FF626810480168B61A00232A4342
:105820008E42C4E9003238BF0660C8F8006004F058
:1058300003F87B07C4D04FF0500383F31188BFF304
:105840006F8FBFF34F8FFEE72C060020300600203D
:105850003C0600200000001038060020340600201E
:10586000E0B1194A50F8043C1268134210B50446DE
:105870000BD050F8081C91B14FF0500383F31188FE
:10588000BFF36F8FBFF34F8FFEE74FF0500383F3EB
:105890001188BFF36F8FBFF34F8FFEE7704723EA86
:1058A000020340F8043C03F001FF084A54F8043CAA
:1058B0001168A4F108000B441360FFF711FFBDE865
:1058C000104003F0B9BF00BF3006002034060020AE
:1058D000014B1868704700BF380600200020704751
:1058E00008B509681CF042FC002008BD10B50C4C3E
:1058F0000C4901232046002203F0B8F90A4920464A
:10590000012203F0C7F9032308492046002203F0CF
:10591000ADF907492046032203F0BCF9002010BD71
:10592000F4D1002038CE0020B8CD002078CE002061
:10593000F8CD0020212801D000207047002310B4AA
:105940000120C22408224C7088705DF8044B0B7053
:105950000020CB700B714B718A717047402923D89E
:10596000134B012A70B5D3F818320D46144618D0DF
:10597000032A1BD10F4E5C331B7A83B901462A469A
:1059800030461EF0F7F9314623462A46084803F010
:105990006DF921460648BDE8704003F08BB901203F
:1059A00070BD054E4433E7E702207047022070BD0A
:1059B000F4D1002078CE002038CE0020002866D018
:1059C000F0B5032305468BB080F8B9330446FEF7E3
:1059D00027FE2868FDF70EF854F810CB26460FCEA8
:1059E0006F460FC70FCE0FC796E8030087E8030086
:1059F0002E1D96E80E006046FCF7B8FF00212868CF
:105A0000FDF700F8002108462B462A46012782F8B8
:105A10003810D18701310F29C2E9100082F839709E
:105A200082F83B00D06402F11C02F0D100222F6802
:105A3000114602F1400083F8F821DA8707EB800075
:105A400001320F2AC3E9801183F8F91183F8FB11A1
:105A5000C3F80C1203F11C034160EAD10FCCEC46F1
:105A6000ACE80F000FCCACE80F0094E803008CE822
:105A70000300384696E80E00FCF7DEFF0123286895
:105A800085F8B933FDF74CFB00200BB0F0BD0120C9
:105A9000704700BF90F8B833012B0ED010B501232A
:105AA000044680F8B8330068FDF72CFB2068FCF74B
:105AB00099FF002084F8B80310BD0220704700BF92
:105AC0002DE9F04FD0F8008087B004464046FDF73E
:105AD00067FB10B107B0BDE8F08F05462068FDF701
:105AE0002DFB0028F6D02068FDF728FB10F0020FF0
:105AF00020681EBF436903F002034361FDF71EFBEC
:105B0000000300F170814FF0000B2068FDF716FBD9
:105B1000420300F1BF80D4F800A05046FDF70EFB11
:105B20000028C0F20A822068FDF708FB01054AD46C
:105B30002068FDF703FBC3046ED42068FDF7FEFA6E
:105B400010F4005F206849D1FDF7F8FA10F0100F4B
:105B5000206813D0836923F010038361D8F82050A4
:105B6000C5F34343022B05F00F0600F0F581062B29
:105B700000F0C181836943F010038361FDF7DEFA11
:105B8000070700F193812068FDF7D8FAC60200F1FB
:105B900082812068FDF7D2FA850200F171812068C8
:105BA000FDF7CCFA400000F162812068FDF7C6FAEB
:105BB00041078FD523685D686A0700F1EF815A6855
:105BC0002A435A6086E7D8F80838DA0700F1E281FC
:105BD0002068436903F400634361AAE7FDF7E4FA30
:105BE0002068C36823F47053C360FCF7F5FF0028F6
:105BF00040F070812268E060D3684FF4007143F494
:105C000010536161D3602046FEF78EFD2068436922
:105C100003F40053436197E7D8F80438206823F071
:105C200001031021C8F80438FCF7C4FF606808F5C8
:105C3000006650B108F51063FF22013585429A6075
:105C4000C3F8082203F12003F7D14FF0FF33B3610B
:105C5000F369226B43F00113F361002A40F02F81B6
:105C6000736943F00B037361336943F00B033361D2
:105C7000D8F80038217C206823F4FE63C8F8003887
:105C800004F56F72FDF7ACFA2068436903F48053A2
:105C9000436153E72068FDF75DFA8146002800F074
:105CA0003D8108F51063CDE90238D4F800A00495D1
:105CB00026464FF0000B07E05FEA59090BF1010B94
:105CC00006F11C0600F02E8119F0010FF4D05FFAE6
:105CD0008BF750463946FDF74FFAC30705461ED5E8
:105CE000039B2069012202FA0BF1D3F8342822EA3F
:105CF0000101029AC3F8341802EB4B121346012239
:105D000090429A6003D1D6E9102313447364394654
:105D10002046FEF7FBFC2169012900F0538128078A
:105D200004D5029B03EB4B1308229A60E90604D5C5
:105D3000029B03EB4B1310229A606A0604D5029B68
:105D400003EB4B1340229A60AB0704D5029B03EB95
:105D50004B1302229A602806D4F800A0ACD5D6E9ED
:105D600013130AF51068306CCDF814A008EB4B182B
:105D7000CD1A8542D8F8182028BF054692B2E81CF3
:105D8000B2EB900F19D820E0E9B1D6E91051654582
:105D900028BF6546237C0093ABB2FDF745F9D8F8E0
:105DA0001820716C336DE81C92B229442B44B2EB7D
:105DB000900F7164336506D9F16C8B42A1EB030C33
:105DC0003A465046E0D3D4F800A0002D7FF474AFDB
:105DD000059B0122D3F8341802FA0BF221EA0202E1
:105DE000C3F8342868E72068FDF7ACF906460028B8
:105DF0003FF489AE04F500774FF0000B08F53069E9
:105E000006E076080BF1010B07F11C073FF47DAEAD
:105E1000F107F6D55FFA8BF120680291FDF7A2F940
:105E200010F0010F824617D022690299012009EB78
:105E30004B138242986008D1D7E900021B69C3F373
:105E40001203C31A02443B617A602046FEF754FCF9
:105E50002169012900F0A7801AF0080F65D11AF016
:105E6000100FCED009EB4B1310229A60C9E72046E1
:105E7000FEF78EFC2068436903F08043436195E69A
:105E800020465FFA8BF1FEF77BFC2068436903F440
:105E90000013436184E620465FFA8BF1FEF774FC41
:105EA0002068436903F48013436173E62046FEF7DC
:105EB00037FC2068436903F00803436164E6D6F8C1
:105EC000843043F00B03C6F88430736C43F00B034B
:105ED0007364CDE603224023E260636101F04CFC71
:105EE0006F4B704A034493427AD82268D36843F4D4
:105EF0007053D36087E6082204F56F714046C6EB05
:105F0000C606FDF7A7F804EB8602C5F30A13D2F81C
:105F1000101220680B44C2F810322BE6D4F800A00F
:105F20008346FAE5DDE90385F7E52046FEF7ACFB9D
:105F300009EB4B1308229A6091E7D8F8042822F065
:105F400001022046C8F80428FEF716FC20684369C1
:105F500003F000434361E7E547F6F0731D423FF469
:105F600009AEC6EBC60604EB8606C5F30A12D6F8E0
:105F700004124046FDF76EF8D6F80422D6F8103227
:105F80002068C5F30A152A442B44C6F80422C6F833
:105F90001032EFE52046FEF7D7FB19E62046FEF764
:105FA000FBFB23680BE6BBF1000F7FF455AFD4F881
:105FB0000C32002B7FF450AF206804F56F72FDF7B0
:105FC0000FF949E7BBF1000F7FF4A9AEE36C002B9A
:105FD0007FF4A5AE206804F56F72FDF701F99EE627
:105FE000314B324A0344934205D82268D36843F4C4
:105FF0006053D36007E62E4AA0F57403A3F510534F
:10600000934205D82268D36843F45053D360FAE52D
:10601000284AA0F18373A3F5E743934205D222688F
:10602000D36843F44053D360EDE5234B234A034444
:10603000934205D82268D36843F43053D360E2E535
:106040001F4B204A0344934205D22268D36843F48D
:106050002053D360D7E51C4B1C4A0344934205D21E
:106060002268D36843F41053D360CCE5184AA0F1FA
:10607000B773A3F55853934205D22268D36843F40B
:106080000053D360BFE5134B134A03449342226885
:10609000D36834BF43F4E05343F4C053D360B2E554
:1060A000405327FFFF340C00401E1BFF3F420F00F0
:1060B0007F4F120020D6130060B6E5FE5FE31600A6
:1060C00000D3CEFE40771B00C05BB3FEC091210021
:1060D00020753800E05459FEE09C410090F8B83338
:1060E000012B0BD010B50123044680F8B8330068AB
:1060F000FCF7F8FF002084F8B80310BD02207047B9
:1061000038B50446080623D4C1EBC10504EB850568
:106110001C2000FB014085F8F811002185F8F911D9
:10612000C5F8002285F8FB3100F5FC71022B04BF95
:1061300000230B7194F8B833012B1ED00123206883
:1061400084F8B833FCF764FD002084F8B80338BD48
:1061500001F07F01C1EBC10504EB85051C2000FBAC
:1061600001402A64012285F83810E98785F83B3020
:1061700085F8392000F13801D8E7022038BD00BF8A
:106180004AB2002A10B5044618DB1C2303FB0103A6
:10619000D20F83F8F92183F8F81194F8B823012A73
:1061A00003F5FC731AD00122206884F8B82319463D
:1061B000FCF776FD002084F8B80310BD01F07F01E4
:1061C0001C2303FB0103D20F83F8392083F8381016
:1061D00094F8B823012A03F13803E4D1022010BD5A
:1061E00038B501F07F05C5EBC50400EB8404002140
:1061F000C4F80422C4F8101284F8F911C4F80C325F
:1062000084F8F85103691C2101FB0501012B08BF2B
:10621000C4F80822006801F5FC71DAB21DB9FCF778
:1062200081FE002038BDFCF799FD002038BD00BF7D
:1062300001F00F01C1EBC10100EB8101B1F81002C7
:10624000704700BF70B501F07F05C5EBC50400EBDA
:10625000840401210026626484F83910E36484F820
:106260003850266503691C2101FB0501012B08BF7D
:10627000A26400683831DAB21DB9FCF753FE002081
:1062800070BDFCF76BFD002070BD00BF4AB2002A54
:1062900038B50D46044618DB1C2303FB010303F548
:1062A000FC73D20F01215A701D70997094F8B823B5
:1062B0008A4218D084F8B81320681946FCF7DCFE2F
:1062C00055B1002084F8B80338BD01F07F051C23C8
:1062D00003FB05033833E4E7217C206804F56F7283
:1062E000FCF77EFFEDE7022038BD00BF4AB2002A6E
:1062F00038B5044618DB1C2303FB010303F5FC73CC
:10630000D20F00255A7019709D7094F8B823012A95
:1063100011D00122206884F8B8231946FCF7CAFE80
:1063200084F8B853284638BD01F07F011C2303FBD5
:1063300001033833E4E7022038BD00BF30B52448FC
:10634000244B25490360012200238FB04FF4803491
:10635000446081628360036183610362C362C360DE
:106360000363C261426104F03FFC08BB06240122C2
:1063700000231748039301A9CDE9014204F0AEFDC3
:1063800008BB0620002301224FF480154FF480340F
:10639000059005A90E480692CDE90A33CDE90C45D2
:1063A00009920793089302F0E1FC30B90FB030BDB9
:1063B0000A485E21FEF732F9D8E708487821FEF74F
:1063C0002DF90FB030BD05486821FEF727F9D8E751
:1063D00000CF0020002001400100000FD88F0208EC
:1063E00030B52648264B03604FF4803200238FB02F
:1063F0004FF080544FF0606142600122C0E90A14FE
:106400008360036183610362C3600363C2614261AD
:1064100004F0EAFB08BB0D24012200231748039374
:1064200001A9CDE9014204F059FD08BB0A2000236F
:1064300001224FF480154FF48034059005A90F48D0
:106440000692CDE90A33CDE90C45099207930893EA
:1064500002F08CFC30B90FB030BD0A489221FEF733
:10646000DDF8D8E70748AC21FEF7D8F80FB030BD0B
:1064700004489C21FEF7D2F8D8E700BFB8CE002030
:1064800000210140D88F020830B52648264B036012
:106490004FF4803200238FB04FF080544FF0606192
:1064A00042600122C0E90A148360036183610362D0
:1064B000C3600363C261426104F096FB08BB0C2415
:1064C000012200231748039301A9CDE9014204F0FA
:1064D00005FD08BB0B20002301224FF480154FF46B
:1064E0008034059005A90F480692CDE90A33CDE91D
:1064F0000C4509920793089302F038FC30B90FB0AD
:1065000030BD0A48C621FEF789F8D8E70748E021E0
:10651000FEF784F80FB030BD0448D021FEF77EF8B6
:10652000D8E700BF48CF002000220140D88F0208E2
:10653000F0B5484A0368934289B007D0464A93426F
:1065400047D0464A93426BD009B0F0BD0026444B79
:1065500000965A6C434D42F480725A645B6C059607
:1065600003F48073009303272F2303A904463E48B6
:10657000009A0393049704F059FD70233B4803935A
:1065800003A9CDE9047604F051FD394828604FF4A1
:1065900080674FF400614FF400524FF48073284637
:1065A000C5E90266C5E90866C5E90471C5E90623BF
:1065B0006E60FEF733FE002846D1A5630022052158
:1065C0001220AC63FBF7E0FC1220FBF715FD09B0CD
:1065D000F0BD234B2448002401945A6C42F400720D
:1065E0005A645B6C059403F40073019303A92F2391
:1065F0000325CDE90335019A04F018FDCDE90454D3
:1066000070231A48039303A904F010FD22460521C4
:106610001220FBF7B9FC1220FBF7EEFC09B0F0BD2D
:106620000F4B1148002402945A6C42F480625A6461
:106630005B6C059403F4806302930F220323CDE97E
:106640000323029D03A9DFE70A484FF48A71FDF78F
:10665000E5FFB2E700200140002101400022014097
:106660000038024090CF00200008024000000240A5
:1066700010640240D88F020830B54B7883B00D46C5
:106680000446092B0BD8DFE803F035480A580A0501
:10669000650A7B158B8813B9CB88002B7DD08021B0
:1066A0002046FEF7E5F820460021FEF7E1F800203D
:1066B00003B030BD8978984D01292970EFD890F842
:1066C000FC31022B00F08080032BE8D1002900F080
:1066D00011814168012909D0C9B2FEF787FC2978E8
:1066E00061602046FEF778FC0228D8D02046FBF7F0
:1066F000EFFCDCE790F8FC31023B012BCFD8D0F85F
:1067000004320122C2600BB10323C360022204F1F0
:106710000C012046FBF7B0FCC9E790F8FC31023BC6
:10672000012BBCD84B88012BC1D1D0F814320022E8
:106730009B68C0F804229847D8E74B88012BB6D154
:10674000D0F81422C0F80432936898472046FBF72B
:10675000BFFCACE749880B0A013B062B9FD801A27E
:1067600052F823F0EF6700086368000853680008D8
:106770009F6600089F6600083D68000823680008BF
:10678000CA88012A8BD190F8FC31022B28D0032B28
:1067900085D1011DFBF770FC89E790F8FC31032BD4
:1067A0003FF47DAF8D7805F07F0580F8FE512946D6
:1067B000FEF78EF82046FBF78BFC002D00F08D8055
:1067C000022384F8FC3172E700298FD001210323D2
:1067D000416080F8FC31FEF7FFFB022886D15EE7BE
:1067E0000146002341F8083FFBF746FC5FE7D0F87D
:1067F0001032007C1B680DF106019847BDF8062099
:10680000002A3FF454AFEB88002B3FF450AF9A427C
:1068100028BF1A4601462046ADF80620FBF72CFC9F
:1068200045E7037C002B7FF43AAFD0F814320DF12A
:1068300006001B6B984707234370DFE7037C002BA0
:106840007FF42DAFD0F814320DF106005B6B984742
:10685000D4E7C9B2052957D8DFE801F0372F271F41
:10686000170F037C002B3CD1D0F814320DF1060039
:106870009B6A984702234370C0E7D0F81032007C2F
:106880009B690DF106019847B8E7D0F81032007CFB
:106890005B690DF106019847B0E7D0F81032007C33
:1068A0001B690DF106019847A8E7D0F81032007C6B
:1068B000DB680DF106019847A0E7D0F81032007CA4
:1068C0009B680DF10601984798E7D0F81032007CDC
:1068D0005B680DF10601984790E7012384F8FC31CD
:1068E000E5E6D0F814320DF10600DB6A9847022382
:1068F000437083E70223416080F8FC31FEF776FBAA
:106900002046FBF7E5FBD2E6D0F814320DF1060283
:106910009B6B984772E700BF4406002038B590F89B
:10692000FC31032B04460DD10B79012B0D4609D800
:10693000D0F814329B689847EB885BB92046FBF788
:10694000C7FB07E080212046FDF792FF204600218B
:10695000FDF78EFF002038BD70B50B788A8803F0F4
:106960006003202B054609D04B78012B0C46D6B28C
:1069700026D0032B3CD03BB1002070BDD0F81432A0
:106980009B689847002070BD90F8FC31022B48D0DE
:10699000032B3CD106F07F0400EB041413063146B0
:1069A0004CBF143404F58274FDF77EFF003818BF25
:1069B00001202060214628460222FBF75DFBDBE731
:1069C00090F8FC31022B2CD0032B20D14B88002BCC
:1069D000D2D1710608D03146FDF758FFD5F81432F0
:1069E00021469B68284698472846FBF771FBC3E77A
:1069F00090F8FC31022B14D0032B08D14B88002BCC
:106A0000ECD17306EAD03146FDF732FFE6E780218C
:106A10002846FDF72DFF28460021FDF729FF00201D
:106A200070BD7206A8D03146FDF722FFA4E700BF73
:106A30000B7803704B784370CA788B7803EB022392
:106A400043804A790B7903EB02238380CA798B79DF
:106A500003EB0223C380704710B580210446FDF785
:106A600007FF20460021BDE81040FDF701BF00BF31
:106A700010B3037870B403B30446C0F10106A31940
:106A800014F8015FDBB2002DF9D101335B00DCB2F9
:106A9000032513800C704D7004785CB1022300252F
:106AA0005A1CD2B2CC548D5410F8014F0233DBB2D1
:106AB000002CF5D170BC7047704702242346E7E7ED
:106AC00000F108034FF0FF310022C0E90023C0E9C4
:106AD00003338160704700BF00230361704700BF2C
:106AE000D0E9002310B49C688C609C684B60013234
:106AF000616099605DF8044B08610260704700BFF7
:106B000030B40D686B1C10D000F108031C465B68A4
:106B10001A68AA42FAD902684B60013299608C6007
:106B20006160086130BC0260704704696368F2E725
:106B3000026910B4D0E9011354688B608442596033
:106B400008BF536013685DF8044B013B00210161ED
:106B500018461360704700BF10B582B00024224B66
:106B600000945A6C42F480425A645A6C02F4804297
:106B70000092009A01941A6C42F080521A641B6CC5
:106B800003F0805301930320019BFBF7E9F92246B0
:106B900021466FF00B00FBF7F7F9224621466FF014
:106BA0000A00FBF7F1F9224621466FF00900FBF7D6
:106BB000EBF9224621466FF00400FBF7E5F9224687
:106BC00021466FF00300FBF7DFF922460F216FF03B
:106BD0000100FBF7D9F922460F214FF0FF3002B038
:106BE000BDE81040FBF7D0B90038024008B50B4BA8
:106BF0001A6842F400721A601A6842F480621A60DD
:106C00001A6842F480721A600320FBF7A9F9002089
:106C1000FBF776FAFFF7A0FF002008BD003C02401A
:106C2000034A044B11681B780B441360704700BF84
:106C3000F0CF002014000020014B1868704700BFFF
:106C4000F0CF002038B50446FFF7F6FF631C054679
:106C500002D0044B1B781C44FFF7EEFF431BA342FA
:106C6000FAD338BD14000020122301480B8070476E
:106C700034000020042301480B80704748000020A6
:106C800010B5044C04480A462146FFF7F1FE2046A1
:106C900010BD00BFF4CF0020EC8F020810B5044CEB
:106CA00004480A462146FFF7E3FE204610BD00BF18
:106CB000F4CF0020A0BE002010B5044C04480A46C2
:106CC0002146FFF7D5FE204610BD00BFF4CF0020BF
:106CD000FC8F020810B5044C04480A462146FFF711
:106CE000C7FE204610BD00BFF4CF00201890020858
:106CF00010B5044C04480A462146FFF7B9FE204669
:106D000010BD00BFF4CF0020249002080020EE291F
:106D100008B5108002D0062905D008BD13461222FE
:106D200004481A8008BD04490448FFF7A1FE024840
:106D300008BD00BF4C000020F4CF002034900208B2
:106D400039B101291CD002290CBF4FF400714FF456
:106D500040710D4B1A6922F440721A611A6911438D
:106D600019611A6922F0F8021A611A6942EAC00030
:106D700040F0020018611A6942F480321A617047CB
:106D80004FF48071E5E700BF003C0240144B1A68E5
:106D900091050FD51A6822F400721A601A6842F43D
:106DA00000621A601A6822F400621A601A6842F4DB
:106DB00000721A600A4B1A6852050FD51A6822F43D
:106DC00080621A601A6842F480521A601A6822F4CB
:106DD00080521A601A6842F480621A60704700BFDD
:106DE000003C02402DE9F8432D4F3B7E012B38D06B
:106DF000012304464CF2503088463B7601F02CF9D2
:106E0000064648BB4FF0FF33C8F800302368012B1B
:106E10002BD0D4E902532B449D421BD2DFF884903F
:106E200005E0D4E9022301351344AB4212D9217C99
:106E30002846FFF785FF4CF2503001F00DF9D9F8E4
:106E4000103023F0FA03C9F810300028E9D0C8F850
:106E500000500646FFF79AFF00233B763046BDE818
:106E6000F88302263046BDE8F8830E4D23692A696F
:106E700022F440722A612A6942F004022A612A69D6
:106E80001B029BB2134343F480332B614CF250300E
:106E900001F0E2F82B6923F0040306462B61D9E7E1
:106EA00040D40020003C0240704700BF70B4D0E9DD
:106EB0000041D0E902268BB0056902940391049247
:106EC000D0E90612446905960123069507940891B6
:106ED00009928DF807309DF80730002BFBD10BB0DD
:106EE00070BC70471EF0040F0CBFEFF30880EFF387
:106EF0000980FFF7DBBF00BFFEE700BFFEE700BF72
:106F0000FEE700BF704700BF01F064BD0148FEF717
:106F1000F7BA00BF58CC00200148FEF7F1BA00BF15
:106F2000B8CC00200148FEF7EBBA00BF58CD0020D6
:106F30000148FEF7E5BA00BFF8CB00200148FBF797
:106F4000D1BB00BF18D40020FFF7F8BFFFF7F6BF92
:106F5000FFF7F4BF08B5044803F0CAFABDE80840DB
:106F6000024803F0C5BA00BFF0C50020B4C5002038
:106F70000148FDF749B900BFA0CB0020014800F04F
:106F800041BF00BF18CD002008B54320FBF740F8F3
:106F9000024B1868BDE8084001F01ABDA4C70020E4
:106FA00003681A68520770B55E6804460D4601D53D
:106FB00031060DD41A685B68920708D59B0606D582
:106FC00000212046A84723686FF012021A6070BDA6
:106FD0000121A84723686FF00C021A60EAE700BF9E
:106FE00010B5074C07490848FFF7DAFF2146074864
:106FF000FFF7D6FF21460648BDE81040FFF7D0BF97
:107000000DD40008F1D1000800CF0020B8CE002038
:1070100048CF002003681A6970B5960704460D46EC
:1070200006D56FF002021A61596B0120A847236848
:107030001A69500706D56FF004021A61996B022095
:10704000A84723681A69110706D56FF008021A616C
:10705000D96B0320A84723681A69D20608D56FF0B8
:1070600010021A61196C04202B46BDE870401847C5
:1070700070BD00BF08B504480449FFF7CBFFBDE869
:107080000840014803F034BA68C60020E9D6000879
:10709000034803686FF001021A6106F0BDB800BF33
:1070A0001CC70020034803686FF001021A6106F054
:1070B000B3B800BFF0C50020014804F05FBB00BFBB
:1070C000C0D40020014804F027BF00BFC0D4002076
:1070D000012004F087B900BF042004F083B900BF89
:1070E000082004F07FB900BF102004F07BB900BF76
:1070F00008B5202004F076F9402004F073F98020D0
:1071000004F070F94FF4807004F06CF9BDE80840A9
:107110004FF4007004F066B908B54FF4806004F0D5
:1071200061F94FF4006004F05DF94FF4805004F011
:1071300059F94FF4005004F055F94FF4804004F031
:1071400051F9BDE808404FF4004004F04BB900BFCE
:1071500010B5094C094900222046FDF719FF0849DE
:107160002046FDF72BFF2046064901F077FD20461B
:10717000BDE81040FDF72ABFF4D100201800002020
:1071800060000020040000200E480F4A38B50F4B65
:1071900003604FF04073C360002308254FF4702450
:1071A0004FF4401182618383C0E9044145608360EC
:1071B000FAF7E6FF00B938BDBDE8384004484F2172
:1071C000FDF72CBA18D40020000101010064004032
:1071D00050900208214B02689A4200D0704770B567
:1071E00086B0002403F5EA3300941A6C1C4842F080
:1071F00000721A641B6C039403F000734FF4407127
:107200000093032209230191022501A9CDE904235A
:10721000009E029503F00AFF224606211320FAF78A
:10722000B3FE1320FAF7E8FE224606211420FAF7EF
:10723000ABFE1420FAF7E0FE224606211520FAF7ED
:10724000A3FE1520FAF7D8FE224606211620FAF7EB
:107250009BFE1620FAF7D0FE06B070BD0064004019
:1072600000040240002800F060812DE9F04103682D
:10727000DD0782B004462FD5AD498A6802F00C02C2
:10728000042A00F0EC808A6802F00C02082A00F060
:10729000E2806368B3F5803F00F0EB80B3F5A02F88
:1072A00000F05081A24D2A6822F480322A602A68B8
:1072B00022F480222A60002B40F0E080FFF7BCFC23
:1072C000064605E0FFF7B8FC801B642800F2008149
:1072D0002B689B03F6D423689F0728D5944A9168AE
:1072E00011F00C0F00F09A80916801F00C01082950
:1072F00000F09080E368002B00F006818D4B8C4EEF
:1073000001221A60FFF798FC054605E0FFF794FCA0
:10731000401B022800F2DC8033689807F6D53368FA
:10732000226923F0F80343EAC203336023681A0793
:107330005CD458073AD57E4A136C13F0805340F062
:1073400088800193136C43F080531364136C03F033
:1073500080530193019B0125774E3368D90540F195
:10736000A780A368012B00F0B780052B00F02681D1
:107370006F4E326F22F001023267326F22F0040248
:107380003267002B40F0AD80FFF756FC41F28838A1
:10739000074605E0FFF750FCC01B404500F298800F
:1073A000336F9807F6D4002D40F0D680A369CBB197
:1073B0005F4DAA6802F00C02082A36D0022B5F4B00
:1073C0004FF000021A6000F0CD80FFF735FC2C462C
:1073D000054604E0FFF730FC401B022878D82368FC
:1073E0009B01F7D4002002B0BDE8F081636903B3CC
:1073F000534B4F4E01221A60FFF71EFC054604E076
:10740000FFF71AFC401B022862D8736F9B07F7D561
:1074100023688EE7526856023FF56CAF444A126803
:10742000950739D5E268012A36D0012002B0BDE8BF
:10743000F081434A3E4E1360FFF7FEFB054604E031
:10744000FFF7FAFB401B022842D8736F9F07F7D45F
:10745000DEE7002580E74A6850027FF51AAF344A1C
:10746000126891037FF538AF6268002A7FF434AF69
:10747000DBE72F4A136843F480331360FFF7DCFB2C
:107480002B4E054604E0FFF7D7FB401B64281FD8AE
:1074900033689A03F7D51EE7254920690A6822F068
:1074A000F80242EAC0020A601A077FF542AF9DE780
:1074B000336843F480733360FFF7BEFB07463368DD
:1074C000DA053FF54EAFFFF7B7FBC01B0228F6D930
:1074D000032002B0BDE8F081154A136F43F00103A9
:1074E0001367FFF7A9FB124F064641F2883804E004
:1074F000FFF7A2FB801B4045EAD83B6F9B07F7D5FF
:10750000002D3FF453AF27E00A4A094E1360FFF7FE
:1075100093FB054604E0FFF78FFB401B0228D7D8FA
:1075200033689907F7D4236801E70120704700BF4B
:1075300000380240000047420070004060004742AF
:10754000800E4742224B1A6842F480221A601A6861
:1075500042F480321A6091E71D4A136C23F0805385
:10756000136423E7FFF768FB064604E0FFF764FBBC
:10757000801B0228ACD82B689901F7D4D4E90736D0
:10758000D4E90902E16A334343EA8013520843EA2B
:107590000163013A0F490E4E43EA024301226B6038
:1075A0000A60FFF749FB044604E0FFF745FB001BB8
:1075B00002288DD833689A01F7D513E7044B1A6F68
:1075C00042F004021A671A6F42F001021A6788E754
:1075D0000038024060004742174908B58B6803F045
:1075E0000C03042B1BD0082B17D14A684B6813F4EB
:1075F000800302F03F0214D149681048C1F388119A
:10760000A1FB0001F9F7A0FB0B4B5B68C3F301433F
:1076100001335B00B0FBF3F008BD084808BD084823
:1076200008BD4B680648C3F38813A3FB0001002381
:10763000F9F78AFBE8E700BF003802400024F400B5
:1076400000127A00002800F08680474A136803F091
:107650000F038B422DE9F0410D46044609D2CBB20F
:107660001370136803F00F038B4202D00120BDE8B2
:10767000F0812368980714D5590704D53B498A68D7
:1076800042F4E0528A601A0704D538498A6842F405
:1076900060428A603549A0688A6822F0F00202439D
:1076A0008A60DF0721D56268012A56D0931E012B1C
:1076B0002E4B1B684CD99907D8D52C4EB36823F0B4
:1076C00003031343B360FFF7B7FA41F28838074664
:1076D00004E0FFF7B1FAC01B404543D8B3686268C5
:1076E00003F00C03B3EB820FF3D11F4A136803F0CE
:1076F0000F03AB4206D9EBB21370136803F00F030C
:10770000AB42B3D123685A0706D51849E0688A68A6
:1077100022F4E05202438A601B0707D5134A21690D
:10772000936823F4604343EAC1039360FFF754FF77
:107730000E4A0F4C92680F49C2F303120346A25C33
:107740000020D3400B60FAF7DBFC0020BDE8F0819D
:107750009801B2D48AE701207047044B1B689E034E
:10776000ABD483E7032082E7003C024000380240AC
:1077700064900208F4010020014B1868704700BFB4
:10778000F4010020044B054A9B680549C3F382239A
:107790000868D35CD84070470038024074900208F3
:1077A000F4010020044B054A9B680549C3F34233AA
:1077B0000868D35CD84070470038024074900208D3
:1077C000F40100200E4B0F2202609A6802F00302BF
:1077D00042609A6802F0F00282609A6802F4E05215
:1077E000C2609B68DB0810B403F4E053054C0361EE
:1077F00023685DF8044B03F00F030B60704700BF74
:1078000000380240003C0240026811692DE9F8434B
:10781000C568836821F44051044629430069116119
:10782000D16865690343E06921F416412B4321F0D7
:107830000C0103430B43D3605369A16923F44073E4
:107840000B43B0F5004F53619B4B00F09A809A4276
:1078500059D003F580639A4255D0FFF793FF974FB5
:10786000636800EB800000EB80009B00B0FBF3F34B
:10787000A7FB03235B091D01FFF784FF666800EB8C
:10788000800000EB8000B600B0FBF6F6FFF77AFF51
:10789000636800EB800000EB80009B00B0FBF3F31B
:1078A000A7FB03235B094FF0640909FB13631B016A
:1078B0003233A7FB03235B0903F0F006FFF762FFF7
:1078C000626800EB800000EB80009300B0FBF3F8EF
:1078D000FFF758FFD4E9002300EB800000EB8000A5
:1078E0009B00B0FBF3F3A7FB03135B0909FB1383B6
:1078F0001B013233A7FB0313C3F3431333432B445E
:107900009360BDE8F883FFF74DFF6C4F636800EBB1
:10791000800000EB80009B00B0FBF3F3A7FB032388
:107920005B091D01FFF73EFF666800EB800000EB7E
:107930008000B600B0FBF6F6FFF734FF636800EB9B
:10794000800000EB80009B00B0FBF3F3A7FB032358
:107950004FF064095B0909FB13631B013233A7FB7A
:1079600003235B0903F0F006FFF71CFF626800EBDE
:107970008000930000EB8000B0FBF3F8FFF712FFEC
:10798000A8E79A4259D003F580639A4255D0FFF791
:10799000F9FE4A4F636800EB800000EB80005B005B
:1079A000B0FBF3F3A7FB03235B091E01FFF7EAFE1D
:1079B000656800EB800000EB80006D00B0FBF5F522
:1079C000FFF7E0FE636800EB800000EB80005B00E7
:1079D000B0FBF3F3A7FB03235B094FF0640909FB3A
:1079E0001353DB003233A7FB03231B0903F4F875A1
:1079F000FFF7C8FE626800EB800000EB80005300D8
:107A0000B0FBF3F8FFF7BEFED4E9002300EB8000E3
:107A100000EB80005B00B0FBF3F3A7FB03135B09F3
:107A200009FB1383DB003233A7FB0313C3F34213B9
:107A300033442B449360BDE8F883FFF7B3FE1F4F38
:107A4000636800EB800000EB80005B00B0FBF3F3A9
:107A5000A7FB03235B091E01FFF7A4FE656800EB8B
:107A6000800000EB80006D00B0FBF5F5FFF79AFE9B
:107A7000636800EB800000EB80005B00B0FBF3F379
:107A8000A7FB03234FF064095B0909FB1353DB00D9
:107A90003233A7FB03231B0903F4F875FFF782FEBB
:107AA000626800EB8000530000EB8000B0FBF3F84D
:107AB000FFF778FEA8E700BF001001401F85EB51DB
:107AC00060B338B590F83930044603F0FF0203B3D1
:107AD0002268242384F83930D36823F40053D36018
:107AE0002046FFF791FE23681A6922F490421A613A
:107AF0005A6922F02A025A61DA680025202142F4EC
:107B00000052DA60E56384F8391084F83A102846A8
:107B100038BD80F83820FDF797F9D9E70120704784
:107B200080B110B52423044680F83930FDF70EFAF1
:107B30000023E36384F8383084F8393084F83A302D
:107B4000184610BD01207047F8B5044690F839007A
:107B500020282BD141B33AB394F83800012825D01E
:107B6000E284A284206B266821620025134621222C
:107B7000E563012784F839200D4A84F83870C26320
:107B80000C4A02640C4A0565C264321DFDF71CFCF8
:107B900023686FF040021A6084F838505A6942F046
:107BA000800228465A61F8BD0120F8BD0220F8BDC8
:107BB000917C0008C17C00089D7D000890F83A3057
:107BC000202B3BD1002937D0002A35D0F0B590F8D2
:107BD0003830012B83B0044632D0406BA162A285BD
:107BE000002513460A462221E563012784F83A104E
:107BF0001549266884F83870C16314490164144932
:107C00000565C164311DFDF7DFFB236801951A6826
:107C100001925A68019284F83850019ADA6842F465
:107C20008072DA605A693A435A615A69284642F0CA
:107C300040025A6103B0F0BD012070470220704736
:107C4000022003B0F0BD00BFD17C00088D7D00088C
:107C50009D7D00080368DA6822F4907210B5DA603E
:107C60005A6922F001025A615A695206044609D53E
:107C70005A69406B22F040025A6118B10023036533
:107C8000FDF7E4FB00202023E08584F83A3010BDA6
:107C900008B50368806B1B6813F480730AD102680F
:107CA000C384536923F080035361D36843F04003D6
:107CB000D36008BD1AF082F908BD00BF704700BF4D
:107CC00008B5806BFFF7FAFF08BD00BF704700BF23
:107CD00008B50368806B1B6813F4807310D10268C9
:107CE000C385D36823F48073D360536923F0010301
:107CF00053615369202123F04003536180F83A1007
:107D0000FFF7E4FF08BD00BF08B58368B3F5805FE7
:107D100017D0036973B10368826A5B68511C03F072
:107D20007F0381621370C38D013B9BB2C3859BB1FE
:107D3000002008BD836A0268591C526881621A706B
:107D4000F1E70269836ABAB902685268C2F30802AD
:107D500023F8022B8362E6E70368DA6822F4907264
:107D6000DA605A69202122F001025A6180F83A1043
:107D7000FFF7ACFF002008BD02685268D2B223F8BA
:107D8000012B8362CFE700BF704700BF08B5806B4F
:107D9000FFF7FAFF08BD00BF704700BF08B5806B52
:107DA0000368596990F83920212A0BD0596990F855
:107DB0003A20222A16D0C36B43F01003C363FFF7A7
:107DC000EBFF08BD0906F1D50022C284DA68202144
:107DD00022F0C002DA6080F83910596990F83A2030
:107DE000222AE8D14A06E6D50022C285DA6822F4C2
:107DF0009072DA605A69202122F001025A6180F8FB
:107E00003A10D8E703681A6870B51607DD68596933
:107E100004460CD1960601D5A9064DD4100601D50D
:107E2000290651D4560601D5680669D470BD01F003
:107E3000010105F490700843F0D0D60705D5E80598
:107E400003D5E06B40F00100E063560729D561B12E
:107E5000E16B900741F00201E16340F18380E16B47
:107E600041F00401E163110721D4E16B0029DDD069
:107E7000920609D5AE0607D594F83A20222A03D1F6
:107E80002046FFF741FF23685A69E56B02F0400284
:107E900005F0080515433ED12046FFF77DFFE56359
:107EA00070BD960757D41007DFD50029DDD0E16BF0
:107EB00041F00801E163D8E790F83A30222BB5D1C0
:107EC000BDE87040FFF720BF94F83920212AADD1DA
:107ED000A268B2F5805F226A47D0511C21621278F5
:107EE0005A60E28C013A92B2E284002A9ED1DA68AA
:107EF00022F08002DA60DA6842F04002DA6070BD97
:107F0000DA68202122F04002DA60204684F8391035
:107F10001AF054F870BDDA6822F49072DA605A6987
:107F2000202122F001025A6184F83A105A6955065C
:107F300014D55A69606B22F040025A6170B1114B3E
:107F40000365FDF7CBFA00283FF470AF606BBDE826
:107F50007040036D1847002981D186E72046FFF75E
:107F60001BFF70BD1107A2D47FE711882069C1F300
:107F70000801596010B902322262B2E7013222626E
:107F8000AFE700BF897F000808B5806B0023C38579
:107F9000C384FFF701FF08BD1B4BDA68D10605D586
:107FA0001A49CA6910200243CA61D860164BDA68C0
:107FB000920606D51549CA69202042F00802CA6116
:107FC000D860114BDA68500606D51049CA694020BE
:107FD00042F00402CA61D8600B4BDA68110606D57C
:107FE0000A49CA69802042F00202CA61D860064B81
:107FF000DA68920706D50549CA69022042F02002D4
:10800000CA61D860704700BF003C024040D40020E5
:10801000064B1A69002A01DB002070470449054A13
:1080200059605A601869C00F704700BF003C024099
:1080300023016745AB89EFCD034A136943F0004341
:1080400013610020704700BF003C0240014BD8691B
:10805000704700BF40D40020124B70B50022044688
:10806000DA61FEF7E9FD104D064601E0611C0DD115
:10807000EB68DA03FAD4EB68DB0744BF0123EB605B
:10808000094BD86810F0F20008D170BD24B1FEF79A
:10809000D3FD801BA042EBD9032070BDFFF77CFF0E
:1080A000012070BD40D40020003C02402DE9F8437F
:1080B0002B4E347E012C31D081461D464CF250307F
:1080C00001230F4690463376FFF7C6FF18B1002311
:1080D0003376BDE8F883234B1A6922F440721A61A3
:1080E0001A69B9F1000F1CD0B9F1010F22D0B9F112
:1080F000020F2AD042F440721A611A6942F001025A
:108100001A61C7F800807D604CF25030FFF7A4FF81
:10811000144A136923F001031361D8E70220BDE874
:10812000F8831A6119695FFA88F241F00101196157
:108130003A70E9E742F480721A6119691FFA88F20D
:1081400041F0010119613A80DEE742F400721A61E0
:108150001A6942F001021A61C7F80080D4E700BF33
:1081600040D40020003C024070B50446006CA66B71
:1081700020B925685DB30136A66370BD1546024679
:1081800085B9A0681BF0F6FDA368216C62680B44FA
:108190009342A36006F1010624BF2368A36028462A
:1081A000A66370BDE0681BF0E5FD226CE368216802
:1081B0009B1A8B42E360C2F1000202D263681A4448
:1081C000E260022D08D001360020A66370BD606811
:1081D00001F0B0FD6560CEE7012E38BF012600201A
:1081E000CAE700BF026C72B10B46C16810B44468A4
:1081F0001144A142C16024BF0168C1605DF8044B15
:1082000018461BF0B7BD704770B50446FCF7C2FCBA
:1082100094F845506DB2002D15DD04F1240604E0FC
:108220006B1E13F0FF0F5DB20DD0636A304653B181
:1082300001F05EFC0028F3D001F0FEFC6B1E13F091
:10824000FF0F5DB2F1D1FF2384F84530FCF7C4FC89
:10825000FCF7A0FC94F844506DB2002D15DD04F13C
:10826000100604E06B1E13F0FF0F5DB20DD0236902
:10827000304653B101F03CFC0028F3D001F0DCFCA7
:108280006B1E13F0FF0F5DB2F1D1FF2384F8443071
:10829000BDE87040FCF7A0BC38B5E0B104460D461F
:1082A000FCF778FCD4E90F032268A26000FB03F01E
:1082B000C31A1344FF2102440020A063E36084F842
:1082C0004410626084F84510EDB9236963B9FCF786
:1082D00083FC012038BD4FF0500383F31188BFF3B6
:1082E0006F8FBFF34F8FFEE704F1100001F000FC29
:1082F0000028ECD00A4B4FF080521A60BFF34F8F2A
:10830000BFF36F8FE3E704F11000FEF7D9FB04F130
:108310002400FEF7D5FBFCF75FFC012038BD00BF51
:1083200004ED00E070B506460D4651B100FB01F0CA
:108330004830FDF705FA044688B100F148030360B0
:1083400005E04820FDF7FCF9044640B12460C4E98B
:108350000F6501212046FFF79FFF204670BD0024D6
:10836000204670BD40B94FF0500383F31188BFF32E
:108370006F8FBFF34F8FFEE7FFF7D4BF2DE9F047B4
:1083800084B00192002876D088461F460446002912
:1083900065D0022F0BD1E36B012B08D04FF05003B7
:1083A00083F31188BFF36F8FBFF34F8FFEE701F0A8
:1083B00063FC0646002867D00026DFF83CA14FF09A
:1083C000000907E0FCF708FC2046FFF71DFF01F05D
:1083D00033FA0126FCF7DEFBA26BE36B9A4263D310
:1083E000022F61D0019D002D00F08280002E57D019
:1083F000FCF7F2FB01F05AF9FCF7CCFB94F844309F
:10840000FF2B08BF84F8449094F84530FF2B08BF39
:1084100084F84590FCF7E0FB01A902A801F0C8FB35
:1084200000285ED1FCF7B6FBA26BE36B9A42C9D180
:10843000FCF7D2FB019904F1100001F03FFB20464C
:10844000FFF7E2FE01F0F8F90028C2D14FF08053A7
:10845000CAF80030BFF34F8FBFF36F8FB9E7036CDB
:10846000002B96D04FF0500383F31188BFF36F8F2A
:10847000BFF34F8FFEE74FF0500383F31188BFF334
:108480006F8FBFF34F8FFEE7019B002B95D04FF00E
:10849000500383F31188BFF36F8FBFF34F8FFEE755
:1084A00002A801F06FFBA3E73A4641462046FFF7DA
:1084B0005BFE636A73B938B10F4B4FF080521A609C
:1084C000BFF34F8FBFF36F8FFCF786FB012004B023
:1084D000BDE8F08704F1240001F00AFB0028F3D086
:1084E000EAE72046FFF790FE01F0A6F90020EEE74C
:1084F000FCF772FB2846EAE704ED00E070B3036C7A
:1085000070B5044643B14FF0500383F31188BFF3B5
:108510006F8FBFF34F8FFEE703680D463BB3FCF749
:1085200045FCEFF311864FF0500383F31188BFF33E
:108530006F8FBFF34F8FA36BE26B9A4223D994F8EE
:1085400045200133FF2AA36353B220D001335BB22D
:1085500084F84530012086F3118870BD4FF0500338
:1085600083F31188BFF36F8FBFF34F8FFEE743682C
:10857000002BD4D04FF0500383F31188BFF36F8FDB
:10858000BFF34F8FFEE7002086F3118870BD636A4A
:10859000002BDFD004F1240001F0AAFA0028D9D082
:1085A000002DD7D001202860EEE700BF2DE9F0476D
:1085B00084B00192002872D00E461F46044600295E
:1085C00054D001F059FB002844D0FCF7E3FAA56B26
:1085D000002D40F08D80019B002B35D002A801F0CA
:1085E000D1FADFF868A1A84604F12409FCF7F4FAEF
:1085F00001F05CF8FCF7CEFA94F84430FF2B08BF8A
:1086000084F8448094F84530FF2B08BF84F84580F7
:10861000FCF7E2FA01A902A801F0CAFA002831D158
:10862000FCF7B8FAA36B002B42D0FCF7D5FA204632
:10863000FFF7EAFD01F000F9FCF7ACFAA56B002D9D
:1086400056D1019B002BD1D1FCF7C6FA002004B013
:10865000BDE8F087019B002BB7D04FF0500383F3A8
:108660001188BFF36F8FBFF34F8FFEE7036C002BB2
:10867000A7D04FF0500383F31188BFF36F8FBFF380
:108680004F8FFEE72046FFF7BFFD01F0D5F8FCF75E
:1086900081FAA36B002BD7D0FCF79EFACCE74FF002
:1086A000500383F31188BFF36F8FBFF34F8FFEE743
:1086B000FCF792FA23689BB10199484601F0FEF954
:1086C0002046FFF7A1FD01F0B7F80028B4D14FF024
:1086D0008053CAF80030BFF34F8FBFF36F8FABE703
:1086E000FCF758FA606801F0D7FAFCF775FAE3E78F
:1086F00031462046E668FFF775FD4FB92368013D16
:10870000A563FBB12369B3B9FCF766FA01209EE7C4
:10871000636AE660002BF7D004F1240001F0E8F969
:108720000028F1D0094B4FF080521A60BFF34F8FF1
:10873000BFF36F8FE8E704F1100001F0D9F90028CA
:10874000E2D0EFE701F052FB6060DBE704ED00E010
:108750002DE9F84310B389469046054691B1FCF7E0
:1087600025FBEFF311874FF0500383F31188BFF31C
:108770006F8FBFF34F8FAC6BCCB9204687F3118856
:10878000BDE8F883036C002BE9D04FF0500383F36E
:108790001188BFF36F8FBFF34F8FFEE74FF0500389
:1087A00083F31188BFF36F8FBFF34F8FFEE795F808
:1087B00044604946284676B2FFF714FD013C731C1D
:1087C000AC6308D0731C5BB285F84430012087F39A
:1087D0001188BDE8F8832B69002BF7D005F1100054
:1087E00001F086F90028F1D0B8F1000FEED0012099
:1087F000C8F80000C2E700BF08B500F01BFF00206A
:1088000008BD00BFEFF305830BB100F05DBF00F0C2
:1088100055BF00BF30B5B0F9084085B0842C024682
:1088200014BF0334002403AD0B4640681168128A5C
:10883000CDE9004500F078FD01280CBF0398002029
:1088400005B030BD08B5012838BF012001F080F81F
:10885000002008BD00B5002385B0CDE90233EFF359
:108860000583ABB102AB0093012203AB01F084FBA3
:10887000012813D1029B3BB10A4B4FF080521A6082
:10888000BFF34F8FBFF36F8F039805B05DF804FB04
:1088900003AB012201F002FB0128F5D04FF00040AC
:1088A000F3E700BF04ED00E030B585B000230446D7
:1088B0000293EFF3058048B18223019304AB13E9DF
:1088C000070084E80700204605B030BD1346154672
:1088D00002AA01F097FA012805D00DB90195EDE73C
:1088E00040230193EAE7029B002BB4BF86230823B1
:1088F0000193E3E710B582B00024019410B3EFF3C5
:10890000058343B90A461946FFF750FE012816D1E0
:10891000002002B010BD01AA2146FFF719FF01286F
:108920000DD1019B002BF3D0084B4FF080521A6001
:10893000BFF34F8FBFF36F8F204602B010BDFF20F3
:1089400002B010BD802002B010BD00BF04ED00E0F9
:1089500010B582B000240194EFF305838BB101A917
:10896000FFF7CCFD012812D1019B9BB10B4B4FF0BF
:1089700080521A60BFF34F8FBFF36F8F204602B053
:1089800010BD1A461946FFF7F9FC012802D0FF2056
:1089900002B010BD002002B010BD00BF04ED00E029
:1089A000012910B502D00024204610BD084603223C
:1089B0000021FFF7D7FC04460028F5D000231A4613
:1089C0001946FFF7DBFC204610BD00BFFFF792BF42
:1089D000FFF7BEBF08B501F04FF9012800D108BD6F
:1089E000BDE80840FCF73EB9D0F81C3283B110B5A1
:1089F000D0F8184294F84000FF2807D09B6894F8FC
:108A0000412021469847FF2384F84030002010BDC4
:108A1000002070476A230380004870479C000020B4
:108A20000A2303800048704708010020012970B51F
:108A3000D0F8184205460E4616D0032912D16834E4
:108A400031462846FBF76EFFD5F8183260604BB10F
:108A5000D5F81C222146D46851F8040B3246A047B1
:108A6000002070BD022070BD5034E9E708B5D0F891
:108A7000183283B101290AD0032904BF002283F8E8
:108A80006420064B1868FFF7A3FF002008BD0022F2
:108A900083F84C20F5E7022008BD00BF9CC70020EA
:108AA000F8B50A7802F06003202B0C4606462DD05C
:108AB000402B0BD013B100252846F8BD4B780A2B6C
:108AC00004D101222749F9F7D7FA227812F00305D9
:108AD0000FD0012D13D16378502B10D1A388A57826
:108AE000052B0CD15DB9E2881F493046F9F7C4FA6D
:108AF000E2E76378502B02D1A388042B2CD03046B8
:108B000021460225FDF7A8FF2846F8BDCD888DB186
:108B10001306D0F8187215D5D0F81C3248789B6827
:108B20002A4639469847E28839463046F9F7A4FA8A
:108B30000025C1E7D0F81C3248789B682A46984740
:108B40002846F8BD4B7887F8403087F841502A46D0
:108B50003946F9F7A7FAAEE7E28804493046F9F753
:108B60008BFAA9E7450600203C01002014010020F3
:108B700010B581210446FBF76DFE01212046FBF76D
:108B800069FE82212046FBF765FE83212046FBF724
:108B900061FE20460321FBF75DFED4F8183253B185
:108BA000D4F81C325B689847D4F818021BF0DAF846
:108BB0000023C4F81832002010BD00BF38B50222CF
:108BC000044640238121FBF735FE40230222012188
:108BD0002046FBF72FFE4023022283212046FBF78D
:108BE00029FE4023022203212046FBF723FE08230F
:108BF000032282212046FBF71DFE74201BF0AAF8F9
:108C0000C4F81802D8B1D4F81C3205461B6898473E
:108C1000002385F84C302A6D85F85830012185F8FD
:108C20006430204685F870304023FBF76DFEAA6E55
:108C3000204640230321FBF767FE002038BD0120BA
:108C400038BD00BF6A230380004870479C000020A5
:108C50006A230380004870479C00002019B1C0F8C7
:108C60001C12002070470220704700BF012BD0F873
:108C7000180209D0032B05D100F15C03C3E90012EF
:108C8000002070470220704700F14403C3E900123E
:108C900000207047012AD0F8183207D0032A03D1E8
:108CA000683300201960704702207047503300205D
:108CB00019607047D0F8182210B56AB101290ED09A
:108CC000032909D192F864305C32832103F0FF0458
:108CD0006BB10124204610BD0224204610BD92F83D
:108CE0004C304432812103F0FF04002BF1D10123E9
:108CF000137293881268FBF7F9FD204610BD00BF80
:108D000008B5D0F818321BB101290AD0032901D0C7
:108D1000022008BD68331A684023FBF7F5FD0020E8
:108D200008BD5033F7E700BF036882B000206FF042
:108D30000402013901901A60032905D8DFE801F027
:108D4000070C11029B6C0193019802B07047DB6B1A
:108D50000193019802B070471B6C0193019802B017
:108D600070475B6C0193019802B07047F0B590F8C2
:108D70003C30CF69012B00F0D980012380F83C30D2
:108D80000E68092E70D803688A681C6906EB460CC9
:108D9000072505FA0CF524EA05041C611C6902FA92
:108DA0000CF222431A6134469A6BD1F810E04D68F8
:108DB00022F440129A639A6B0EF1FF3C42EA0C5C7B
:108DC000EA1CA2EB0E02C3F838C0D2B2D3F838C006
:108DD00002EB82024FF01F0E0EFA02FE2CEA0E0C7E
:108DE000C3F838C0D3F838E0DFF84CC104FA02F217
:108DF00042EA0E0267459A6372D09C68D1F820C09F
:108E000024F470249C609A6817439F609C6824F443
:108E100040149C609A6842EA0C029A608A69002AAF
:108E200039D05A6842F480625A604A69002A39D0BF
:108E30005A68022D42F480525A6039D0032D63D013
:108E4000012D56D01A6AC96822F47F6222F00F02FF
:108E50001A621A6A0A431A62354A934235D00023CD
:108E600080F83C301846F0BD03688A68D3F80CC01F
:108E7000B4B204EB44051E3D4FF0070E0EFA05FE9A
:108E80002CEA0E0CC3F80CC0D3F80CC0AA4042EA7E
:108E90000C02DA6088E75A6822F480625A604A69F4
:108EA000002AC5D15A68022D22F480525A60C5D1D9
:108EB0009A69C96822F47F6222F00F029A619A6966
:108EC0000A439A611A4A9342C9D1122E27D0103E02
:108ED000012EC4D8174A536843F400035360BEE719
:108EE0009A6822F470229A609A6822F440129A607A
:108EF00094E75A69C96822F47F6222F00F025A612E
:108F00005A690A435A61A7E7DA69C96822F47F629D
:108F100022F00F02DA61DA690A43DA619CE7D2F8DB
:108F2000043343F48003C2F8043398E70220F0BD11
:108F3000002001400023014001000F001049114BA7
:108F4000D1F8882042F4700210B4C1F888201A6861
:108F50000D4C002042F001021A6098601A6822F05D
:108F6000847222F480321A605C601A684FF00064E8
:108F700022F480221A60D8608C605DF8044B704740
:108F800000ED00E00038024010300024F0B58BB056
:108F90003D4B3E4F3E4E002400941A6B42F00402BB
:108FA0001A631A6B02F004020092009A01941A6B81
:108FB00042F080021A631A6B02F080020192019A59
:108FC00002941A6B42F001021A631A6B02F001025A
:108FD0000292029A03941A6B42F002021A631A6B0D
:108FE00002F002020392039A04941A6B42F0080200
:108FF0001A631B6B03F008030493384601224FF4F5
:10900000C041049B02F0EAF9224630464FF48051F9
:1090100002F0E4F90125384605A94FF4C043CDE933
:109020000535CDE9074402F001F8384605A948F2B4
:1090300010230593CDE9064401F0F8FF05A9304659
:109040000C230593CDE9064401F0F0FF304605A955
:109050004FF480530593CDE90654089401F0E6FFE0
:1090600005A94FF400430B480593CDE9064401F0F0
:10907000DDFF04230848059305A9CDE9064501F065
:10908000D5FF0BB0F0BD00BF003802400008024021
:109090000004024000000240000C02402DE9F041B3
:1090A000DFF8E4E0DEF800C086B00D46BCF1000F4A
:1090B00053D0304C4FEA0C1804EB0C17002602E09A
:1090C0001034BC420AD054F8041C8142F8D12188E3
:1090D000A94208BF261F1034BC42F4D1002E32D062
:1090E000B3600C9BF360244BB580306001A9CDE9DF
:1090F0000232019501F09AFF204B5D616D082FD07F
:109100002C460023013364089BB2FBD10F2B13D9EB
:10911000224621462046F8F737FF01346D08A4B2F5
:10912000FBD10F2C9ABF164B18572846F8F764FF4F
:10913000012006B0BDE8F08111492246C8562146FB
:10914000F8F722FFE9E7BCF10A0F10D00D4E0CF141
:1091500001014644CEF80010C2E70A4E0121F9E7AA
:1091600006202A462946F8F70FFF0620DEE730469C
:10917000DFE700BF5006002000001110003C014056
:109180007C9002084C06002048060020164B70B464
:109190001D68CDB1154B002403EB0515264605E0EF
:1091A0008A4208BF01241033AB420AD01A688242B7
:1091B0009A88F5D18A42F6D1C3E902661033AB42F0
:1091C000F4D10CB170BC7047480808BF062008D025
:1091D0000023013340089BB2FBD10F2B9CBF044AF4
:1091E000D05670BCF8F714BF480600204C0600208B
:1091F0007C90020870B5114886B00121FFF7C6FFC8
:109200000E480221FFF7C2FF022401A90123032611
:1092100008250A480595CDE90134CDE9034601F05A
:1092200005FF00230548039301A9CDE90144CDE9D9
:10923000046501F0FBFE06B070BD00BF00000240F7
:10924000F8B50E4F3B68BBB10D4C0646002504E057
:109250003B68AB4204F110040ED9A388B34205F178
:109260000105F5D1A368002BF2D0E06898473B6870
:10927000AB4204F11004F0D8F8BD00BF480600204E
:109280004C060020034A044B1268D268D268526828
:109290001A607047F0060020C8070020F8B51B4B85
:1092A0001B4E1D6833680446181D0F46FDF740FC31
:1092B00040B933681749D86A0B680122824023EA13
:1092C00002030B60631C17D033682C195C6007D352
:1092D000114B18683168BDE8F8400431FDF710BC47
:1092E0000E4B186831680431FDF70AFC0C4B1A6804
:1092F000A24288BF1C60F8BD002FE5D03168094844
:10930000BDE8F8400431FDF7EBBB00BF10080020BA
:10931000EC06002098070020F4060020F00600204C
:10932000C8070020E80700202DE9F84F4FEA82091E
:10933000074648460D469846FCF702FA002800F01A
:10934000848006465420FCF7FBF90446002800F010
:10935000898006634A463046A5211AF033FDD4F8C9
:1093600030A06E1E04F133030F3516F8012F03F8F9
:10937000012F32780AB1AE42F7D10A9D062D28BFDF
:1093800006254FF0000B261DE5626564304684F823
:1093900043B0C4F848B0A9F10409FDF79DFBC5F13D
:1093A000070504F11800D144FDF796FBC4F84CB052
:1093B000A56129F0070084F850B024616462424638
:1093C0003946FBF7BDFB0B9B206003B11C60FBF72C
:1093D000E1FB444ADFF85081136801331360D8F889
:1093E0000030002B47D0DFF84491D9F8003083B328
:1093F000E36A3D4ADFF838C11768DCF800E03B4813
:1094000001252F44176005FA03F203EB830342EAB8
:109410000E0200EB83003146CCF80020FDF760FB24
:10942000FBF7DAFBD9F8003013B3D8F80020E36A71
:10943000D26A9A421CD22E4B4FF080521A60BFF370
:109440004F8FBFF36F8F284601E04FF0FF30BDE82C
:10945000F88FD8F80020E36AD26A9A4298BFC8F819
:109460000040C6E73046FCF7FBF94FF0FF30EEE76F
:109470002846BDE8F88FC8F800401368012B03D0D8
:10948000E36ADFF8A890B4E718481A4F1A4DDFF8DE
:109490009C90FDF715FB1948FDF712FB1848FDF7E6
:1094A0000FFB1848FDF70CFB1748FDF709FB1748A1
:1094B000FDF706FB1648FDF703FB3846FDF700FBFA
:1094C0002846FDF7FDFA1348FDF7FAFA1248FDF7B2
:1094D000F7FA1248FDF7F4FA114B124A17601D60B3
:1094E000E36A86E78407002094070020F80600203E
:1094F00004ED00E09C070020B00700200C070020CE
:109500002007002034070020480700205C070020C7
:1095100070070020D0070020FC070020E80700208B
:10952000F4060020F0060020EC060020E4070020EE
:109530009807002070B50446324DFBF72BFB002C3A
:1095400048D0261D3046FDF7F3FA30B9E06A2E4BBD
:1095500000EB800253F822305BB3A36A1BB104F125
:109560001800FDF7E5FA294A29681368A14203F1BA
:109570000103136025D0264A206B1368013B13605A
:10958000FCF76EF92046FCF76BF9224B1B681B6851
:1095900053B1FFF777FEFBF71FFB1F4B1B6813B19F
:1095A0002B68A34218D070BD1C4B4FF0FF321A60DD
:1095B000F1E71B4901220B68824023EA02030B609A
:1095C000CBE718483146FDF78BFA174A1368013389
:1095D0001360E0E72C68B4E7144B1B6843B14FF00D
:1095E000500383F31188BFF36F8FBFF34F8FFEE7F4
:1095F0000F4B4FF080521A60BFF34F8FBFF36F8F46
:1096000070BD00BFEC060020F80600209407002083
:1096100084070020F0060020E4070020C80700208F
:1096200098070020FC0700208807002090070020F2
:1096300004ED00E030B583B0164B019300241649C9
:109640001648009423468022FFF76EFE012803D0BF
:10965000013016D003B030BD4FF0500383F31188B2
:10966000BFF36F8FBFF34F8F0D490E4A0E4B4FF074
:10967000FF350D6010601C6003B0BDE83040FBF7A3
:109680001DBB4FF0500383F31188BFF36F8FBFF3FF
:109690004F8FFEE7C40700208C90020899990008BC
:1096A000C8070020E407002010080020024A1368C1
:1096B00001331360704700BF90070020014B18680A
:1096C000704700BF1008002008B5FBF76FFB014B87
:1096D000186808BD100800202DE9F04F4B4B1B689F
:1096E00083B0002B4DD14A4B1E6801361E60002E00
:1096F00055D0484D2B68B34266D8DFF82891D9F889
:1097000000301C68002C77D0434FDFF82481DFF84D
:1097100024A1002427E00191FDF70AFADBF82820B4
:1097200001990BF1180012B1FDF702FA0199DBF86B
:109730002C00DAF800300122824000EB80001A434E
:1097400007EB8000CAF80020FDF7CAF9D8F800201E
:10975000D9F80000DBF82C10D26A0368914228BFC8
:109760000124002B4BD0D9F80030DB68D3F80CB0C3
:10977000DBF804200BF1040196420846CBD22A60A4
:1097800026E0264A1368013313600024244B1B682B
:10979000002B0CBF2046012003B0BDE8F08F214B09
:1097A0001A681268FAB9204A1868204914681C60BF
:1097B00010600A6801320A601B681B681BBB154DEC
:1097C0004FF0FF332B6095E7134FDFF864800024E0
:1097D000D8F80030DB6A03EB830357F82330022B01
:1097E00028BF0124D2E74FF0500383F31188BFF361
:1097F0006F8FBFF34F8FFEE7074FDFF834804FF0D6
:10980000FF332B60E4E7FFF73DFD72E79007002090
:1098100010080020C8070020F80600208C07002050
:1098200014080020F0060020F4060020CC070020D9
:10983000EC060020980700202DE9F84F394C2368EA
:1098400043B94FF0500383F31188BFF36F8FBFF319
:109850004F8FFEE7FBF79EF92368013B23602368E7
:10986000002B3CD1304B1B68002B38D02F4E336877
:10987000002B3AD0DFF8CC80DFF8CC90DFF8CCA01A
:109880002B4D0127F368DC6804F1040B04F1180088
:10989000FDF74EF95846FDF74BF9E06AD8F800207D
:1098A00007FA00F300EB80001343594609EB8000F0
:1098B000C8F80030FDF714F9DAF80030E16ADA6A26
:1098C0003368914228BF2F60002BDBD1194B1B68F6
:1098D0001B681BBB184B4FF0FF321A6006E00024D8
:1098E000FBF77AF92046BDE8F88F114D134E346826
:1098F0003CB10127FFF7F0FE00B12F60013CF9D128
:1099000034602B68002BEAD00D4B4FF080521A6068
:10991000BFF34F8FBFF36F8F0124E1E7FFF7B2FC76
:10992000E4E700BF9007002084070020D007002054
:1099300014080020F0060020C80700208C07002033
:1099400004ED00E098070020F8060020EC06002057
:1099500008B598B10E4B196841B14FF0500383F32D
:109960001188BFF36F8FBFF34F8FFEE71A68013284
:109970001A60FFF793FCFFF75FFF38B9054B4FF014
:1099800080521A60BFF34F8FBFF36F8F08BD00BFC7
:109990009007002004ED00E02DE988481E4D1F4E81
:1099A0001F4F204CDFF88080DFF880A04FF08059F7
:1099B00009E02B68D6F800B001332B60FFF73CFFBD
:1099C000BBF1000F0FD12368002BF2D1D8F8003083
:1099D000012B05D9CAF80090BFF34F8FBFF36F8FEB
:1099E00008F0C4F9EFE7FBF7D5F8F368D3F80CB04B
:1099F0000BF10400FDF79CF83B68013B3B602368DA
:109A0000013B2360FBF7E8F8DBF83000FBF728FFA9
:109A10005846FBF725FFD6E790070020FC070020FB
:109A20008407002088070020F806002004ED00E0ED
:109A300038B51D4B1B681BB11C4B01221A6038BD89
:109A40001A4A1B4C13602268236812681B6B9A42E7
:109A500024D9184B1B68B3FA83F3DBB2C3F11F039D
:109A600003EB830314499A0001EB8303885840B940
:109A70004FF0500383F31188BFF36F8FBFF34F8F05
:109A8000FEE75D6802F108006A685A6001448A4294
:109A900004BF52685A60D368236038BD20682168CB
:109AA000343108F053F9D4E790070020140800205F
:109AB000EC06002098070020F806002060B110B5E1
:109AC0000A4B0C4619681831FDF71AF82046012197
:109AD000BDE81040FFF7E2BB4FF0500383F311885D
:109AE000BFF36F8FBFF34F8FFEE700BFEC06002080
:109AF00070B5C368DC6882B0002C2DD004F1180169
:109B000008460191FDF714F8184B01991B6873B1D1
:109B10001748FCF7E5FF174BE26A1B68DB6A9A42BD
:109B200085BF154B01200020186002B070BD211DBB
:109B3000124D01910846FCF7FBFFE26A2E681048BF
:109B400001990123934002EB8202334300EB820030
:109B50002B60FCF7C5FFDEE74FF0500383F311885D
:109B6000BFF36F8FBFF34F8FFEE700BF900700205A
:109B7000D0070020EC0600201408002098070020E1
:109B8000F806002030B1084A084B12681B68C0E98B
:109B9000002370474FF0500383F31188BFF36F8F9A
:109BA000BFF34F8FFEE700BFCC0700201008002056
:109BB000F8B548B30D46F1B10446FAF7EBFF2B6850
:109BC0001B485A1C01682DD01A4E276832689742EC
:109BD000626801D08A4220D98F1ABB421DD95B1A14
:109BE0001344316802682B60C4E900120025FAF7BB
:109BF000F3FF2846F8BD4FF0500383F31188BFF3FD
:109C00006F8FBFF34F8FFEE74FF0500383F3118840
:109C1000BFF36F8FBFF34F8FFEE70125FAF7DCFF2D
:109C20002846F8BD0025FAF7D7FF2846F8BD00BF43
:109C300010080020CC070020014B01221A60704759
:109C40001408002068B1036B1A78A52A0FD1C3F15C
:109C50000101C81813F8012FA52AFAD0C0F38F000C
:109C60007047044B1868036B1A78A52AEFD00020C0
:109C7000704700BFEC060020054B1B6833B1054B55
:109C80001B68002B0CBF022000207047012070478A
:109C9000E407002090070020E8B1F0B5224DC36A28
:109CA0002A68D26A934283B0044612D28269002A9B
:109CB00004DB2A68D26AC2F1070282611B4E626924
:109CC00003EB830306EB83039A4205D02B68DB6A20
:109CD000E36203B0F0BD7047211D08460191FCF717
:109CE00027FF019970B9E36A03EB830256F822203B
:109CF00042B90F4A0127106807FA03F320EA030369
:109D0000136000E00A4A2B681568D86AE0620123F4
:109D1000834000EB80002B4306EB8000136003B010
:109D2000BDE8F040FCF7DCBEEC060020F8060020A1
:109D300098070020D8B1F0B5294B1B68834283B047
:109D4000044608D04FF0500383F31188BFF36F8FA0
:109D5000BFF34F8FFEE79B6C5BB1C16A426C013B66
:109D60009142836400D06BB1002003B0F0BD0020AD
:109D700070474FF0500383F31188BFF36F8FBFF329
:109D80004F8FFEE7011D08460191FCF7D1FE0199B6
:109D9000B0B11448144A636CD2F800C0E3620125E4
:109DA00005FA03F6C3F1070703EB830346EA0C0643
:109DB00000EB8300A7611660FCF792FE2846D4E70B
:109DC000E66A0848084A06EB860350F82330002B61
:109DD000E1D113680125B54023EA05031360DAE7F2
:109DE000EC060020F806002098070020044B1A68B3
:109DF0001AB119688A6C01328A641868704700BF0A
:109E0000EC0600202DE9F041224C82B00E460746B8
:109E100015469846FAF7BEFE216891F850100229BF
:109E20000BD02368D96C21EA0701D964236801218A
:109E300083F85010B8F1000F1DD1FAF7CDFEFAF7F4
:109E4000A9FE15B12368DB6C2B60236893F85030B2
:109E5000012B1CD02368D96C21EA0606DE640120A0
:109E600023680190002283F85020FAF7B5FE01988C
:109E700002B0BDE8F0814046FFF710FA064B4FF004
:109E800080521A60BFF34F8FBFF36F8FD5E700206A
:109E9000E6E700BFEC06002004ED00E0B8B1F0B545
:109EA0001D4683B00F4616460446FAF773FE0DB101
:109EB000E36C2B6094F850500222731EEDB284F8CC
:109EC0005020032B0FD8DFE803F048440D0B4FF070
:109ED000500383F31188BFF36F8FBFF34F8FFEE7FB
:109EE000022D3ED0E764012D05D00125FAF774FE5E
:109EF000284603B0F0BD211D1B4E01910846FCF71A
:109F000017FEE36A37681948019905FA03F203EB73
:109F100083033A4300EB83003260FCF7E1FDA36A60
:109F200043B14FF0500383F31188BFF36F8FBFF33A
:109F30004F8FFEE70E4BE26A1B68DB6A9A42D4D968
:109F40000C4B4FF080521A60BFF34F8FBFF36F8FEF
:109F5000CCE7E36C0133E364C5E7E36C1F43E764DC
:109F6000C1E70025C2E700BF98070020F8060020DF
:109F7000EC06002004ED00E02DE9F04383B00A9FD9
:109F800000B3894690461D460446FAF70FFFEFF3EB
:109F900011864FF0500383F31188BFF36F8FBFF327
:109FA0004F8F0DB1E36C2B6094F85050022208F1F2
:109FB000FF33EDB284F85020032B10D8DFE803F014
:109FC0004B470D0B4FF0500383F31188BFF36F8F96
:109FD000BFF34F8FFEE7022D42D0C4F84C90012D05
:109FE00005D0012086F3118803B0BDE8F083A36A91
:109FF00043B14FF0500383F31188BFF36F8FBFF36A
:10A000004F8FFEE71C4B1B6863BB211D0846019167
:10A01000FCF78EFDDFF874C0E26ADCF800E0174858
:10A02000019905FA02F302EB820243EA0E0300EB08
:10A030008200CCF80030FCF753FD114BE26A1B683C
:10A04000DB6A9A42CDD99FB101203860CAE7E36C40
:10A050000133E364C3E7E36C43EA0903E364BEE767
:10A060000020BFE7074804F11801FCF739FDE4E7D9
:10A07000054B01201860B5E790070020F806002086
:10A08000EC060020D00700201408002098070020CC
:10A09000036A23F001030362F0B4036A134C4768B8
:10A0A00082698E680D6823F0020322F07302A042D9
:10A0B00043EA060342EA05020AD004F58064A0429E
:10A0C00006D0496847608261F0BC41630362704713
:10A0D000D1E90556CC6823F00803234327F44077E1
:10A0E00045EA060423F004032743EAE700000140A1
:10A0F000036A23F480730362F0B4036A144C476864
:10A10000C2698E680D6823F4007322F07302A042C6
:10A1100043EA062342EA05020AD004F58064A0421D
:10A1200006D049684760C261F0BCC16303627047F2
:10A13000D1E90556CC6823F4006343EA042327F4ED
:10A14000405745EA060423F4806347EA0417E8E72A
:10A1500000000140036A23F480530362F0B4036AF1
:10A160000F4F4668C2698D680C6823F4005322F4CF
:10A17000E642B84243EA053342EA042209D0094CD8
:10A18000A04206D049684660C261F0BC0164036227
:10A1900070474C6926F4804646EA8416F2E700BF11
:10A1A0000000014000040140034600201B68DA68FB
:10A1B00042F00102DA601A6842F001021A60704748
:10A1C000704700BF03680122186A02FA01F120EA11
:10A1D000010010B418621A6A0A4C1143A3421962B2
:10A1E0000AD0094A934207D01A685DF8044B42F03E
:10A1F000010200201A6070475A6C42F400425A640F
:10A20000F2E700BF000001400004014010B40C2937
:10A2100008D8DFE801F032070707380707072C07DF
:10A22000070726000368186A1A4C012202FA01F196
:10A2300020EA010018621A6AA34241EA0201196287
:10A240000AD0154A934207D01A685DF8044B42F0D1
:10A25000010200201A6070475A6C42F400425A64AE
:10A26000F2E70368DA6842F01002DA60DBE70368BD
:10A27000DA6842F00802DA60D5E70368DA6842F08B
:10A280000202DA60CFE70368DA6842F00402DA60BB
:10A29000C9E700BF0000014000040140FFF792BF82
:10A2A000FFF7B4BF0C2908D8DFE801F01E07070745
:10A2B000240707072A07070718000368186A0122FE
:10A2C00002FA01F120EA010018621A6A11431962C8
:10A2D0001A6842F001021A60002070470368DA68C9
:10A2E00042F01002DA60E9E70368DA6842F002023D
:10A2F000DA60E3E70368DA6842F00402DA60DDE777
:10A300000368DA6842F00802DA60D7E7C1B10429CD
:10A3100020D003681A6A22F001021A621A6A42F017
:10A3200001021A621A6A22F010021A621A6A42F0D4
:10A3300010021A621A6842F001021A600020704787
:10A3400003681A6A22F001021A621A6A42F00102D4
:10A350001A62EFE70368E5E790F83830012B00F068
:10A360009880F0B402680124022380F8384080F815
:10A37000393094680B6824F47F4424F07704502B20
:10A38000946000F0888027D8202B00F09C803AD978
:10A39000302B70D0402B16D1156A166A4C68CF68E6
:10A3A00026F001061662936925F00A0123F0F003F6
:10A3B00043EA0713214393611162936823F070030A
:10A3C00043F0470393600023012280F8392080F88E
:10A3D0003830F0BC18467047B3F5805F7AD01DD98D
:10A3E000B3F5005FEFD1D1E90153CC6891682B43FD
:10A3F00043EA042321F47F410B439360936843F4C1
:10A4000080439360DFE7002B3CD0102BDBD19368B7
:10A4100023F0700343F017039360D4E7602B11D04F
:10A42000702BD0D1D1E90153CC6891682B4343EA1A
:10A43000042321F47F410B439360936843F0770337
:10A440009360C0E7146A4D68CE6824F0100414626B
:10A450009169136A21F4704123F0A00343EA0513C4
:10A4600041EA063191611362936823F0700343F06F
:10A4700067039360A7E7936823F0700343F0370303
:10A480009360A0E7936823F0700343F007039360A1
:10A4900099E702207047156A166A4C68CF6826F063
:10A4A00001061662936925F00A0123F0F00343EADE
:10A4B0000713214393611162936823F0700343F003
:10A4C000570393607FE7936823F0700343F02703FB
:10A4D000936078E7936823F00703936073E700BF06
:10A4E000704700BF704700BF704700BF704700BF94
:10A4F00003681A69910710B5044602D5DA68920715
:10A500005FD41A69500702D5DA68510746D41A6930
:10A51000120702D5DA6810072ED41A69D20602D5BE
:10A52000DA68D00618D41A69D10702D5DA68D207DA
:10A530005DD41A69100602D5DA6811065FD41A696B
:10A54000520602D5DA68500661D41A69910602D51E
:10A55000DA68920643D410BD6FF010010822196129
:10A560002276DB6913F4407F204664D0FFF7BAFF00
:10A57000002223682276D6E76FF0080104221961D1
:10A580002276DB699907204652D1FFF7A9FF2046C2
:10A59000FFF7AAFF002223682276BEE76FF00401CE
:10A5A0000222196122769B6913F4407F20463CD138
:10A5B000FFF796FF2046FFF797FF002223682276D9
:10A5C000A5E76FF002010122196102769B699B07E2
:10A5D00025D0FFF787FF00222368227691E76FF0EE
:10A5E000200220461A61BDE81040F9F733BA6FF037
:10A5F00001021A612046FAF707F8236899E76FF01D
:10A6000080021A612046F9F727FA236897E76FF06E
:10A6100040021A612046FFF769FF236895E7FFF7BC
:10A620005FFF2046FFF760FFD5E7FFF75BFFC4E75A
:10A63000FFF758FFAEE7FFF753FF2046FFF754FF41
:10A6400096E700BF2E4A0368904230B444D0B0F180
:10A65000804F30D0A2F57C4290422CD002F580622F
:10A66000904228D002F58062904224D002F57842D0
:10A67000904231D002F57052904220D002F58062B3
:10A6800090421CD002F58062904218D0A2F5983218
:10A69000904214D002F58062904210D002F58062A0
:10A6A00090420CD08C680A6803600123C462826205
:10A6B00030BC436170474A6823F070031343D1E90B
:10A6C000024523F440732B430A6803600123C462EC
:10A6D000826230BC436170474C68CA6823F07003E3
:10A6E000234323F44073134303608B68C3620B68F6
:10A6F00083620B690363012330BC4361704700BF71
:10A7000000000140C0B110B590F83930044603F0A4
:10A71000FF0263B10223214684F8393051F8040B5B
:10A72000FFF790FF012384F83930002010BD80F836
:10A730003820F8F763FEEDE701207047C0B110B58F
:10A7400090F83930044603F0FF0263B1022321463A
:10A7500084F8393051F8040BFFF774FF012384F8B3
:10A760003930002010BD80F83820FFF729FDEDE7D3
:10A7700001207047C0B110B590F83930044603F09D
:10A78000FF0263B10223214684F8393051F8040BEB
:10A79000FFF758FF012384F83930002010BD80F8FE
:10A7A0003820F8F769FEEDE701207047C0B110B519
:10A7B00090F83930044603F0FF0263B102232146CA
:10A7C00084F8393051F8040BFFF73CFF012384F87B
:10A7D0003930002010BD80F83820F8F7C9FEEDE7C9
:10A7E0000120704700284DD0F0B590F8393083B083
:10A7F0000C46054603F0FF02002B3ED029460223FB
:10A8000085F8393051F8040B836823F0070383601F
:10A81000FFF718FF2968236988688E69A769A2680D
:10A82000D4F800C026F4407EE6691B0143EA062303
:10A83000266A0196E6683343019E2EF0030E42EA33
:10A84000072242EA0E020F6A43EA06336669646829
:10A8500022F47C4244EA061440EA0C0022F0FC0296
:10A8600027F0AA07886027431343012400208B6147
:10A870000F6285F8394003B0F0BD80F83820F8F752
:10A8800039FEBBE70120704770B4046A1C4E24F007
:10A8900001040462B0428469056A1FD0B0F1804FA0
:10A8A0001CD0A6F57C46B04218D006F58066B042B2
:10A8B00014D006F58066B04210D006F57846B04256
:10A8C0000CD006F57056B04208D0A6F59436B042CA
:10A8D00004D024F0030242F0010202E024F0030459
:10A8E00022431B0125F00A04DBB222F0F00201F042
:10A8F0000A0121431343836170BC0162704700BFAA
:10A9000000000140F8B590F83830012B00F08C8041
:10A910000D4602230121044680F8381080F83930B2
:10A9200072B3042A03683BD0082A1E6A2A685BD0E7
:10A9300026F480566F68D5E902511E62D8691E6AF6
:10A9400020F440701203090340EA072002F4204279
:10A9500089B220F4704026F4204632430143D96185
:10A960001A62DA6922F44062DA61DA6942EA05259C
:10A97000DD610123002084F8393084F83800F8BD07
:10A98000D5E90012EB680068FFF77EFF2368A8682E
:10A99000996921F00C0199619A6902439A61E8E78B
:10A9A0001E6A2A686F6826F01006D5E902511E62F9
:10A9B00098691E6A20F440701201090340EA0720DA
:10A9C00002F0A00289B220F4704026F0A0063243C3
:10A9D000014399611A629A6922F440629A619A6904
:10A9E00042EA05259D61C4E726F480766868D5E9CA
:10A9F00002511E62DF691E6A27F003071202090175
:10AA0000384302F42062C9B220F0F00026F4206638
:10AA100032430143D9611A62DA6922F00C02DA6129
:10AA2000DA692A43DA61A4E70220F8BD036A23F059
:10AA300010030362F0B4036A144C476882698E689D
:10AA40000D6823F0200322F4E642A04243EA0613F5
:10AA500042EA05220AD004F58064A04206D0496883
:10AA600047608261F0BC816303627047D1E905569B
:10AA7000CC6823F0800343EA041327F4406745EAD7
:10AA8000060423F0400347EA8407E8E7000001409A
:10AA900090F83830012B28D010B50446022301204D
:10AAA00084F8380084F839300C2A0BD8DFE802F03B
:10AAB000070A0A0A150A0A0A190A0A0A110020686E
:10AAC000FFF7E6FA0123002084F8393084F83800D3
:10AAD00010BD2068FFF73EFBF4E72068FFF7A6FFF4
:10AAE000F0E72068FFF704FBECE70220704700BFA7
:10AAF00038B590F83830012B74D00D46022301216F
:10AB0000044680F8381080F839300C2A19D8DFE86C
:10AB100002F00718181838181818511818181F00BC
:10AB200000682946FFF7B4FA23682869996941F05B
:10AB300008019961996921F0040199619A690243B8
:10AB40009A610123002084F8393084F8380038BD38
:10AB500000682946FFF7FEFA23682869D96941F49D
:10AB60000061D961D96921F48061D961DA6942EA69
:10AB70000022DA610020012384F8393084F838009B
:10AB8000E5E700682946FFF751FF236828699969BE
:10AB900041F400619961996921F4806199619A6930
:10ABA00042EA00229A610020012384F8393084F8B7
:10ABB0003800CCE700682946FFF79AFA236828692D
:10ABC000D96941F00801D961D96921F00401D9613D
:10ABD000DA690243DA610020012384F8393084F80D
:10ABE0003800B4E7022038BD002800F09E80F8B598
:10ABF000036C04463BB1236CDB060CD5002384F8C0
:10AC00003C300120F8BD436480F83C30FBF790FCF9
:10AC1000236CDB06F2D4226C47492368474D22F4AB
:10AC2000885222F0020242F0020222644A6822F4B0
:10AC300040324A604A68606802434A605868216945
:10AC4000A768E66820F4807058605A6842EA0122DA
:10AC50005A60586820F0407058605968A06A3943BB
:10AC60005960996821F4006199609A68A84242EAA3
:10AC700006029A6050D09968E56A21F07061996087
:10AC80009A6810439860996821F0405199609A68D9
:10AC90002A439A609968A569206A21F002019960A7
:10ACA0009A6842EA45029A605A6800283FD042F406
:10ACB0000062616A5A605A6822F460425A605A68B7
:10ACC000013942EA41325A60DA6AE569276B6669FE
:10ACD00022F47002DA62D86A013D40EA0550D86277
:10ACE000986820F400709860996841EA472199605B
:10ACF000996821F4806199609A68002042EA86226E
:10AD00009A606064236C23F0030343F0010323641F
:10AD1000002384F83C30F8BD9A6822F070629A6093
:10AD20009A6822F040529A60B4E70120704722F4FA
:10AD300000625A60C8E700BF002301400100000F15
:10AD4000F0B5054690F83C0083B00024012801943A
:10AD500068D001232E6885F83C30B368DC0714D432
:10AD6000324B334C1868B368A4FB0040800C43F0AE
:10AD7000010300EB4000B3600190019B2BB1019CEB
:10AD8000013C019401980028F9D1B368D8073CD55B
:10AD9000286C20F4E06020F0010040F4807028640A
:10ADA00073685B0505D52B6C23F4405343F4805343
:10ADB0002B642B6CA86B1F4C13F480531CBF6B6C63
:10ADC00023F006036B6400271B4B85F83C70C463BB
:10ADD00003641A4CC4646FF022033360736843F059
:10ADE00080637360B46844F480741346B4600A46A8
:10ADF00006F14C01FAF7E8FA114B5B6813F01F0FEC
:10AE00002B6805D00F4A934202D0002003B0F0BD5A
:10AE1000986810F04050F8D19A6842F080429A60E9
:10AE200003B0F0BD022003B0F0BD00BFF40100206C
:10AE300083DE1B4355AE0008B5AE0008C5AE000862
:10AE400000230140002001400368D86C704700BF18
:10AE5000704700BF836B1A6C12F0500F25D11A6C2B
:10AE6000196842F4007210B51A648A6812F0405FE3
:10AE700017D19A69AAB9CA6A12F4700F02D08A6807
:10AE800050050ED44A6822F020024A601A6C22F45F
:10AE900080721A641A6CD20403D41A6C42F0010254
:10AEA0001A641846FFF7D4FF10BD9B6BDB6C184784
:10AEB000704700BF08B5806BFFF7FAFF08BD00BF01
:10AEC000704700BF806B08B540230364436C43F0B8
:10AED00004034364FFF7F4FF08BD00BFF0B490F82B
:10AEE0003C3082B00022012B019200F094800123BB
:10AEF00080F83C300D68092D29D804688B682269D8
:10AF000005EB45070726BE4022EA060222612269B8
:10AF1000BB40134323614B68062B2E462CD803EB12
:10AF20008303626B053B1F21994022EA01026263A1
:10AF3000626B06FA03F313436363394B9C422FD0D1
:10AF4000002380F83C30184602B0F0BC704704681B
:10AF50008B68E768AEB206EB46021E3A4FF0070C6C
:10AF60000CFA02FC27EA0C07E760E76893403B43D2
:10AF7000E3604B68062BD2D90C2B37D803EB830345
:10AF8000A3F123011F22236B8A4023EA02032363D8
:10AF9000236B06FA01F11943214B21639C42CFD167
:10AFA000122D32D0A5F11003012BC9D81D4A5368C8
:10AFB000102D43F400035360C2D11B4B02F14672C3
:10AFC0001B6802F52E3202F28332A2FB03239B0C94
:10AFD00003EB83035B000193019B002BB0D0019B2B
:10AFE000013B0193019B002BF9D1A9E703EB8302FD
:10AFF000413AE36A1F21914023EA0103E362E36AD5
:10B0000006FA02F11943E16297E7064A536843F4EE
:10B010008003536094E7022002B0F0BC704700BF89
:10B020000020014000230140F40100202DE9F04FF1
:10B0300000230E68DFF83882DFF838E283B003E0DF
:10B040000133102B00F0A18001229A4032EA06045D
:10B0500002EA060CF4D14D6825F0100ABAF1020F8D
:10B0600000F09680D0F800B04FEA4309032404FAB8
:10B0700009F405F003072BEA040B07FA09F70AF1B4
:10B08000FF3A47EA0B07BAF1010F6FEA04040760C1
:10B0900040F2A480C7688A683C4002FA09F2224361
:10B0A000EF00C260CCD500220192D8F8442042F4CF
:10B0B0008042C8F84420D8F8442023F0030404F167
:10B0C000804402F4804204F59C34019203F00307AB
:10B0D000019AD4F80890BF000F22BA4029EA020A68
:10B0E0005D4A904224D002F58062904200F089804F
:10B0F0005A4A904200F08C80594A904200F08F806A
:10B10000584A904200F09280574A904200F0958051
:10B11000564A904200F09880DFF85C9148450CBF99
:10B120004FF007094FF0080909FA07F74AEA070A3A
:10B13000C4F808A0DEF800206FEA0C07EC0354BF47
:10B140003A404CEA0202CEF80020DEF80440AA039E
:10B1500054BF3C404CEA0404CEF80440DEF80840FA
:10B16000EA0254BF3C404CEA0404CEF80840DEF842
:10B170000C20AC0203F1010354BF3A404CEA020236
:10B18000102BCEF80C207FF45FAF03B0BDE8F08F3A
:10B190004FEAD30900EB890903F00707D9F82040EB
:10B1A000BF004FF00F0B0BFA07FB24EA0B0A0C69E8
:10B1B000BC4044EA0A04C9F82040D0F800A04FEA95
:10B1C0004309032404FA09F405F003072AEA040AF0
:10B1D00007FA09F747EA0A07E4430760876807EABE
:10B1E000040ACF6807FA09F747EA0A078760D0F828
:10B1F00004A0C5F300172AEA02029F4017434760E4
:10B2000048E74FF0010909FA07F74AEA070A8FE70A
:10B210004FF0020909FA07F74AEA070A88E74FF0F0
:10B22000030909FA07F74AEA070A81E74FF0040918
:10B2300009FA07F74AEA070A7AE74FF0050909FA17
:10B2400007F74AEA070A73E74FF0060909FA07F712
:10B250004AEA070A6CE700BF00000240000802400B
:10B26000000C02400010024000140240001802408E
:10B2700000380240003C0140001C02402DE9F04F24
:10B280000023DFF840A1DFF84081DFF840B18E46AF
:10B2900002E00133102B70D0012606FA03F232EAE5
:10B2A0000E01F6D104684FF0030C03FA06F10CFA14
:10B2B00001F123FA0CF524EA010400EB8505046092
:10B2C00003F00704D5F820900F27A40007FA04F430
:10B2D00029EA04042C62846824EA01048460446836
:10B2E00024EA02044460C56823F0030404F18044A6
:10B2F00025EA010104F59C34C16003EA0C01A5684C
:10B3000089008F4050456FEA020205EA070536D0F2
:10B31000584539D0254EB04239D0254EB0423AD0AA
:10B32000244EB0423AD0244EB0423BD0234EB042DD
:10B3300029D0234EB0420CBF0726082606FA01F199
:10B340008D42A6D1A16821EA0707A760D8F80010AE
:10B350001140C8F80010D8F804101140C8F80410C3
:10B36000D8F808101140C8F80810D8F80C100133AC
:10B370000A40102BC8F80C208ED1BDE8F08F0021B8
:10B380008D4286D1DEE7062606FA01F1F8E70226AD
:10B3900006FA01F1F4E70CFA01F1F1E7042606FAE6
:10B3A00001F1EDE7052606FA01F1E9E700080240A0
:10B3B000000C02400010024000140240001802403D
:10B3C000001C024000000240003C0140000402401A
:10B3D0000369194214BF01200020704702B9090413
:10B3E00081617047044A5169014200D1704708B534
:10B3F0005061FDF725FF08BD003C014000286BD0DF
:10B4000070B590F83D30044603F0FF02002B4ED09B
:10B410002268324D242384F83D30136823F0010361
:10B420001360FCF7AFF9D4E900212D4BA3FB0063B7
:10B430009B0CA942536025D840F6FC7549000133A6
:10B44000B0FBF1F02842136208BF0420D4E90735AD
:10B45000D4E90361D06143EA0500D4E905353143FD
:10B460002B4310609160D3601168002341F001010B
:10B4700020251160236484F83D50236384F83E3016
:10B48000184670BD4FF49675164E05FB03F3A6FBE8
:10B4900003539B09A568013313626DB901EB4101A8
:10B4A000B0FBF1F0C0F30B039BB90120CEE780F8AD
:10B4B0003C2000F02DFEABE701EB810101EB8101A7
:10B4C000B0FBF1F0C0F30B03002BEED040F4404092
:10B4D000BCE740F40040B9E701207047A0860100B6
:10B4E00083DE1B43D34D6210F0B490F83D40282C0E
:10B4F00082B034D100292ED0002A2CD090F83C40C4
:10B50000012C2CD005682C68E40703D42C6844F087
:10B5100001042C602C6824F400642C60292700248A
:10B52000202680F83D7080F83E6004644285C36246
:10B53000428D01946B690193AB69019380F83C40A3
:10B54000019B6B684162028543F4E06320466B60B7
:10B5500002B0F0BC7047012002B0F0BC704702207E
:10B5600002B0F0BC704700BFF0B490F83D40282C0A
:10B5700082B034D100292ED0002A2CD090F83C4043
:10B58000012C2CD005682C68E40703D42C6844F007
:10B5900001042C602C6824F400642C602A27002409
:10B5A000202680F83D7080F83E6004644285C362C6
:10B5B000428D01946B690193AB69019380F83C4023
:10B5C000019B6B684162028543F4E06320466B6037
:10B5D00002B0F0BC7047012002B0F0BC70470220FE
:10B5E00002B0F0BC704700BF90F83D30202B01D076
:10B5F000022070472822036880F83D201A68D2078D
:10B6000003D41A6842F001021A601A6842F4806298
:10B610001A605A6842F440725A600020704700BFB6
:10B62000704700BF704700BF704700BF704700BF42
:10B63000704700BF704700BF704700BF10B590F85B
:10B640003D30293B012B044658D990F83D30602B02
:10B65000036805D05A6812055CBF202280F83D209F
:10B660000022226384F83E201A6822F400621A60E5
:10B670005A6812F400622DD05A68606B22F400629E
:10B680005A6090F83530012B3FD03A4B0365F9F7FB
:10B6900025FF50B12268606B1368202123F001035D
:10B6A000136084F83D10036D984794F83D30282BC3
:10B6B00000D010BD236C5B07FBD52F4BE36220222B
:10B6C00000232363204684F83D2084F83E3016F0A2
:10B6D00083FF10BD94F83D10602932D05A6952069C
:10B6E00004D5626A1B69511C61621370204616F012
:10B6F0009DFF94F83D30282BDBD1DBE70023282287
:10B700000363036880F83D20AEE7A06B194B036527
:10B71000F9F7E4FE0028C8D023685A69500605D519
:10B72000626A1B69511C6162137023681A68A06BFE
:10B7300022F0010220211A6084F83D10036D984721
:10B74000B3E7202184F83D1022645A69510605D5DB
:10B75000626A1B69511C6162137023681A6822F0C7
:10B7600001021A602046FFF767FF94F83D30282B4E
:10B770009FD19FE77DC000080000FFFFF0B5036880
:10B780009D695A695C6890F83E1010298DB03DD0D3
:10B79000CEB2402E3AD099491140002900F0CC8019
:10B7A000A10500F17E8196492940002900F03481ED
:10B7B00094491140002900F08181650540F17E81A6
:10B7C00091491140002940F07E8190F83D10428D52
:10B7D00092B2C9B2C2B1426A541C446212781A6170
:10B7E000428D013A92B24285428D92B262B92929C4
:10B7F0000AD15A68212422F4806228215A60046305
:10B8000080F83D10FFF710FF0DB0F0BD12F0011FE2
:10B8100039D0A60500F130817C491140002966D05D
:10B820007749294000293BD076491140002977D03B
:10B83000670575D574491140002900F08281A6057D
:10B84000E2D5C16A90F83D20212ADDD1428D92B225
:10B85000002A40F04081042900F00382082900F00A
:10B86000008211F5803F00F0FC815968112521F418
:10B87000E06120245960056380F83E2080F83D4057
:10B88000FFF7CEFEC0E76149114000292FD0A10586
:10B89000C6D5416CC9B21961594929400029C3D1A3
:10B8A0005B491140002941D065053FD556491140FB
:10B8B000002900F02881A405A6D5C16A428D92B264
:10B8C000042A00F0B381428D92B2032A00F0BF81B6
:10B8D000428D92B2022A00F0FE81426A1B69511C1D
:10B8E00041621370438D013B9BB243858CE7434912
:10B8F0001140002994D0A70592D590F83E10C76A50
:10B90000D0F830C090F83D60222EC9B200F04781D7
:10B9100000210A9159690A9199690A910A997FE768
:10B920003949114000298AD10DB0F0BD3649114086
:10B930000029C0D10DB0F0BD364E1640002E3FF4A8
:10B9400032AFA6057FF52FAF90F83D405A6822F43C
:10B95000E0625A600B915A690B921A6842F0010238
:10B960001A600B9A1A6822F480621A605A681205EB
:10B97000E4B20ED590F83D20222A00F04B8190F8D9
:10B980003D202A2A00F04681426B1268526892B22A
:10B990004285428D92B2C2B15A69570709D5426AAF
:10B9A0001B69511C41621370428D0368013A92B2C7
:10B9B00042855A69560608D5426A1B69511C416284
:10B9C0001370438D013B9BB24385036C002B40F009
:10B9D000E180A4F12802022A40F20581036B222BA8
:10B9E00002D0222C7FF410AF00232022036380F8C2
:10B9F0003D2080F83E30FFF719FE05E70200010008
:10BA00000400100080000100040001000800010093
:10BA100040000100100001009D491140002964D040
:10BA2000610562D59B491140002963D190F83D1012
:10BA3000428D92B2C9B2002A3FF4E6AE426A1B6957
:10BA4000541C44621370438D013B9BB24385438D6C
:10BA50009BB2002B7FF4D8AE2A297FF4D5AE0268C2
:10BA60005368222423F4806328215360046380F800
:10BA70003D10FFF7DBFDC7E690F83E10402900F0CF
:10BA8000AB800169B1F5804F78D0016D002940F09D
:10BA9000B580416CC91101F0060141F0F001196156
:10BAA000BEE699699B6981F004011F0654BF828933
:10BAB000028BC1F3800116F099FDA5E6754911408E
:10BAC00000293FF4A1AEA4057FF59EAE428D92B24F
:10BAD000002A3FF499AE426A511C416212781A6101
:10BAE000438D013B9BB243858EE66A491140002994
:10BAF0003FF48AAEA2057FF587AE428D92B2002A4E
:10BB00003FF482AEE9E690F83D20222A7FF47CAE35
:10BB1000428D92B2032A40F22181426A1B69511C74
:10BB200041621370438D013B9BB24385438D9BB2B1
:10BB3000032B7FF469AE0268536823F4806353607B
:10BB400062E690F83D20048D90F83E10C56AD2B2AE
:10BB5000C9B2002C78D1212A00F0EB8040297FF473
:10BB600053AE222A7FF450AE428D92B2002A40F0AA
:10BB700016815A6822F480625A6045E690F83D10BA
:10BB80002129416C16BF41F0010101F0FE01C9B24B
:10BB9000196145E60DB0BDE8F040FFF74FBD066DF9
:10BBA00016B9402900F01081066D26B90169B1F57A
:10BBB000404F00F01081418D89B200296ED1039170
:10BBC00059690391996903910399196841F40071C6
:10BBD00019600021016523E6016D09BB416C01F08C
:10BBE000FE0119611CE62C4AC2622022036380F820
:10BBF0003D2080F83E3016F0EFFC05E6016D01298E
:10BC00007FF40EAE416CC91101F0060141F0F10163
:10BC1000196105E6826B1268526892B24285B8E6F5
:10BC2000416C41F00101C9B21961F9E55A68416AF4
:10BC300022F480625A601B694A1C42620B70438D79
:10BC4000013B9BB24385DFE5212A8DD086E75A6808
:10BC5000416A22F480625A601A6822F480621A6093
:10BC6000E9E75A6822F4E0625A601A68002142F457
:10BC7000007220241A60016380F83D4090F83E3045
:10BC800080F83E10402B7FF4FBADFFF7D1FCBBE505
:10BC900040000100040001000000FFFF418D89B257
:10BCA000012900F0AE80418D89B2022900F0C480E4
:10BCB000196841F4806119605968090503D559680C
:10BCC00041F480515960002109915969099199699C
:10BCD000099109997DE7013901291A6840F28980A3
:10BCE00042F400721A60426A1B69511C416213706F
:10BCF000438D426A0168013B9BB243850B69511C2D
:10BD000041621370438D0168013B9BB243854B68D0
:10BD1000002223F4407320244B6080F83D400263EE
:10BD200090F83E3080F83E20402B35D0FFF77AFC6B
:10BD30006AE5042D95D0082D93D015F5803F90D05D
:10BD40005A68112522F4E06220215A60056380F8C8
:10BD50003E4080F83D10FFF763FC55E5012A3FF6B1
:10BD600053AD1A68446A22F480621A605A6822F459
:10BD7000E0625A601B69621C42622370438D013B82
:10BD80009BB22022438580F83D20016390F83E302D
:10BD900080F83E10402BC9D1FFF74CFC34E590F8F9
:10BDA0003E20402A7FF497AE026D002A40F0828048
:10BDB000C26C012A826C00F09D80C2F307221A61D6
:10BDC000036D013303651FE5019659690191996976
:10BDD0000191019924E502965969029199690291AC
:10BDE0000299196841F480711960016D0131016592
:10BDF00016E522F480621A601A6842F480721A60B2
:10BE000071E717F5803F41D0042F2FD0082F2DD098
:10BE1000BCF1120F2AD0C16A0229196814BF21F49B
:10BE2000806141F480611960002106915969069191
:10BE3000996906910699CCE6C16A022919684AD027
:10BE400021F480611960196841F400611960596832
:10BE50000E0503D5596841F48051596000210891BD
:10BE600059690891996908910899B2E619680026FC
:10BE700021F48061196007965969079199690791C2
:10BE80000799196841F400711960A2E6196821F454
:10BE900080611960596811F4006120D0196800268A
:10BEA00021F480611960049659690491996904919B
:10BEB00004998EE6026D012A22D0026D022A7FF4D7
:10BEC000A3AC90F83D20222A21D090F83D20212AD1
:10BED0007FF49AACFFE541F480611960B7E7059102
:10BEE00059690591996905910599196841F400719D
:10BEF00019606EE6D2B21A61036D0233036583E402
:10BF0000826CD2B21A61036D013303657CE41A6856
:10BF100042F480721A6077E470B5036855495C6931
:10BF20005A680C4282B01ED0D6051CD5016C6FF445
:10BF3000807541F0010114F4813F01645D6148D0D6
:10BF4000016C6FF4007541F0020114F4823F01644A
:10BF50005D611DD114F4843F01D0D20531D4036C4E
:10BF600063B902B070BD14F4813F0CD0D505E7D49D
:10BF700014F4823FEED0036C002BF2D002B0BDE887
:10BF80007040FFF75BBB14F4823FE3D0D105E6D5E8
:10BF900090F83E50428D90F83D10066B202D92B2E5
:10BFA000C9B21AD0026C42F00402026490F83E203A
:10BFB000102A3ED06FF480625A6114F4843FCED0D0
:10BFC0000368026C6FF4006142F008020264596178
:10BFD000C5E714F4823FDBD1BCE7002AE2D101F0CF
:10BFE000F702212A03D02829DCD1212EDAD190F8BA
:10BFF0003D20C16A0429D2B220D008291ED0212AAE
:10C00000D8D11D49C16220250021026380F83D502E
:10C0100080F83E105A6801906FF4806122F4E0626B
:10C020005A6059611A680A401A60FFF7FDFA0198D0
:10C03000C3E71A6842F400721A60BBE7282ADED10F
:10C040000D4AC2625A6801906FF4806122F4E06286
:10C050005A6059611A68002122F4806220251A6012
:10C06000016380F83D5080F83E1016F0B5FA019853
:10C07000A3E700BF000101000000FFFF806B026822
:10C0800038B51168456B846B002321F48061116021
:10C0900043852B65236590F83D1060294FF0200102
:10C0A00080F83D1080F83E3006D0136823F001037D
:10C0B000136016F0BBFA38BD0364136823F0010364
:10C0C0001360FFF7B9FA38BD38B50D4B0D4A0E4D68
:10C0D0001A60410000224FF480441846C3E905224B
:10C0E000C3E90722D9605D601C619A60FFF786F999
:10C0F00000B938BDBDE8384004484F21F8F78EBA82
:10C10000C0D4002000540040A08601009490020892
:10C11000374B02689A4200D0704770B586B004234E
:10C120004FF4407104461220032201250191029030
:10C130000DEB03012F480593CDE90352FEF776FF7F
:10C1400000232D4A0093116C2C4E2D48B36041F40E
:10C1500000111164126CF36002F400120092C6E93F
:10C160000533C6E908334FF000714FF480624FF495
:10C17000807330603046009D71603261F361F9F781
:10C180004DF858BB1F4D2048A6634FF00073402167
:10C190004FF4806228606B6028460023C5E90332B3
:10C1A000C5E90533C5E90733B463A9606B62F9F7E4
:10C1B00035F8C0B96563002205211F20AC63F5F78F
:10C1C000E3FE1F20F5F718FF002205212020F5F7D8
:10C1D000DBFE2020F5F710FF06B070BD0B487A217A
:10C1E000F8F71CFACEE709488C21F8F717FAE1E7CF
:10C1F00000540040000402400038024014D50020E2
:10C200001060024060D40020A060024094900208B8
:10C21000DFF838D0002103E00D4B5B584350043168
:10C220000C480D4B42189A42F6D30C4A02E0002308
:10C2300042F8043B0A4B9A42F9D3FCF77FFEF8F729
:10C24000EFF817F063FDF8F783F97047000002205C
:10C25000FC7F0308000000200406002008060020E0
:10C2600090D50020FEE7000010B50446FDF71EFA49
:10C27000094A106860B1094B196803198B4296BFCF
:10C2800004464FF0FF341360FDF7D6FA204610BD88
:10C29000034B18681060EEE718080020FC0100202E
:10C2A000F801002070B5044684B00D460022218AB2
:10C2B000C068FFF793F8012000F032FB6FEA4541B8
:10C2C0006FEA51414FF47A73ADF80C1000264BF62B
:10C2D000EF65012203A92068ADF80A60ADF80E50A1
:10C2E000F7F7C4FC218AE0680122FFF777F8012004
:10C2F00000F016FB218AE0683246FFF76FF8012054
:10C3000000F00EFB4FF47A730DF10E020DF10A01ED
:10C31000206800930123F7F779FD012000F000FB6E
:10C32000218AE0680122FFF759F8012000F0F8FAAD
:10C33000BDF80E00A84203D0C0F30A0004B070BDDF
:10C34000034B044A044840F2871117F0A9FC00BFD0
:10C35000A8900208D8900208BC90020810B5018984
:10C36000044601224068FFF739F80A20FCF76AFA10
:10C3700000212046FFF796FF4305F9D4BDE81040A1
:10C380000120FCF75FBA00BF10B500210446FFF79B
:10C3900089FF420503D5C0F30A0010B110BD00208B
:10C3A00010BD20464FF40061FFF77CFF0306F6D571
:10C3B0004FF4806010BD00BF70B5044682B00E46D9
:10C3C0001546018AC0680022FFF708F8012000F036
:10C3D000A7FAC5F30A030DF1060143EA0605012297
:10C3E0004FF47A732068ADF80650F7F73FFC012050
:10C3F00000F096FA218AE0680122FEF7EFFF0120A3
:10C4000000F08EFA02B070BD38B591F8223003B951
:10C4100038BD0C460B7C497CA27C0B43E17C13436A
:10C42000A28A0B431A434FF480510546FFF7C4FF1D
:10C43000E07DA37D217E627E03430B431A432846A1
:10C440004FF4C051FFF7B8FF002384F8223038BD05
:10C4500091F8233003B9704770B50C4600210546AA
:10C46000FFF720FF0346C0F38022C3F30021C0F38F
:10C4700040202270C3F3C0126070A170C3F380101B
:10C48000C3F34011E270C3F3001263832071617142
:10C49000C3F3C000C3F38001A271C3F3400203F0F1
:10C4A0000103E07121726272A3724FF400612846A9
:10C4B000FFF7F8FEC0F3C01200F00F03A083227351
:10C4C000E3814FF480512846FFF7ECFE034600F06D
:10C4D000030200F0040600F00801227403F03002A9
:10C4E00003F4F863E08366742846A174E274A382BF
:10C4F0004FF4C051FFF7D6FE00F0030600F00C0524
:10C5000000F0300100F040020023A675E5752176A9
:10C510006276208484F8233070BD00BF70B5002699
:10C5200005464E8401200C46FCF78CF9314628461E
:10C53000FFF7B8FEC0F38023C0F34021C0F3002210
:10C540002370C0F3C0136170A270C0F38011C0F3F8
:10C550004012E370C0F30013C0F3C0062171627192
:10C56000C0F38001C0F34002A37100F001036272C6
:10C57000E6712172A3724FF400612846FFF792FE24
:10C58000C0F3C01300F00F002373E0814FF480511B
:10C590002846FFF787FE034600F0030200F008017B
:10C5A00000F00406227403F0300203F4F863A1746F
:10C5B000E274A3824FF4C05128466674FFF772FEFE
:10C5C00000F0030100F00C0200F0300300F0400026
:10C5D000A175E2752376607670BD00BFF5EEC00AE6
:10C5E000F1EE10FAB5EEC00A7CDBF1EE10FA50DB8A
:10C5F000DFED877A60EEA77AF4EEC07AF1EE10FAFA
:10C6000040F39B80DFED836AB7EE007AA0EEE67A16
:10C61000F6EE006A27EE267A70EE276A37EE400AB9
:10C6200081ED007A70EE277A37EEA67AC0ED007AB7
:10C6300082ED007A90ED000AB5EEC00AF1EE10FA34
:10C64000C0F2E280F7EE007AB4EEE70AF1EE10FAFB
:10C6500000F2DA8091ED007AB5EEC07AF1EE10FAD0
:10C66000C0F2D280B4EEE77AF1EE10FA00F2CC809C
:10C6700092ED007AB5EEC07AF1EE10FAC0F2C48005
:10C68000B4EE677AF1EE10FA8CBF4FF0FF30002065
:10C690007047DFED617A60EEA77AF4EEC07AF1EED2
:10C6A00010FADFED5B7A40F38680A0EEA70A9FEDDB
:10C6B000597AF0EE407AE0EEC77AB7EE006A77EE8C
:10C6C000867AF6EE006A67EEA67AF0EE676AE0EE2A
:10C6D000876AC1ED007A36EEC00AC2ED006A80EDCD
:10C6E000000AA9E7F1EE10FA68DBDFED4B7A60EEA5
:10C6F000A77AF4EEC07AF1EE10FA3DDDDFED447A70
:10C7000060EEA77AF0EE006AB7EE007AA7EEA67A9E
:10C71000F6EE006A27EE267A70EE276A30EE670A98
:10C7200077EE667A82ED007A30EE270AC0ED007A65
:10C7300081ED000A90ED000A7EE7B7EE007A37EE51
:10C74000407ADFED346A37EE277AB6EE006AA0EE63
:10C75000E67A30EE670A67EE067A37EE800AC0EDB9
:10C76000007AF0EE407AE0EEA67A81ED000AC2EDA2
:10C77000007A90ED000A5FE7DFED256A9FED277AEA
:10C78000F7EE007AA0EEA60AE0EEC77AF6EE006AAF
:10C7900077EEC07A67EEA67A37EE800AC0ED007AAF
:10C7A000F0EE407AE0EE877A82ED000AC1ED007A81
:10C7B00090ED000A40E760EEA77A23E7DFED147AF8
:10C7C00060EEA77AF4EEC07AF1EE10FA9ADDB7EED9
:10C7D000007A30EE077ADFED116AA0EEE67AB6EE67
:10C7E000006A37EE677A37EEC00A67EE067AB0EE77
:10C7F000677AA0EEA67AC2ED007A37EE000A81EDE4
:10C80000007A80ED000A17E74FF0FF30704700BF55
:10C810003ACD133F3ACD933F3ACD13BF3ACD93BFB4
:10C82000B0EEC06AF0EEE06ADFED207A9FED204ABC
:10C83000DFED204A9FED205AB4EEE66AF1EE10FAE1
:10C840004CBF76EEA77A76EE277AD4BFF0EE465A42
:10C85000F0EE665AB0EE407A85EEA70AF7EE007A5F
:10C8600060EE005AB4EEE66AE5EE844AF1EE10FAA4
:10C87000A4EEA55AF5EEC00AE5EE257A27EE800A69
:10C88000C4BFDFED0E7A37EEC00AF1EE10FA48BFF2
:10C89000DFED0B7AB5EEC07A48BF37EEC00AF1EE95
:10C8A00010FA48BFB1EE400A704700BF0000800098
:10C8B00016733EBD4423233E2CBEA7BEDB0FC93FEB
:10C8C000DB0F4940B0EE407A9FED070A51B100EB13
:10C8D0008101F0EC017AE0EE077A8842B0EE670A57
:10C8E000F7D17047704700BF0000000090FBF1F3E4
:10C8F00003FB11000028B8BF4018704770B5074E01
:10C90000FAF79AF9756A0446FAF796F98442F7D16C
:10C910004FF47A7000FB045070BD00BF002000404F
:10C9200038B50546FFF7EAFF044600E000BFFFF711
:10C93000E5FF031BAB42F9D338BD00BFDFED217A21
:10C94000B5EEC00A60EE277AF1EE10FABDEEE77A96
:10C9500004D517EE103A013B07EE103AB8EEC77A4D
:10C96000DFED196A77EEC77A67EEA67ABCEEE77A52
:10C9700017EE103A9BB2B3F5007F1AD207EE103AC9
:10C98000B8EE477A591C37EEC70A104AB7EE006A6C
:10C9900002EB8101D1ED006A37EE067A02EB8303E8
:10C9A00020EE260A77EE677AD3ED006AA7EEA60A94
:10C9B000704777EEE67A9FED067AB0EE670A0121BE
:10C9C0000023E2E783F9223E00000044A06603084A
:10C9D000000000009FED237ADFED236AF5EE007A78
:10C9E000E0EE077AB4EEE60AF1EE10FABDEEE77A71
:10C9F00004D517EE103A013B07EE103AB8EEC77AAD
:10CA0000DFED1A6A77EEC77A67EEA67ABCEEE77AB0
:10CA100017EE103A9BB2B3F5007F1AD207EE103A28
:10CA2000B8EE477A591C37EEC70A114AB7EE006ACA
:10CA300002EB8101D1ED006A37EE067A02EB830347
:10CA400020EE260A77EE677AD3ED006AA7EEA60AF3
:10CA5000704777EEE67A9FED077AB0EE670A01211C
:10CA60000023E2E783F9223EDB0FC9BF0000004448
:10CA7000A06603080000000010B4134C134B144AC6
:10CA8000DFED147A0138A14200EB400003EB800097
:10CA900028BF214690ED300A90ED317A5DF8044BC5
:10CAA000D0F8BC00914238BF114637EE407AA1F56C
:10CAB000A431203927EE277A07EE901AF8EEE77AAC
:10CAC000A7EE870A08F0DCBB409002001C7B002028
:10CAD0002048010090BA473702881143018070470F
:10CAE000EFF3108372B6044A127812B1012280F873
:10CAF000662083F3108870477808002030B403461E
:10CB0000EFF3108472B6026890F86600126811683C
:10CB10004A6C002522F40042401B83F8665018BF7F
:10CB200001204A6484F3108830BC704770B4EFF37E
:10CB3000108272B6234B1B78EBB9046880F866301C
:10CB400023680D881B684C8889885D639C63D96362
:10CB5000EFF3108472B603681B6819684B6C0025EC
:10CB600023F4004380F866504B6484F3108882F30A
:10CB7000108870BC7047036890F866401B680E8888
:10CB80001B684D8889885E63012C9D63D9630CD036
:10CB9000022C11D1596C032441F4004180F8664005
:10CBA000596482F3108870BC7047022380F86630A5
:10CBB00082F3108870BC7047032CC9D182F31088AF
:10CBC00070BC70477808002070B4EFF3108472B620
:10CBD000164B17491A68174E0868002341F20105E1
:10CBE000D36333701564426AEFF3108572B6106830
:10CBF00082F8663002681068426C22F40042426497
:10CC000085F310884A68526AEFF3108172B6106893
:10CC100082F8663003681A68536C23F40043536447
:10CC200081F3108884F3108870BC704758C70020C7
:10CC30008808002078080020F8B5114C054604F15A
:10CC40000807002623685B6AEFF3108172B61A6842
:10CC500083F8666013681A68536C23F400435364C6
:10CC600081F3108854F8043B586A29466430FFF772
:10CC700033FFBC42E6D1BDE8F840FFF7A5BF00BFD7
:10CC80008808002038B50B1A272B05460C4611D909
:10CC9000EFF3108272B60A4B1B7843B1094B1B6845
:10CCA000002041F20101D8631964DD631C6482F342
:10CCB000108838BD4FF48070FFF7BEFFE8E700BF73
:10CCC0007808002058C70020036840F2D66210B5EB
:10CCD00000215A6304469A63DA63FDF7DFFA2046BF
:10CCE0000021F6F765FE20460421FDF7D7FA20461D
:10CCF0000421F6F75DFE20460821FDF7CFFA204615
:10CD00000821F6F755FE2368012220461A64BDE883
:10CD100010400C21FDF7C4BA096800682DE9F04104
:10CD2000456C4C6CD0F804C08F68466CDDF818E098
:10CD300026F4004646644E6C26F400464E640668AF
:10CD400026F0010606600E6826F001060E604668B1
:10CD500026F070064660466846F0100646608E680B
:10CD600026F070068E608E6832438A608A6822F0F0
:10CD700007028A608A6842F006028A6006680A68CA
:10CD8000D0F8008028F06008C0F80080D1F800805A
:10CD900028F06008C1F80080D0F8008028F0100862
:10CDA000C0F80080D1F8008028F01008C1F8008099
:10CDB000D0F8008006F0600646EA080606600E68B5
:10CDC00002F06002324300260A6005F40045436227
:10CDD00004F400444E62BEF1000F06D0DEF80020DD
:10CDE0005362136843F00103136002681FFA8CF367
:10CDF000BFB242F00102026043608F60436C1D438A
:10CE000045644B6C1C434C64BDE8F0812DE9F04354
:10CE1000DFF86491DFF86481D9F80000D8F80010D9
:10CE200083684D4F4D4E3A684D4C4E4D43F00103D3
:10CE300083608B6843F001038B60936843F00103C8
:10CE400083B093600220FBF7FDFCD9F800C0D8F84E
:10CE50000000DCF804103A68434B41F08001CCF844
:10CE60000410416841F080014160516841F0800147
:10CE70005160416841F020014160516841F020015A
:10CE80005160DA6842F00102DA60DA6842F00202C8
:10CE9000DA609A6842F080029A603046FFF714FF29
:10CEA0002046FFF711FF314B00932146304640F2F8
:10CEB00056630022FFF730FF32682368516C2E68FA
:10CEC00021F400415164596C21F400415964D16846
:10CED00041F00101D160DA68002442F0010241F220
:10CEE0000107DA602846F46308213764FDF7D6F9B4
:10CEF00028460C21FDF7D2F91D4A13685B6AEFF34F
:10CF0000108072B6196883F866400B6819684B6C1C
:10CF100023F400434B6480F3108853685B6AEFF39B
:10CF2000108172B61A6883F8664013681A68536CE9
:10CF300023F40043536481F31088EFF3108272B638
:10CF40000C492B680120DC6308701F6482F3108891
:10CF500003B0BDE8F08300BF48CF00201CC700200D
:10CF6000F0C5002058C70020002004E0E0C60020E3
:10CF7000880800207808002000CF0020B8CE0020CC
:10CF800070B51E481E4B03604FF4803300221D4CC9
:10CF9000436084B001231021C0E903238462C1618E
:10CFA00082600262C262836103634361FDF71CFE1B
:10CFB000F0B90123114D144E0293002401E0102C0E
:10CFC0000FD000946946013428460194FDF786FF8E
:10CFD0000028F4D04FF4B9713046F7F71FFB102C3E
:10CFE000EFD10A4905482246FDF7AAFE04B070BDFC
:10CFF000054840F26911F7F711FBDAE700CF00208E
:10D00000002001400100000FE890020858080020AD
:10D01000284B984210D0284B984205D0274B984275
:10D020001ED04FF6FF70704701292FD002294FF60E
:10D03000FF7008BF09207047012921D0022921D0A3
:10D0400004292BD008292DD010292FD020291FD01A
:10D0500040292DD080294FF6FF7008BF0720704768
:10D06000012911D0022915D0042915D0082917D07B
:10D07000102919D020294FF6FF7008BF0F207047E4
:10D0800000207047012070470A2070470820704731
:10D09000052070470B2070470C2070470220704716
:10D0A0000D207047032070470E2070470420704702
:10D0B00006207047000002400004024000080240C1
:10D0C00008B5FFF7A5FF0F280BD8074BDFED077A50
:10D0D00033F8103000EE103AB8EE400A20EE270A7E
:10D0E00008BD9FED030A08BD580800203333533AAA
:10D0F0000000C07F2DE9F843DFF8BC90DFF8BC806A
:10D10000274F284E2DED048B9FED278A9FED279A00
:10D11000DFED278A274C012504E00135092D04F1B4
:10D120000C042CD0206808F097F80028F5D0ABB29A
:10D130005A1F92B2023B032A9BB224D859F822000C
:10D1400038F81310FFF764FF0F2825D837F8103090
:10D1500007EE103AB8EE477A27EE287A94ED010AE6
:10D16000D4ED027A206877EEC07A013567EE887ACE
:10D170000C34A7EE870A08F083F8092DD2D10A20D3
:10D18000FBF760FBC6E7062B304688BF0121D7D9E5
:10D19000FFF73EFF0F28D9D9B0EE497ADEE700BF8E
:10D1A0005808002000000240CA269B3E0000C07FB5
:10D1B0003333533A387C002004910208149102085A
:10D1C0000F280BD8074BDFED087A33F8103000EE4C
:10D1D000103AB8EE400A20EE270A70479FED030A86
:10D1E000704700BF580800203333533A0000C07F17
:10D1F00008B50121FBF798FD07EE900A9FED047A30
:10D20000044BF8EE677A67EE877AC3ED007A08BDC3
:10D210003333113C0002002038B503681C6814F059
:10D2200010041AD1124B984218D0124B984218D1C0
:10D23000114B5B6801241869104D03F0DDF8104AAA
:10D24000104811492D690069096963001C4402EB0B
:10D25000440322F814505880998038BD064B1B684F
:10D26000E9E7BDE838404FF40070FFF7E5BC00BFC8
:10D270001CC70020F0C500208808002000000240E4
:10D280001C0800200004024000080240584B1A68A5
:10D290005B68526A5B6A92F8661010B503292DED3F
:10D2A000048B08BFD2ED238A93F8662018BFDFED08
:10D2B000518A514C032A08BFD3ED237AD4ED279A23
:10D2C0004E4B08BF78EEA78AD4ED267A93ED009AEC
:10D2D00094F8A83078EEA77A69EEE77A87EE898A23
:10D2E0006BB1F5EEC09AF1EE10FA08DDD4ED2B7AB1
:10D2F00094ED2C0AF4EEC07AF1EE10FA6BD4B4EE91
:10D30000488AF1EE10FA68BF4FF4005052D6DFEDB4
:10D310003C7AB4EEE78AF1EE10FA02DB394B0122D7
:10D320001A70B5EE408AF1EE10FA2ED59FED318AD3
:10D33000354B94ED096AD3ED007A94ED2D7A78EEB1
:10D34000E76AB4EEE87AE6EE267AF1EE10FAC3ED7B
:10D35000007A2DD4D4ED2E7AF4EEE87AF1EE10FABC
:10D360002EDCF7EE007A37EEC88AF0EE487AFEEE51
:10D37000CA7ABDEC048B17EE901AA1F12800BDE823
:10D38000104020EAE070FFF77DBCDFED1D7AB4EEBF
:10D39000E78AF1EE10FA1BDCB5EE408AF1EE10FAE6
:10D3A000C6D029EE089AC9EE297A78EEA78ABFE797
:10D3B0004FF40040BDEC048BBDE81040FFF73CBCCF
:10D3C000BDEC048B4FF48040BDE81040FFF734BC47
:10D3D000B0EE678AE5E730EE670A79EE677ADFED4F
:10D3E000050A87EE800A16F001FB38EE008A86E710
:10D3F00088080020000000001C7B002000020020A4
:10D400003333733F790800207C0800202DE9F04F6A
:10D41000DFF81892484587B004460E4602D0804B8C
:10D42000984270D1DFF808B2002E67D1DBE900A77F
:10D430004FF00108786A03681B681B681D6815F0C7
:10D4400010050CBF0121022101F01CFF4C4560D0EA
:10D45000002E70D001212046FBF766FC0146786A59
:10D4600001F01EFF002D6FD14C4500F0AA80D7F8C7
:10D4700010E0D7F824B0DEF80830DBED1D7AD3F8E1
:10D480001490D3F80CA01E8B1A8AD969188C654C9D
:10D49000DFF8A0C1CDF810904FEA4803984430EE71
:10D4A000670A04EB480461452B46CDF814A0ADF89B
:10D4B0000660ADF80820DFF880918BED1B0A04F1BF
:10D4C000040A04F102080DF1060204AD0DF10A068A
:10D4D00012D0494514BF5146414609885B000842B5
:10D4E00018BF43F001039642DBB23DD055F8041B50
:10D4F00032F8020B6145ECD12146EEE7DBE9007A18
:10D500004FF0000896E7042007B0BDE8F04FFFF7A2
:10D5100093BBDBF80430BB422ED0DBF80030BB42BB
:10D5200049D0002D48D1B8F1000F91D1386902F0EF
:10D53000FDFF002E8ED12046FDF786FC0146786A5D
:10D5400001F0AEFE002D8FD04C457B6A9FED367A00
:10D5500041D0D3ED1D7A30EE670AE0EE077AC3EDD5
:10D560001D7A07B0BDE8F08F38468EF85C3007B002
:10D57000BDE8F04F00F080BC002D37D0B8F1000FAF
:10D580003BD1DAF8240090F84220002A39D1EFF399
:10D59000108C72B6036890F866101B6880F86620DD
:10D5A0001A68536C23F4004353648CF3108881BBD6
:10D5B000FFF76CFE4CE7EDB1B8F1000F3FF448AF58
:10D5C000B4E77B6AD3ED1C7A30EE670A83ED1A0A62
:10D5D00007B0BDE8F08FD3ED1C7A30EE670AE0EEBD
:10D5E000077AC3ED1C7A07B0BDE8F08FDBF8003096
:10D5F000BB4298D1B8F1000FC3D1386902F096FF51
:10D60000BFE7002380F8423000F13C01FFF78EFABB
:10D61000CEE7DAF8240010216430FFF75DFAC7E79F
:10D6200048CF00201C0800200BD7233AB8CE00209A
:10D630008808002000000240000402402DE9F04369
:10D6400002238BB0CDE9063300220A2401200F21EA
:10D65000DFF88C80204E214FDFF8889001940993E9
:10D6600008920392029004914FF0FF342546013452
:10D6700004EB440308EB8303D3F8BC0007F0ECFD94
:10D68000ABB2D8B10122062B304611461BD839F86F
:10D6900013100591FDF7F2FD05A93046FDF7C6FC14
:10D6A000022D254694BFA500002501A92A4638462B
:10D6B000FDF728F929463846FCF7F4FD032CD5D1AF
:10D6C0000BB0BDE8F0830592FDF7D8FD05A9304603
:10D6D0000025FDF7ABFCE8E70000024068C600202B
:10D6E0001C7B0020149102082DE9F041441E032CFC
:10D6F00082B019D8831E9BB2062B05460E4616D95A
:10D7000001211948194FFDF763FE3B5DB0F1000898
:10D7100018BF4FF0010873B9154B164A42F8246040
:10D72000012103F80480395502B0BDE8F081124AA6
:10D7300032F81310E5E70E4B1A5D002AEDD00D4AC2
:10D740000028EBD152F82410DFF830C0711AA1F58F
:10D75000244010386045E1D82846CDE90032FFF773
:10D760008BF9DDE90032D9E70000024050080020C3
:10D770002808002030080020149102084090020080
:10D7800030B5064D0FCD87B001AC0FC42B682360B8
:10D79000002101A8FBF73EF807B030BD988E0208C3
:10D7A000084A13681969836B01F16A00834206D045
:10D7B0005268106900F16A02934201D0704708462E
:10D7C00002F0E0BE8808002030B587B042680392BE
:10D7D000002301210222CDE90412CDE901330546DF
:10D7E000FAF716FC0A4BF322DA60694601A8F9F74A
:10D7F000F9FA38B9EB682B600446FAF71DFC2046AD
:10D8000007B030BDFAF718FCFAF720FC07B030BDBE
:10D81000003C02402DE9F0410746C06888424FD8DD
:10D82000B8688C1884424BD2180140EA83004C003F
:10D83000184304F0060540EA8316FF2401F00303B1
:10D8400003EB0208AC4021F00305FAF7E1FB1E4BA5
:10D85000E443F322F6B2E4B2DA600EE0396946EA54
:10D86000040201EB9501D2B200230020FAF71EFC5E
:10D87000A8F1040804350446E0B9B8F1030FEDD867
:10D88000B8F1000F11D0C8F104035B00FF221A4168
:10D8900064EA0202396952B2324301EB9501D2B215
:10D8A00000230020FAF702FC20B9FAF7C5FB00209C
:10D8B000BDE8F081FAF7C0FBBDE8F041FAF7C6BB5E
:10D8C0004FF0FF30F4E700BF003C0240F0B4150118
:10D8D00045EA8206C56816430746C81C46EA821414
:10D8E00020F003002E1DB042E4B2A0EB010136D3BC
:10D8F000421E3F699208BA5CD2B281B14FEA410C34
:10D90000FF2141FA0CF1C943C9B222EA01022140C8
:10D910000A4304E0B44520D37A5C6046D2B2411F8A
:10D92000A2424FEA9101A0F1040CF3D004F00304E9
:10D93000B4EB921F4FEA92110CD1A84202D809E031
:10D94000A84207D09200C2F38111A14200F1FF303A
:10D95000D2B2F5D0F0BC197070476046E6E72246B7
:10D96000E4E700BF70B5194C82B0A1680DF1050362
:10D9700003222046FFF7AAFF0DF1060320600322D1
:10D98000216A04F11800FFF7A1FF114B9DF8062052
:10D99000A06100251D7092B1216820460DF107039A
:10D9A0000022FFF793FF6A0015440A4E54F8352011
:10D9B0000949121A00203260086002B070BD0125CA
:10D9C00001461D7004F11800E8E700BF04020020C2
:10D9D00074D500207CD5002078D5002010B5094CE6
:10D9E000094B616AE268A1612260204600221A7038
:10D9F000FFF7EAFE034604F118001C46FFF7E4FEB9
:10DA0000204310BD0402002074D50020014B18688B
:10DA1000C00070477CD50020064B074A1B78C3F135
:10DA2000010303EB430302EBC303D3E90203C01A70
:10DA3000C000704774D500200402002070B50E4C61
:10DA400025688418B4EBC50F13D80C4C2478034612
:10DA500004EB440408460A4901EBC40651F834407B
:10DA60007169641B03EBC403194416F083F90020A9
:10DA700070BD4FF0FF3070BD7CD5002074D5002004
:10DA8000040200202DE9F041154B164F1B78C3F11D
:10DA9000010303EB430307EBC306D6E90252073049
:10DAA000AA1AB2EBD00F18D3DC004FEAD0083959CC
:10DAB0006D1A45450AD3304601234246FFF7AAFEB8
:10DAC00010B9094BC3F80080BDE8F0813046FFF77C
:10DAD0007BFE0028F8D13959EDE74FF0FF30F3E72E
:10DAE00074D500200402002078D500202DE9F843E9
:10DAF000404B15461A684319B3EBC20F76D83E4B1C
:10DB000004461F788846FAF783FA3C4BF322DA6022
:10DB1000A207C7F1010725D0FDB1394A07EB470637
:10DB2000C14602EBC60602E0A3071BD0ADB13368C5
:10DB3000716919F8012B01EBC30121440023002076
:10DB4000FAF7B4FA0134013DC8460028ECD0FAF7E0
:10DB500073FABDE8F843FAF779BAFAF76DFA0020DC
:10DB6000BDE8F883032D1ED9254A07EB4706C146B9
:10DB700002EBC60601E0032D15D93368716959F827
:10DB8000042B01EBC301214400230220FAF78EFA93
:10DB9000043DC84604340028EDD0FAF74DFABDE83C
:10DBA000F843FAF753BA002DD7D0154A07EB4707C9
:10DBB000C1464544A4EB080402EBC70701E0A945B0
:10DBC000CBD03A687B6904EB090103EBC20319442B
:10DBD00019F8012B00230020FAF768FA0028EED08C
:10DBE000FAF72AFABDE8F843FAF730BA4FF0FF30F7
:10DBF000B6E700BF78D5002074D50020003C024075
:10DC0000040200202DE9F0411D4E1E4D34781E4FB8
:10DC1000C4F1010000EB40004FEAC0083A6855F833
:10DC2000081005EBC0000023FFF7F4FD08BB3968BE
:10DC300055F8083038605A1804EB4403134845F887
:10DC40000820DF0005EBC3033278D3F808C0016079
:10DC5000E95904EB4404C2F10103614505EBC4003A
:10DC6000337008D201231A46FFF7D4FDEB59013374
:10DC7000EB51BDE8F081BDE8F041FFF7A5BD00BF65
:10DC800074D500200402002078D500207CD5002027
:10DC900070B4D0E90545466A026900230021A6F860
:10DCA00064302B7523729382516470BC0365704796
:10DCB000036E8269196990F8543092ED107A30B48D
:10DCC000B0F86440C06801250C4214BF29464FF0EB
:10DCD000FF3103FB01F307EE903AD0ED026A82F8C0
:10DCE0005450F8EEE77A30BCA7EEA67A82ED107AAF
:10DCF000704700BFC368D3ED037AF5EE407AF1EECA
:10DD000010FA0AD49FED0C7AF4EEC77AF1EE10FA0D
:10DD100007DD0A4BC0F8843070470023C0F8843018
:10DD200070479FED077A67EE877AFCEEE77A17EE89
:10DD3000903AC0F884307047300E034900B6F7FFC0
:10DD40000000FA45026811430160704710B5D0F831
:10DD5000844024B1013CC0F88440012010BD4FF440
:10DD600000615030FFF7EEFF204610BD0268114001
:10DD700001607047C0437047F0B4104EDFF850C0E8
:10DD80000F4F04460FCE25460FC596E807000D4BF2
:10DD90000D4EC4F804C085E807002660A3600B4E52
:10DDA000DFF830C0C4F80CC04FF480720123204665
:10DDB000276166612283A376F0BC7047AC8E0208AF
:10DDC00000002042DB0F49400000204163141D4445
:10DDD000CDCCCC3E0000A041F0B40F4E0F4FDFF889
:10DDE00050C004460FCE25460FC596E807000C4BE1
:10DDF0000C4E67600C4F2760A6600C4FE360012655
:10DE0000002385E807002046C4F810C06761268318
:10DE1000A376F0BC704700BFAC8E0208CDCCCC3EE0
:10DE200000004843DB0F4940000020410000C84289
:10DE30000000C843704700BF10B58268836C86B08D
:10DE4000044690880A4A01920022CDE903229B08E9
:10DE5000084AADF80C00214601A805930292FAF792
:10DE6000D9FC0123606484F84C3006B010BD00BFBB
:10DE70008C640308F9EE000890F84C3003B9704741
:10DE8000406C0121FAF7E6BC00B585B001A802227A
:10DE90000121FAF709FD0198A0F10800B0FA80F01D
:10DEA000400905B05DF804FB028843888B824A82F2
:10DEB000704700BF0368CB66704700BFC1684B8ADC
:10DEC0005A1F92B2032A10B41DD81A4C023B54F8C0
:10DED000222082659BB2184A32F813208B8AA0F860
:10DEE0005C205A1F92B2032A16D81249023B51F8FD
:10DEF000222002669BB2104A5DF8044B32F81330C0
:10DF0000A0F864307047023B9BB20C4A8265062B36
:10DF100088BF0122E2D8DEE7023B9BB2074A0266D5
:10DF2000062B88BF0123E6D95DF8044BA0F86430C6
:10DF3000704700BF48910208589102080000024053
:10DF40002DE9F84FC360DDE90C96DDE90E58DDE9F7
:10DF500010ECDDE90ABA4FF4006382608364334A4F
:10DF6000129B41600027026000F16701022280F8E5
:10DF70006620C0E905A9C0E9098EC0F810B0C661E5
:10DF80004663C663056285630564C0F82CC00363FD
:10DF900080F84C70076580F85470C0F86770A0F87E
:10DFA0007C70C0F86B70CBF81000A0F86F70CAF8E6
:10DFB00000004167C9F8100087677062C0F8807080
:10DFC0006862C0F88470C8F82400CEF80000CCF86D
:10DFD000040058600446FFF771FFC268D2ED037A6F
:10DFE000F5EE407AF1EE10FA0CD49FED117AF4EED2
:10DFF000C77AF1EE10FA0BDD0E4BC4F884302046E0
:10E00000BDE8F88F3B46C4F884302046BDE8F88F61
:10E010009FED097A67EE877A2046FCEEE77A17EEE5
:10E02000903AC4F88430BDE8F88F00BF84910208AC
:10E03000300E034900B6F7FF0000FA4510B504465C
:10E0400088B0B1B1B0F86430039303A90023006E27
:10E05000CDE90433FCF7EAFF00940A4BB4F85C10F6
:10E06000A06D0222FBF71AF8012384F8543008B09F
:10E0700010BD80F85410B0F85C10806DFBF786F886
:10E0800008B010BDB1DC0008364B1B7870B50446F3
:10E09000002B35D0636F1B78012B03D0636A93F894
:10E0A00066303BB3304E314DD6ED007A95ED287A8F
:10E0B000B4EE677AF1EE10FA40D895ED297AB4EE15
:10E0C000677AF1EE10FA33DBE06B01F089FD206C2A
:10E0D00001F086FD606A01F057F8E06A03689B7AF8
:10E0E0009BB9206B03689B7A83BB206DB0FA80F0EC
:10E0F000400970BD202104F15000FFF723FED1E755
:10E1000010215030FFF71EFEC4E702F02BFD00285F
:10E11000E7D0636F1B780B2BE3D04FF4805104F1F1
:10E120005000FFF70FFE206DB0FA80F0400970BD7F
:10E13000042104F15000FFF705FEC5E7022104F1B8
:10E140005000FFF7FFFDD6ED007AB6E702F00AFDBA
:10E150000028CAD0636F1B780B2BC6D04FF4005138
:10E16000DDE700BF78080020000200201C7B0020B3
:10E1700038B50446C06B01F01FFD206C01F01CFD9A
:10E18000206902F0ABFA606903F072F9E06A02F00C
:10E1900093FC206B02F090FC256D054BB5FA85F5DC
:10E1A00018686D09214614F095F9284638BD00BF5E
:10E1B000187B0020C3681B7C0BB1FFF7C7BD012093
:10E1C000704700BFF0B52DED088B9FEDA88ADFEDFD
:10E1D000A98A9FEDA9AADFEDA69A012385B004467E
:10E1E000B0EE489A0D4680F87C3043E02046FFF7B9
:10E1F000ADFD0FB106B118B9636F1B78012B5DD16E
:10E20000D5ED027ADFED9C0AB0EE680AA8EE270A87
:10E2100015F04CFCD5ED017A606AD5ED006A036A11
:10E2200089EEA77AB5EEC00AD3ED067AF1EE10FAC0
:10E2300048BF30EE0A0A67EEA67A70EE680AB0EEC2
:10E24000491A27EE880A38EE078A01F065FBA36FAA
:10E250000133A3670222012100B301A8FAF724FBCE
:10E26000019B082B20D1F7EE007AB4EEE78AF1EE9D
:10E2700010FA23D594F8666016BB2046FFF704FF1A
:10E2800007462046FFF774FFE3681B7C0646002B19
:10E29000ACD1002FB0D00028B2D1ADE701A8FAF779
:10E2A00003FB019B082B09D0606AFEF727FCFEF7F1
:10E2B000EDFF082104F15000FFF744FD94F866607B
:10E2C00095ED029A9FED6C8A9FED6A0ADFED698AEF
:10E2D0009FED67AADFED68AAF0EE480A39EE000A62
:10E2E00015F0E4FBD5ED017AC9EE279A022384F8F4
:10E2F0007C30B5EEC00AF1EE10FA48BF30EE080AE5
:10E3000030EE688A002E7AD12046FFF7BDFE074620
:10E310002046FFF72DFFE3681B7C0646002B00F02C
:10E320009D802046FFF712FD0FB106B118B9636F4B
:10E330001B78012B63D1D5ED037ADFED4F0AE7EEB1
:10E340008A9A38EE280AA9EE8A9AA9EE8A0A15F066
:10E35000ADFBB5EEC00AF1EE10FA01D530EE2A0A97
:10E36000606AD5ED007A036A30EE688A93ED060A9A
:10E37000F0EE480A20EE270AB0EE691A01F0CCFA56
:10E3800040B3D5ED047AB0EEE97AF0EEE77AB4EE78
:10E39000E77AF1EE10FA1DDA6B7E53B1D5ED057A0E
:10E3A000B0EEC97AF0EEE77AB4EEE77AF1EE10FA61
:10E3B00010DAAB7E002B41D1A36F0133A367022299
:10E3C000012101A8FAF770FA019B082B0DD194F8EE
:10E3D000666097E7A36F0133A3670222012101A8BA
:10E3E000FAF762FA019B082B09D0606AFEF786FBF8
:10E3F000FEF74CFF082104F15000FFF7A3FC206951
:10E40000837D002B00F0F9802B7E002B36D0D5EDDC
:10E41000048AF0EEE99AF0EEE87AF4EEE79AF1EE8B
:10E4200010FAC0F2B080206DB0FA80F000234009ED
:10E4300084F87C3005B0BDEC088BF0BDA36F226979
:10E440000133967DA3670222012101A8FAF72CFA75
:10E45000019B082BC9D1002EB9D0D0E7002F3FF483
:10E4600066AF00283FF463AF65E700BF000000001F
:10E470006F120339DB0F4940DB0FC9406B7E53B18C
:10E48000D5ED057AB0EEC97AF0EEE77AB4EEE77A28
:10E49000F1EE10FAC7DAAB7E002B7BD1D5ED048A02
:10E4A0001FED0DAA5FED0D9A5FED0DBA28EE8AAA59
:10E4B000B0EE69BA03237AEE299A84F87C30F0EE44
:10E4C000E8AA94F86630002BADD12046FFF7DCFDBA
:10E4D00007462046FFF74CFEE3681B7C0646002BF0
:10E4E00075D02046FFF732FC0FB106B118B9636F43
:10E4F0001B78012B97D138EE290A5FED210A15F020
:10E50000D5FAB5EEC00AF1EE10FA01D530EE2B0ABD
:10E51000606AD5ED007A036A30EE4B8A93ED060A05
:10E52000F0EE480A20EE270AB0EE681A01F0F4F97E
:10E53000002835D02B7E39EE0A9A43B1D5ED047A06
:10E54000F0EEE77AF4EEE7AAF1EE10FA28DA6B7E45
:10E5500053B1D5ED057AB0EEC97AF0EEE77AB4EEB4
:10E56000E77AF1EE10FA1BDAAB7E002B34D1A36F01
:10E570000133A3670222012101A8FAF795F9019B53
:10E58000082B9ED018E06B7E002B7FF479AFAB7E1A
:10E59000002B85D023699B7D002B7FF444AF7DE762
:10E5A000A36F0133A3670222012101A8FAF77CF9C6
:10E5B000019B082B3FF437AF606AFEF79FFAFEF726
:10E5C00065FE082104F15000FFF7BCFB2BE7002F8C
:10E5D0008DD000288BD08EE7A36F22690133967D02
:10E5E000A3670222012101A8FAF75EF9019B082B1B
:10E5F000E2D1002E3FF465AF15E7012101F09EFB4B
:10E6000002E700BFD0E9052370B50021044602F1FE
:10E6100014001C32C3E90902C3E9061184B019626F
:10E6200094F86630A3BB2046FFF72EFD0646204631
:10E63000FFF79EFDE3681B7C05467BB32046FFF792
:10E6400085FB0EB105B118B9636F1B78012B1FD183
:10E65000A06901A902F026FC50BB4FF4007104F13F
:10E660005000FFF76FFBA36F0133A36701A80222DD
:10E670000121FAF719F9019B082B09D0606AFEF70E
:10E680003DFAFEF703FE082104F15000FFF75AFBA4
:10E69000206DB0FA80F0400904B070BD002ED3D0D8
:10E6A0000028D1D0A06901A902F0FCFB0028D4D039
:10E6B0006369606A93ED051AD3ED030A9DED010AC3
:10E6C00001F02AF90028CED0A36F0133A3670222FC
:10E6D000012101A8FAF7E8F8019B082BA0D0CDE7AB
:10E6E00070B5044680692DED028BC26843F69C0329
:10E6F00084B0D15C02F006FB002864D0A369DA681C
:10E7000092F82020002A5BD0DA69002A5BD01268D8
:10E71000E1681A63012083F854001A6400228979A1
:10E720009A632046FFF78AFC9FED3F8A94F8663093
:10E73000002B36D12046FFF7A7FC05462046FFF701
:10E7400017FDE3681B7C0646002B68D02046FFF7C8
:10E75000FDFA0DB106B118B9636F1B78012B20D1FA
:10E76000A06901A902F09EFB002837D14FF4007187
:10E7700004F15000FFF7E6FAA36F0133A36701A885
:10E7800002220121FAF790F8019B082B09D0606A58
:10E79000FEF7B4F9FEF77AFD082104F15000FFF707
:10E7A000D1FAE368997901B1D9792046FFF746FC9F
:10E7B000206DB0FA80F0400904B0BDEC028B70BD52
:10E7C0009A69002AA3D104F150004FF40071FFF7B9
:10E7D000B9FA002004B0BDEC028B70BD606A2369F9
:10E7E000026AD3ED137A92ED011AD3ED090A9DED79
:10E7F000010AB8EEC11A67EE887A21EE271A01F0F5
:10E800008BF80028B8D0A36F0133A367022201213F
:10E8100001A8FAF749F8019B082B87D0B7E7002D2C
:10E820009AD0002898D09BE7DB0FC9402DE9F04132
:10E83000C36A1B682DED028B9D7A84B0044655B9DE
:10E840004FF400315030FFF77DFA284604B0BDEC9C
:10E85000028BBDE8F0818069C36840F20221D3EDEC
:10E860000C7AB3F8008019800022012180F854103E
:10E87000026482640021F1EE677A43F69C02C0EDE7
:10E88000117A84F87D10995C02F03CFA002800F0BF
:10E89000C880A369DA6892F82020002A00F0CE80B0
:10E8A000DA69002A00F0BD8012681A639FED978A2A
:10E8B00000229A6394F86630002B40F0E8802046EE
:10E8C000FFF7E2FB05462046FFF752FCE3681B7C9E
:10E8D0000646002B00F005812046FFF737FA0DB100
:10E8E00006B120B9636F1B78012B40F0D080A0697E
:10E8F00001A902F0D7FA002840F0A28004F15005E7
:10E9000028464FF40071FFF71DFAA36F0133A36788
:10E9100001A802220121F9F7C7FF019B082B08D0AB
:10E92000606AFEF7EBF8FEF7B1FC08212846FFF716
:10E9300009FA4FF48050FFF71DFA01462846FFF709
:10E9400015FA2069E36AC2681B68D2ED027A93ED7A
:10E95000007A0268A3699FED6D8A83ED0C7AF8EE68
:10E96000E77A002667EE877A5E63FDEEE77A136842
:10E9700017EE901A9847A369D96840F20350012214
:10E9800008801E645E649E6483F8542094F86630A8
:10E99000002B35D12046FFF777FB06462046FFF7D0
:10E9A000E7FBE3681B7C0746002B00F0A1802046B4
:10E9B000FFF7CCF90EB107B118B9636F1B78012BC3
:10E9C0001ED1A06901A902F06DFA002862D14FF4AE
:10E9D00000712846FFF7B6F9A36F0133A36701A8BA
:10E9E00002220121F9F760FF019B082B08D0606A21
:10E9F000FEF784F8FEF74AFC28460821FFF7A2F943
:10EA0000A369DB68A3F80080256DB5FA85F56D096B
:10EA10000123284684F87D3004B0BDEC028BBDE8AC
:10EA2000F08104F150004FF40071FFF78BF90025DD
:10EA3000284604B0BDEC028BBDE8F0819A6930E74E
:10EA4000606A2369026AD3ED137A92ED011AD3ED5D
:10EA5000090A9DED010AB8EEC11A67EE887A21EE27
:10EA6000271A00F059FF002849D0E06A02F07AF82E
:10EA7000A36F0133A36705460222012101A8F9F71C
:10EA800013FF019B082B3DD1002D3FF413AF04F180
:10EA900050054EE7606A2369026AD3ED137A92ED5E
:10EAA000011AD3ED090A9DED010AB8EEC11A67EE0D
:10EAB000887A21EE271A00F02FFF00288CD0A36F50
:10EAC000A269013392F85560A3670222012101A8CF
:10EAD000F9F7EAFE019B082B89D1002E3FF456AFCF
:10EAE0008EE7002D3FF4FEAE00287FF400AFF9E67C
:10EAF000002E3FF462AF00283FF45FAF61E704F1FE
:10EB0000500502E704F150050AE700BFDB0FC940DA
:10EB100070B5044684B0406AFDF7F0FFE368997968
:10EB200001B1D9792046FFF789FA13E0FFF70EF912
:10EB30000EB105B118B9636F1B78012B22D1A36FF9
:10EB40000133A3670222012101A8F9F7ADFE019B61
:10EB5000082B1DD194F8663020469BB9FFF794FA34
:10EB600006462046FFF704FBE3681B7C054620466B
:10EB7000002BDBD1002EDED0002DE0D1636F1B789F
:10EB8000012BDCD0206DB0FA80F0400904B070BDDC
:10EB9000606AFDF7B3FFFEF779FB082104F150002E
:10EBA000FFF7D0F8EEE700BF8842F8B553D09142A6
:10EBB000064653D00C1A551AAC42A2EB000C39D0C1
:10EBC0000544ACEB0407A7421CDD012C49D0002F03
:10EBD00006EB04030BDD711E03EB070E11F8012F8A
:10EBE0001878087003F8012B7345F7D13E449CFB5D
:10EBF000F4F304FB13C353B3A446E41AACEB0407C9
:10EC0000A742E2DC012F33D006EB0C02002CA2EB72
:10EC100007031EDD1E1B13F8011D12F8014D1C70A9
:10EC2000B3421170F7D19CFBF7F407FB14C474B125
:10EC3000BC46C6E70138C6EB41020B4610F8014F4F
:10EC40001D78057003F8014B9342F7D10D46284615
:10EC5000F8BD1E46E7E715462846F8BD0546284696
:10EC6000F8BDBCF1010437780FD137552846F8BDFF
:10EC70000CF1FF32B45C12B934702846F8BD31464D
:10EC8000701C15F085F83470F7E72246711C304689
:10EC900015F07EF83755E9E72DE9F04705462DEDEB
:10ECA000028B406A9FED938A00F08AF905F17106A4
:10ECB00005F1670805F1500905F1680A00240127EC
:10ECC00095F86630B3B1022B00F0C580032B00F03D
:10ECD000F18085F8673085F8687002216B18012093
:10ECE00083F8674085F86640FFF744F801464846D8
:10ECF000FFF73CF86B6F1B78013B0A2B07D8DFE866
:10ED000003F0A0060699725F543D2C2112000121E8
:10ED10004846FFF717F8434603F8014BB342FBD1CF
:10ED20006B6F1F70CCE72846FFF780FD0028F2D0FC
:10ED30004FF00003324651464046FFF735FF85F855
:10ED40007040BDE76B6A93F86730002BDFD028690D
:10ED500001F0F0F80028DED0EAE76B6A93F867204C
:10ED6000002AD4D01B6ADB69002BD0D0E968284682
:10ED70005031FFF727FA0028CDD0D9E76B6A93F816
:10ED80006720002AC3D01B6ADB69002BBFD02B6928
:10ED9000DB7D002BBBD02B6828461B689847284694
:10EDA000FFF79EFC0028B6D0C2E76B6A93F8673085
:10EDB000002BACD0286901F005F90028ABD0B7E7EB
:10EDC0006B6A93F86720002AA1D02869C26892F87C
:10EDD00029201AB11B6ADB69002B98D001F08EF84C
:10EDE000002898D0A4E76B6A93F86720002A8ED099
:10EDF0001B6ADB69002B8AD0E96828463431FFF7AB
:10EE0000E1F9002887D06B6AEA681B6A92ED117AF3
:10EE1000D3ED017AAB69F8EEE77A27EE087A284657
:10EE2000C7EE276AC3ED0D6AFFF7ECFB00283FF43D
:10EE300072AF7DE7686A00F0CDFB00283FF46BAF4E
:10EE400076E72846FFF764FE686A00F0B9F8002804
:10EE50003FF461AF6CE7E8680278002A3CD00422F6
:10EE600085F867200122417849B12969C968897804
:10EE700029B12A44062182F867101A4601338178A5
:10EE800029B12A44072182F867101A4601334179D3
:10EE900029B12A440B2182F867101A460133C17840
:10EEA000E1B12A44082182F86710591CEA1882F857
:10EEB000677013E72A69D2689278042185F8671091
:10EEC0008AB106201A4685F8680002232B440720E1
:10EED0002A4483F86700EAE70123C4E7017931B1E6
:10EEE0002A440521DFE7194602220123EEE71946ED
:10EEF0001346DBE783F9223E08B5FFF7CDFE00BFDE
:10EF00002DE9F041164604461F468C460FCE254695
:10EF100045F804CB0FC596E80700274BB4F80CC0A2
:10EF2000D4E9018685E8070093E803000025A28A5A
:10EF3000E662266925630023A563A4F830C0228712
:10EF4000C4E90875C4F828806663E0633A78A4F8D9
:10EF5000401084F86720A366E36623676367A367AE
:10EF600084F84250A4F84450A564A4F8645084F88E
:10EF7000665004F17C002946442214F023FFD7EDAB
:10EF8000047A97ED056AD7ED0D6A0C4BA4F8C050D2
:10EF900086EE277A4FF07E522046C4F8A820C4F8A7
:10EFA000E83067EEA67A27EE277AC4ED1F7A84ED63
:10EFB000207ABDE8F08100BFC88E02080000204121
:10EFC00038B5436A0446986901F096FE0023606AEA
:10EFD000C4F88430C4F88830C4F8B430C4F88C3035
:10EFE000FEF752FF054630B9606A08215030FEF73F
:10EFF000A9FE284638BD0023204684F84230FDF79C
:10F000006FFD284638BD00BF036AD3ED047A93ED47
:10F01000056AD3ED0D6A86EE277A67EEA67A27EEAB
:10F02000277AC0ED1F7A80ED207A704770B50268AC
:10F03000036A9FED3C7AD2ED027AD3ED0C6A3A4B2B
:10F040003A4D3B4E8CB0002267EE877A07920992C8
:10F050000B920446089337480592042308210C229A
:10F06000049587EEA67A0A9606908DF81C308DF8E6
:10F0700024108DF82C200CAD08E051ED026AB4EE9E
:10F08000E67AF1EE10FA58BF134642D45A10002B1C
:10F09000A5EBC201F1DC04AB9D423FD055ED026A05
:10F0A000B7EE006A86EE267A04F1280004F1C20168
:10F0B0000390019167EE877ADFED1F6AC4ED2B7A2A
:10F0C00067EEA67A84ED1E7AC4ED2C7AFDF746F938
:10F0D0000199039802910190FDF720FA15F8043C7C
:10F0E00084F8D93010224FF4A8630125DDE901012D
:10F0F00084F8D520A4F8D63084F8E450FDF784F9DC
:10F10000DDE9010184F8E5500CB0BDE87040FDF781
:10F110009FB99B1A013BA1F10805B7E79FED077A5C
:10F1200006ADC1E71F859B3F000020420000204143
:10F130000000A0420000A041E4388E3FCDCCCC3D81
:10F1400038B5818B05468069FCF742F908B101208A
:10F1500038BD044605F12800FDF716F9A5F8C000F2
:10F16000204638BD10B504466430FDF7B5FC606A32
:10F1700040215030FEF7E6FD2046FDF7BFFCBDE81C
:10F180001040FEF783B800BF38B50546FFF7D8FF3B
:10F19000044608B1204638BD28460821FFF7E2FFA3
:10F1A000204638BD38B5D0E908256B6A92ED090ACA
:10F1B0001A6A92F82020022A2DED028B044628D0EC
:10F1C000D3ED2B8A686B0368B4EEE80AF1EE10FA0F
:10F1D0009B68D8BFF0EE408A9847A86B226A036804
:10F1E000B0EE408AF4EEC88AF1EE10FA92ED090A08
:10F1F0009B68D8BFB0EE688A9847B4EEC80AF1EEB3
:10F2000010FA58BFB0EE480ABDEC028B84ED3A0A02
:10F2100038BD044BDFED047AD3ED008A68EEA78A8F
:10F22000D0E700BF000200207CD8103F036A93F8AB
:10F230002030032B10B5044618D0FFF7B3FF236A24
:10F24000D3ED067A20EE270AB5EE400AF1EE10FA69
:10F2500009D4D3ED0B7AB4EE670AF1EE10FAC8BF09
:10F26000B0EE670A10BD9FED060A10BDFFF79AFFCA
:10F27000236A94ED2D7AD3ED067A67EE877AE1E77B
:10F2800000000000054B1B680B295B6A04D800EBEB
:10F2900041005B00A0F84C30704700BFE0C6002082
:10F2A000D0ED1E7A03689FED087A93ED020AA1F56E
:10F2B000006167EE877A07EE101A67EE807AB8EE83
:10F2C000C70A27EE800A70473333533A10B584B02B
:10F2D000044603AA02A901A8FDF780F910BB9FED1F
:10F2E000156ADDED016A9DED027ADDED037A66EEC9
:10F2F000866A27EE067AFCEEE66A67EE867A16EEF6
:10F30000903ABCEEC77AFCEEE77AA38717EE103A84
:10F31000E38717EE903A0120A4F8403084F84200C9
:10F3200004B010BD20468021FFF71CFF002004B070
:10F3300010BD00BF00C05A450B4B93ED007AF7EEAD
:10F34000086AC6EE877A10B5044667EEA00A27EE73
:10F35000800AFFF7BBFF28B1044B1B685B6A5B00A8
:10F36000A4F85A3010BD00BF00020020E0C6002003
:10F370002DE9F8432DED068B9FED3F8A446A9FED02
:10F380003FAA3F4F0546B0EE409AF0EE608AF0EE9D
:10F39000489A45F6BF5694F866302046002B3FD178
:10F3A000FEF772FE81462046FEF7E2FE80462046CA
:10F3B000FEF700FFB1EE687AB9F1000F03D0B8F1A3
:10F3C000000F00D018B9636F1B78012B28D1D5ED41
:10F3D0001A7AD5ED1B6A77EEA67A77EE897AA7EED0
:10F3E0008A8AB4EEE88AF1EE10FA04DCB4EEC78A39
:10F3F000F1EE10FA21D501212846FFF7B3FEA36FE5
:10F400000133A3672046FEF73FFD48B9606AFDF768
:10F4100075FBFDF73BFF04F150000821FEF792FC5D
:10F420006B6A1B6D1BBBC8EE097ABDEC068B2B6AA1
:10F430000120C3ED057ABDE8F883F0EE690AB0EE6D
:10F44000480A2846FFF778FF03462046002BD6D00F
:10F450003A68A36F526A01335200A5F85220A3679D
:10F46000FEF712FD0028D1D0013E94D1D8E7BDECC3
:10F47000068B0020BDE8F883000000000BD7A33AFC
:10F48000E0C600202DE9F0472DED048B002684B066
:10F49000CDE90266446A9FED4B9A4B4F8DED000A11
:10F4A0000546F0EE408AB0EE608ACDED010A42F2E8
:10F4B00010780DE03A68A36F526A01335200A5F844
:10F4C0005420A367FEF7E0FC00283FD0464547D014
:10F4D00094F866302046002B42D1FEF7D5FD8246D7
:10F4E0002046FEF745FE81462046FEF763FE06F005
:10F4F000010304A9024601EB8303F0EE490A284602
:10F50000BAF1000F03D0B9F1000F00D01AB9626F41
:10F510001278012A24D195ED1A7AD5ED1B6A53EDA4
:10F52000027A13ED040A37EE267A013677EEC77AAF
:10F5300043ED027AFFF700FF03462046002BB9D1C6
:10F54000A36F0133A367FEF79FFC48B9606AFDF71C
:10F55000D5FAFDF79BFE04F150000821FEF7F2FBFF
:10F560006B6A1B6D43BB9DED027ADDED037ADFED27
:10F57000176A2B6A38EE688AF5EE040A28EE208AAC
:10F5800077EEC77A88EE277AB4EEE67AF1EE10FAD3
:10F5900083ED047A0CD4DFED0E7AB4EEE77AF1EE67
:10F5A00010FA05DC012004B0BDEC048BBDE8F08747
:10F5B00028460221FFF7D6FD002004B0BDEC048BE5
:10F5C000BDE8F08700000000E0C60020BD37063629
:10F5D0006F12833B10B5036A93F8202082B0044673
:10F5E000C2B1032A16D0022A20D1D3ED047A93EDBA
:10F5F000056AD3ED0D6A86EE277A012084F867004C
:10F6000067EEA67A27EE277AC4ED1F7A84ED207A7A
:10F6100002B010BDD3ED030A93ED020ACDED010A4D
:10F620002046FFF7A5FEDDED010A10B9002002B06B
:10F6300010BDB1EE600A2046FFF724FF0028F5D088
:10F64000236AD2E700B52DED048B83B0B0EE409A6B
:10F65000B0EE410AB0EE608AF0EE419A0190FDF7FB
:10F66000B9F9F0EE408AB0EE690AFDF767F9F0EEFD
:10F67000407A67EE890A28EE400AE8EE880A019887
:10F68000A8EE890A03B0BDEC048B5DF804EBFFF72C
:10F6900053BE00BF10B5D0ED1A7A90ED2C7AF0EE83
:10F6A000E76AB4EEE67AF1EE10FA2DED088B044627
:10F6B000C0ED270A08D490ED1B8AF0EEC86AB4EEBC
:10F6C000E67AF1EE10FA08D520464FF48061FFF794
:10F6D00049FD0020BDEC088B10BD37EE88AA77EEFF
:10F6E000C87A9FED828AB0EE40BAB0EE410AF0EEE1
:10F6F000418A27EE888AB0EE609AF0EE61BAFDF793
:10F7000069F9F0EE407AB0EE680AF0EE678AFDF72C
:10F7100015F968EE00AAB1EE4AAAEAEE28AA204638
:10F7200028EE288A6AEE008A94ED297AD4ED287AA8
:10F73000D4ED2A6A78EE689A7AEEC75A39EEE76A0B
:10F74000A6EEA57AE6EE867A84ED297AC4ED287ACB
:10F75000FFF728FD236A29EEA97AD3ED0A7AAAEEEB
:10F76000AA7A70EE277A67EEA77AB4EEE77AF1EE1E
:10F7700010FA00F3B6805E4B94ED227AD3ED005A76
:10F7800094ED1F5AD4ED216A9FED5A4ADFED5A3AA3
:10F79000F7EE087A87EEA56A78EE897AF0EE478A66
:10F7A00037EEC88A3BEE6A0AE5EE088AB0EE669A42
:10F7B000A5EE009A68EE868A29EE069A28EEA86AD7
:10F7C000F7EE004AA9EE096A25EEA3BAF1EEC67A71
:10F7D00084EE275AB4EEE45AF1EE10FA69D494EDAF
:10F7E000205ADFED467A25EE275AE0EE056AA8EEAC
:10F7F000057AC4ED216A84ED227A68EEA99AB0EE0A
:10F800006B0AE9EE2A9AC4ED239AFDF7E3F8B0EE0D
:10F81000408AB0EE6B0AFDF791F860EE687A69EE07
:10F82000000AE9EE087A2046E8EE880A2BEE277AED
:10F83000B0EE670A6BEE207A84ED247AC4ED257A67
:10F84000FFF744FD00283FF445AF2D4B626A1B686B
:10F8500052685B6A5B00A4F85C30002A7FF43AAF20
:10F86000D4ED217A274BB6EE007AF4EEC77AF1EEAA
:10F8700010FA2DD501221A70B6EE007AF4EEC77A8E
:10F88000F1EE10FA27DB204A0124002114701970D0
:10F890001E4C1F49236801EB83010133B3F5805FE0
:10F8A00028BF002381ED00AA32BF236023601370BC
:10F8B00010E7DFED184A66EEA46A67EE244A29EEE7
:10F8C000059A68EE858AC4ED216AC4ED224A94E760
:10F8D0001A78002AD0D10C4A1378002B3FF4FAAEE4
:10F8E000D6E720464FF48051F1E600BF3ACD133FF2
:10F8F00000020020AC5C313FABAA2A3F6F120339F3
:10F90000E0C60020800800208108002094BE00206E
:10F91000947E0020A4707D3F38B5056AD5ED077A46
:10F9200095F820302DED068BB8EEE78A032B28EEF4
:10F9300020AA68EE019A0446F0EE408A00F0EB80BF
:10F9400095ED067AC0EE077A204628EE278AFFF763
:10F9500029FCD4ED268AB1EE409AB4EE689AF1EE15
:10F9600010FA2FDCF4EE408AF1EE10FAC8BFF0EE88
:10F97000408AB4EE498AF1EE10FA08D4B4EEC08A97
:10F98000F1EE10FAD4BFB0EE489AB0EE409A226A77
:10F9900092F82030032B2DD0DFED657AF0EE4A1A75
:10F9A000022BE9EEA71A18D07BB9B0EE4A1AF0EE96
:10F9B000490AB0EE680ABDEC068B2046BDE8384027
:10F9C000FFF768BEF0EE498AD3E720462021FFF713
:10F9D000C9FBBDEC068B002038BDF0EE490AB0EE45
:10F9E000680ABDEC068B2046B0EE611ABDE83840CF
:10F9F000FFF728BE92F84C3033B3F0EEC97AF4EE3C
:10FA0000E78ADFED4C6A77EEE87AF1EE10FA4CBF48
:10FA100092ED147A92ED157A67EEA67AE7EE878A70
:10FA2000F0EE687AD2ED128AF4EE687AF1EE10FA0E
:10FA300008D4F4EEC07AF1EE10FAD4BFF0EE678A83
:10FA4000F0EE408AC4ED268AD2ED106A94ED2D7A4C
:10FA50009FED380A9FED386A9FED388A66EE807A0E
:10FA600078EEC75AF0EE480AA5EEA77AC9EE077AF3
:10FA700084ED2D7A67EEA67ADFED316AB0EEE77A93
:10FA8000B4EE467AF1EE10FA98BF27EE807A94ED44
:10FA90002F0A88BF9FED2B7A30EE260A88BFF0EE42
:10FAA000477AC4ED2E7A30EE070A98BF79EEA79A0E
:10FAB00013F0FCFFB5EEC00AF1EE10FA48BF30EECD
:10FAC000080ADFED1F7A9FED1D8A70EE677AF0EE6F
:10FAD000480AC4ED2F7A3AEE000A13F0E7FFB5EEBC
:10FAE000C00AF1EE10FA48BF30EE080A9FED141A72
:10FAF000DFED0F7A30EE411AF0EE490AF0EE411ACE
:10FB0000E9EEA71A2046B0EE680ABDEC068BBDE808
:10FB10003840FFF7BFBDD5ED110A90ED2D0A13F067
:10FB200065FFD5ED067A20EE270AC8EE807A0BE74E
:10FB3000A69B44396F12033900004844DB0FC940CB
:10FB4000DB0F494000000000C3691B78EBB1D0E92E
:10FB50000532D0ED046AD2ED007A93ED007A77EEAB
:10FB6000E66A37EEC77AC6EE877A67EE807AF5EEF8
:10FB7000407AF1EE10FAB8BFDFED047AF4EEC07A05
:10FB8000F1EE10FAD8BFB0EE670A7047000000002F
:10FB9000704700BF704700BF10B52C21044612F01B
:10FBA00099FF204610BD00BF10B52C21044612F06D
:10FBB00091FF204610BD00BF10B504468088FDF7B8
:10FBC000FFFA064BE168D3ED007AA06880EE270AC1
:10FBD000FCF778FE84ED040A10BD00BF24910208F2
:10FBE000C26908B50346107870B19A6993ED047A3A
:10FBF000D2ED007AF1EE046A77EEA67AB4EEE77AF7
:10FC0000F1EE10FA02DA08BD012008BD586A01229F
:10FC100083F820204FF480215030FEF793F8002025
:10FC200008BD00BFF0B4D1E900478968094E818062
:10FC3000151D09498460426102F1080482620022B4
:10FC4000C0E90654C76006610160F0BC80F820205E
:10FC5000426270470000C07FEC920208836A1B8AF0
:10FC60005A1F92B2032A10B504460BD80B49023B27
:10FC700051F822009BB20A4A32F81310FDF7C8F976
:10FC8000A08010BD023B9BB2062B064888BF012115
:10FC9000F1D9FDF7BDF9A08010BD00BF0C9302089B
:10FCA0001C9302080000024038B501F114054561BB
:10FCB0004FF6FF7585800B4B0B4A816004258162EE
:10FCC000C560036101F1180500231C31C0E906512C
:10FCD0000446026080F820304362FFF7BFFF2046F1
:10FCE00038BD00BF0000C07F00930208EFF310830F
:10FCF00072B6826881611268A0F85A1007EE901AF5
:10FD00001268F8EEE77AC0ED0A7A516283F3108840
:10FD1000704700BF028811430180704710B500236F
:10FD20000446A0F858301430FFF7F4FF20694FF470
:10FD300080715030FEF706F810BD00BFC368024660
:10FD4000987820B9936819895868F9F71FBA19B9D2
:10FD500093F82830002BF5D100B59068054B018948
:10FD6000406883B000920222F9F798F903B05DF879
:10FD700004FB00BFF9FE0008C2689FED0E7AD2EDC9
:10FD8000097A77EEA77AB5EE006A67EEA76A27EEE2
:10FD9000877A66EE866AB7EE006AB4EE467AF1EECE
:10FDA00010FAC0ED0D7AC0ED0E6A00D57047012142
:10FDB000FFF7B4BF6F12033970B51D4E0660002502
:10FDC000164681604FF6FF7200210562456285622A
:10FDD000C562056345638563C56345648564C56421
:10FDE0000565456505664566C0E90411C0E906116B
:10FDF000C660A0F868200164816580F85C1080F816
:10FE00006C10A0F86E101D460446FFF7B5FFF3789E
:10FE100063B13388013B9BB2012B9CBF0123E37587
:10FE200095F82030032B04BF0123E375204670BDF5
:10FE3000E4930208C37D43B90269526A126A92F8D8
:10FE40002020032A1CBFC268D370B0F86E301BB9E3
:10FE5000837D0BB9C268D370704700BFF8B5044604
:10FE60000D46EFF3108672B672B9E36828469968BA
:10FE7000FCF73CFD07EE900AF8EEE77AE061C4ED8E
:10FE80000B7A86F31088F8BDC768C069D7E90213FA
:10FE9000281A1844F860FCF729FDF860E5E700BF70
:10FEA000C3689B7810B5044633B9A368BDE8104019
:10FEB00019895868F9F76AB900221146FFF7CEFF91
:10FEC000E3681A792AB1236800211B682046984705
:10FED000E368DB785BB123699B6943F67802D968F4
:10FEE000895C0122E27519B183F8562000E0E375C0
:10FEF0000123A375D9E700BFFFF7D2BFC368012272
:10FF000093F8291010B59A7000230446837529B917
:10FF100003695B6A1B6AD96901B9DA61204600216D
:10FF2000FFF70CFF2069C168BDE810401831FEF7EB
:10FF300049B900BFD0F810C02DE9F041DCF80C4001
:10FF40008769DCF82450183406460FCC88B0D5F801
:10FF500020E04FF0010801ADCEF81C800FC594E8F9
:10FF6000070085E80700DDED057AB0EE087A67EE58
:10FF7000877A4FF480730024604601A9CDED067A9C
:10FF8000ADF81C308DF81E40FEF71CF948B1B3697E
:10FF900007F10802934207DD33695B6A1B6AC3F805
:10FFA0001C8008B0BDE8F081083FBB4233695B6A42
:10FFB0001B6ABABF4FF0FF32DA61DC6108B0BDE8FE
:10FFC000F08100BF2DE9F04FC3682DED068B9A78C4
:10FFD000D3ED079A93ED08AA83B004461AB1857D44
:10FFE000002D00F0FC812569E2696B6AA2611B6A41
:10FFF00093F82020002A00F0DC81022A40F0E481FE
:020000040801F1
:10000000D3ED028A9FED989A9FED988A002713E01E
:100010002369586AFFF736F9AB6F0133AB6728469F
:10002000FDF732FF07EE907AF8EEE77A70B3F4EE60
:10003000C87AF1EE10FA33D595F8663028460137C4
:1000400073BBFEF721F880462846FEF791F8064676
:100050002846FEF7AFF8F0EE490AB0EE680AB8F1AC
:10006000000F01D006B118B96B6F1B78012B17D1A7
:100070002369586AFFF760F905210028C8D1AB6FE2
:100080000133AB672846FDF7FFFE48B9686AFCF705
:1000900035FDFDF7FBF805F150000821FDF752FE94
:1000A00025692B6D002B40F08F81C9EE8A7AA269F9
:1000B00001929846002600279FED6C7ADFED6C9A3E
:1000C000DFED6DAA67EE877AB7EE007AFDEEE77A8C
:1000D000B6EE00AA17EE909AF8EEE77A87EE279A26
:1000E00011E02369586AFFF7CDF8AB6FA2690133BD
:1000F000B618AB67284647EBE277FDF7C5FE002848
:1001000059D0C14561DD95F866302846002B5CD199
:10011000FDF7BAFF82462846FEF72AF883462846AE
:10012000FEF748F807EE908ADFED530AB8EEE77A5B
:10013000BAF1000F03D0BBF1000F00D018B96B6FFC
:100140001B78012B41D1E368D3ED077AB0EE690A41
:10015000A7EECA0A08F1010867EE897AA7EE270A16
:1001600013F0A4FCB5EEC00AF1EE10FA48BF30EE71
:100170002A0A30EE698AB0EE480AFCF72BFCF0EE52
:10018000407AB0EE480A28EEA78AFCF7D7FB23692D
:10019000F0EE400A68EEA00A586AB0EE480AFFF78F
:1001A000CBF8052100289CD1AB6F0133AB67284603
:1001B000FDF76AFE48B9686AFCF7A0FCFDF766F82F
:1001C00005F150000821FDF7BDFD25692B6D002BC1
:1001D00040F0FA800199A26908318A4200F3FB805D
:1001E000019908398A4280F203816B6A1B6A4FF0D9
:1001F000FF31D9615B68E168DFED1E5AD1ED026A1B
:1002000091ED077A91ED066A5B0007EE903AF8EE01
:10021000E66AF8EEE77A27EE257AC7EEA65A019B42
:10022000A2EB030ABAF1000FB8BFCAF1000A07EE49
:1002300090AAC7EE256AF8EEE77AC4ED0F7A77EE5A
:10024000E67AF0EEE77A87EEA67AB4EEC67AF1EEB9
:1002500010FA00F3B580DFED069ADFED07AA4FF044
:100260000008B6EE00AA1BE0000000000000FA45FE
:10027000DB0F494083F9A23EDB0FC9402369586A6E
:10028000FFF700F8AB6FA2690133B618AB672846D9
:1002900047EBE277FDF7F8FD00285BD0C14563DD51
:1002A00095F866302846002B5ED1FDF7EDFE8246BC
:1002B0002846FDF75DFF83462846FDF77BFF07EEE6
:1002C000908A5FED130AF8EEE77ABAF1000F03D0D7
:1002D000BBF1000F00D018B96B6F1B78012B43D115
:1002E000E36893ED077AB0EE690AA7EE0A0A08F10F
:1002F000010867EE877A67EE897A30EE670A13F0B5
:10030000D5FBB5EEC00AF1EE10FA48BF30EE2A0A6E
:1003100030EE698AB0EE480AFCF75CFBF0EE407AFA
:10032000B0EE480A28EEA78AFCF708FB2369F0EE36
:10033000400A68EEA00A586AB0EE480AFEF7FCFFD1
:10034000052100289AD1AB6F0133AB672846FDF732
:100350009BFD48B9686AFCF7D1FBFCF797FF05F1F4
:1003600050000821FDF7EEFC23691B6D63BB4FEACB
:1003700049052A46EB1730463946F0F795FC09FB4C
:1003800000F9A6EB490907EE105A07EE909AB8EE6D
:10039000C77AF8EEE77AB6EE006AC7EE876AE268D7
:1003A0000123D0601D4676EE867AC2ED047AE375AD
:1003B0000BE0D3ED028AD3ED057A68EEA78A21E639
:1003C00020460221FFF7AAFC0025284603B0BDEC19
:1003D000068BBDE8F08F6B6A01211B6A09E72021BB
:1003E000FFF79CFC284603B0BDEC068BBDE8F08F00
:1003F000204604211D46F3E7B0F86E30022B10B5FD
:10040000044619D001D85BB110BDA3F58073032B4E
:100410000DD80369BDE81040586A0A21FEF732BFC3
:1004200083681B681B685B6AA0F85A3010BDBDE882
:1004300010400821FFF772BCC368DB8D5A1F92B2CF
:10044000032A2AD81D49023B51F822009BB21C4ABC
:1004500032F81310FCF734FEE3689FED1A7A1B8E16
:10046000FEEE007AE0EE077A5A1F92B2032AC4ED3C
:10047000187A1AD81149023B51F822009BB2104A4F
:1004800032F81310FCF71CFE9FED0E7AFEEE007A98
:10049000E0EE077AC4ED197A10BD023B9BB2062B41
:1004A000094888BF0121D5D8D1E7023B9BB2062B72
:1004B000054888BF0121E5D8E1E700BF8C93020819
:1004C0009C930208CA269B3E00000240B0F86E20B2
:1004D00038B512F4807327D083685C6A0123B2F5C3
:1004E000817F63614FF482704FF000034FF400612D
:1004F0002361C4E90833A360A362606008BF0223DC
:10050000E1604FF400754FF00A014FF02000C4E99C
:100510000650E16208BF23612046F3F791FB2046B5
:10052000F3F74EFB012038BD184638BD38B5B0F89A
:100530006E30DB0501D4012038BD03690446092172
:10054000586AFEF79FFEA3685B6A93F85130012B4F
:10055000DDB206D020464FF48071FFF7DFFB0020AC
:1005600038BDB4F87410206F0022FAF737FFA26884
:100570002B46506A04F1680104F16A02F3F74CFD5E
:10058000D9E700BF10B50446B0F87410006F01221F
:10059000FAF724FF23690B21586AFEF773FEB4F8BB
:1005A0006E3040F2011293420CD040F2031293429B
:1005B00032D0B3F5807F21D020460821BDE810401D
:1005C000FFF7ACBBB4F86A3083EA13210AB282EABF
:1005D0001112C2F38D014A4082EA5202D2070CD4B2
:1005E00013F4804F09D1C3F30D03E2682364D2787A
:1005F000012384F86C3002B1E37510BDB4F86A30A1
:1006000083EA13210AB282EA1112C2F38D014A4031
:10061000D24312F0030FE5E7B4F86A309B08E4E731
:10062000C36830B59B8D5A1F92B2032A87B0044627
:1006300021D81549023B51F8220020679BB2134A8A
:1006400032F813301946A4F87430FAF717FEB4F8EC
:100650007430206F01930125002301A90493CDE993
:100660000255FAF7E3FCB4F87410206F2A46FAF743
:10067000B5FE07B030BD023B9BB205482067062B94
:10068000DDD901210B46DEE78C9302089C9302081A
:1006900000000240836810B5182104461868F9F775
:1006A00035FE20460021FFF749FBE3681B88A4F8CC
:1006B0006E30DB0500D410BD2046FFF7B1FF2046A9
:1006C000FFF704FF23699B6943F67802D9688A5CC7
:1006D000002AF0D0012283F8562010BD2DE9F843FE
:1006E000B0F86E30076C022B2DED088B044600F03D
:1006F0006D8100F22881002B00F0848190F85C303D
:10070000013BDBB2052B00F2B481DE49C26951F82E
:1007100023000621801AFCF7E9F80328064640F377
:100720008781A369E268861F91683344E069A36109
:100730003044E061FCF7DAF8DFEDD37A94ED0C9AFF
:1007400094ED0A8AB4F86E30D4ED0BAAE061A9EEFC
:10075000278ADB0548BFE7610546B0EE480A48BF77
:100760003D46E9EE27AA13F0FBF8BDEEC0AAA36947
:100770001AEE102A9B1A07EE903AB0EE6A0AB8EE0B
:10078000E7AA13F0EDF8E768BDEEC00AD7ED027AEC
:1007900010EE103AF8EEE79AEB1AF6EE008A69EEE0
:1007A000A88A00EE103A38EEA8BAB8EEC00AF0EE09
:1007B0004B0A30EE280A13F079F99FEDB37AD4EDA5
:1007C0000D7AB5EEC00A67EE877AF1EE10FA48BFEF
:1007D00030EE0B0AAAEE278A70EE688AB0EE6A0A3B
:1007E000A8EEA70A84ED0A8AF0EE690A13F05EF912
:1007F000D4ED0E7A9FEDA47ADFEDA46A27EE877A16
:10080000B5EEC00AA8EE879A67EEA67AF1EE10FA66
:10081000B0EEC97A48BF30EE290AF4EEC77AF1EE9D
:1008200010FA84ED0B0AF0EE498A00F3C68084EDDD
:100830000C9A4FF00009B7EE00AA8AEE299A94EDBF
:10084000147AF6EE007A77EEC77A28EE098A29EE56
:10085000287A29EE000A84ED128A84ED140A84EDC8
:10086000137A37EE800AF0EE4A0A13F01FF9D4F833
:100870001080D4ED157AD8F81830B5EEC00ADB68D0
:10088000F1EE10FAB6EE007A93ED098A48BF30EE29
:100890000A0A77EEC77AF0EE480A37EE800A13F0BC
:1008A00005F9B5EEC00AF868F1EE10FA48BF30EE6F
:1008B000080A2B1A07EE903A84ED150AB9F1000FD9
:1008C00078D13B7D002B75D0002E40F3B6809FED94
:1008D000707A84ED087AF0EE476AD8F8243097ED04
:1008E000046A1B6A9FED6B0A5B689FED6B8A5B0075
:1008F00007EE103AF8EEE77A29EE009A77EEC67A1C
:10090000B8EEC77A77EEA67A27EE097AF0EE480AB3
:10091000A7EE870A13F0CAF8B5EEC00AF1EE10FA96
:1009200048BF30EE080ADFED5B7A30EE670A40F22E
:10093000011384ED090AA4F858300125BDEC088B99
:100940002846BDE8F883A3F58073032B61D890F89F
:100950006C30D0ED117A33BBB7EE007A9FED4A6A66
:10096000DFED4E6A37EE677AE7EE067AF4EEE67A66
:10097000F1EE10FAC0ED117A00F39680E368E069B9
:100980009968002384F86C30381AFBF7AFFFE368EE
:10099000996801EBD173B0EB630FA3690646C8BF3A
:1009A000461A3344C2E69FED3E7A67EE877AC0ED81
:1009B000117AE3E7B6EE007A8BE7DFED357A4FF098
:1009C0000109F0EE678AC4ED0C7A34E7D0ED190A1C
:1009D00090ED180AFBF724FFDFED327AE36920EE91
:1009E000270A41F68B01FDEEC07A17EE900AC01A75
:1009F000FBF77CFF40F645439842064612DCA369AC
:100A0000E26891E68369B0F85A60C268F61A36B2B5
:100A10008AE60821FFF782F9BDEC088B00252846FD
:100A2000BDE8F883A0F5C456A369E2680B3E7BE6F7
:100A3000E268A3699168334478E617D1DFED126A62
:100A400094ED087AA8EEA67AF0EE476AB7EE007A3F
:100A5000F4EEC76AF1EE10FAC4ED086A06DCF5EEB2
:100A6000C06AF1EE10FA3FF532AF36E7B7EE007A22
:100A70002FE7C36893F82A50D5B199688369002697
:100A800054E600BFAC9302086F1203396F1283382B
:100A900000000000DB0F4940DB0FC9400AD7A33B31
:100AA000CFF77F3F00007A448021FFF737F965E7F1
:100AB0001021FFF733F941E738B5037F044683B1CE
:100AC00090ED047AD0ED066AD0ED057A37EE267AFD
:100AD000B4EEE77AF1EE10FAD8BFF0EE477AC0ED47
:100AE000047A2268937A6BB31389657A9A1E92B25C
:100AF000062A98BF1749A3F105039BB294BF31F8AA
:100B000012100121032B96BF134A144852F82300F8
:100B1000FAF75EFC031E18BF0123AB4217BF9FED1F
:100B2000107AD4ED047A84ED047AF0EE477A94EDED
:100B3000057A6372B4EEE77AF1EE10FA03D8226810
:100B4000D27A0AB1237238BDB0FA80F35B092372FE
:100B5000F9E700BFF8930208E8930208000002409A
:100B600000000000007A704703681B8900220261C0
:100B7000C3B19A1E92B2062A70B5A3F105030446CA
:100B800098BF14489BB294BF30F812600126032B23
:100B900096BF114A114D52F8235086B019B92177EA
:100BA00006B070BD704731462846FAF767FB2368E8
:100BB00001961B7B002B14BF012202220023284632
:100BC00001A9CDE90232FAF731FA0123237706B001
:100BD00070BD00BFF8930208E893020800000240CD
:100BE000036810B50446997AFFF7BEFF23689FEDAE
:100BF000057AD3ED017AF8EE677A67EE877AC4ED6D
:100C0000067A10BD6F12833A10B500230022044605
:100C100001604260897A02810277C36003614361A7
:100C20008361FFF7A1FF024BA361204610BD00BF07
:100C30006F12033949B1D0ED107A30EE270A012343
:100C400080ED100A80F854307047D0ED0C7AF4E74C
:100C500003691B6D23B9C26843F679030121D1549E
:100C6000704700BF0278114301707047D1ED0B7AD5
:100C70009FED1D7AC160F4EEC77A0022002310B404
:100C80004FF48071194C0460F1EE10FAC0E906339C
:100C9000C0E90833C0E90A33A0F8541003610375B2
:100CA00080F85630026342638263C2630264426426
:100CB00082640EDC77EEA77AF5EE006A27EEA77A5B
:100CC0005DF8044BC0ED147A27EE267A80ED137A96
:100CD00070479FED077ADFED077A5DF8044BC0EDB2
:100CE000147A80ED137A70470000FA445494020895
:100CF0000024744A00007A4500230363436383633E
:100D0000C3637047012938B504460BD9102114304C
:100D1000FFF7A8FF20694FF400715030FDF712F87B
:100D2000002038BD0B4BC26853F821301B6903F11A
:100D3000540103F1480503F158002432E16103F145
:100D40004C015933C4E90801C4E90A32A561012004
:100D500038BD00BF88080020036990ED0D1AD0ED62
:100D60000C0A10B50446986A4368D3ED022A93ED45
:100D7000012AD3ED001A00F085FC23699A6A00214C
:100D80000023516384F8553010BD00BFD0E9032122
:100D90000969D0ED107A0346C86890ED027A02F531
:100DA0006151B8EEC77A91ED0F6AC6EE076A30B4AA
:100DB00037EEC00AB0EEC00AF4EEC06AF1EE10FAE7
:100DC00018DA516BB1F5616F31D207EE901A9FEDD1
:100DD000217AF8EEE77A002167EE877A0320012472
:100DE0001070002083F85440C3ED107A30BC596471
:100DF0009964704702F56251D1ED006A516BC6EEFD
:100E0000877AF0EEE00AF4EEE07AF1EE10FAD9DD3E
:100E1000B1F5616F084628BF4FF46160013102EB04
:100E200080009C6B5163B1F5616F8463CDD343F651
:100E300079050320107000210024012054631964F7
:100E40005964996483F8540083F85600545530BCB3
:100E5000704700BFB4A29139C3689FED0F7AD3EDFC
:100E60000B7AF4EEC77AF1EE10FA0CDC77EEA77A83
:100E7000F5EE006A27EEA77AC0ED147A27EE267AFF
:100E800080ED137A70479FED057ADFED057A80EDEE
:100E9000137AC0ED147A70470000FA440024744AB3
:100EA00000007A452DE9F0472DED068B076A84B0E6
:100EB00004468846002F00F0FD803B7853BB9946DE
:100EC0001F46A66A16B1367806B1666ADFEDC07AAB
:100ED000D4E9035343F679021B69AA5C93ED120A25
:100EE00020EE279AFAB193F8582012B193F85920BE
:100EF0009AB9202104F11400FFF7B4FE20694FF4E1
:100F000000715030FCF71EFF002004B0BDEC068BD2
:100F1000BDE8F087D0E90697D3E7D3ED130A204662
:100F2000FFF734FFE56895F8203083B195ED098A25
:100F300094ED100AF0EE480A12F0B8FDB5EEC00AC2
:100F4000F1EE10FA48BF30EE080A84ED100A6B7813
:100F5000072B00F21382DFE813F02200CE01A1017B
:100F60007A011102AF000800D7019FED9C6AD5ED10
:100F7000077A94ED127AD4ED0F6A67EE867A37EE2F
:100F8000666AF0EEE77AF1EE675AB4EE656AF1EE62
:100F900010FA40F1168236EEE77A84ED0F7A94ED7E
:100FA0000D8A95F800A0BAF1020F00F2AD80B7EEFD
:100FB00000AA43F69103D5ED047AEB5C73B1B1EE70
:100FC000677AB4EE487AF1EE10FA00F33D81F4EE60
:100FD000487AF1EE10FA48BFB0EE678A43F6920302
:100FE000EB5C7BB1002E84D0D5ED056A96ED007ADE
:100FF00067EEA67AB0EEC77AF4EEC77AF1EE10FA91
:1010000000F1DB812369D5ED029A5A6AD5ED03AA76
:10101000136A93F82010032900F0B28194F8563037
:10102000D4ED0F8A2BB143F68803EB5C002B40F024
:101030008C81BAF1010F40F28E80002E3FF459AF3F
:1010400096ED007AD4ED0E7A38EE478A2AEE087AC9
:10105000E9EE877A78EEA78A2369586AFEF7E6F800
:10106000F4EEC08AF1EE10FAC8BFF0EE408AB1EE9D
:10107000400AB4EEE80ACCBF01230023F1EE10FAD7
:1010800040F38C80E3681B78012B40F25B81D4ED48
:101090000E7A9FED507A67EE877AC4ED0E7AB8F13A
:1010A000000F01D088ED000A012004B0BDEC068BD2
:1010B000BDE8F087B94604E794F85430002B40F0BF
:1010C000888194F85530002B40F079812369986A23
:1010D00090ED0D0AD0ED0B7AB4EEE70AF1EE10FABE
:1010E00040F3858194ED109A9FED3B8AE5684FF0BF
:1010F000030A012385F800A084ED0C9A84ED0D8A83
:1011000084ED0F8A84F8553095F82030002B69D192
:10111000B9F1000F3FF4EDAE94ED0C0AD9ED007A71
:1011200030EE670A43F69003D5ED017AEB5CA7EE4B
:10113000808A002B3FF43BAF05F56253D3ED037A71
:10114000B0EEC00AF4EEC07AF1EE10FAFFF62FAF5F
:1011500080EE27AA2DE743F69303EB5CDBB1002E6C
:101160003FF4C7AED5ED047AD6ED006A37EEA67A25
:1011700029EEC77AF4EE478AF1EE10FA00F11A81EF
:1011800077EEE67A67EEA99AF4EE698AF1EE10FA44
:10119000C8BFF0EE698A9FED108A5DE7E2681278B9
:1011A000012A40F2CD80002B40F01C81DFED0B7A4C
:1011B00094ED0E7A2AEE27AAF0EE477A6AEE2AAA72
:1011C000B0EE680AEAEE887AC4ED0E7A67E700BFEF
:1011D00000006145A4707D3F000000006F120339DC
:1011E000FFFFF945002F3FF484AED4F82C9094ED26
:1011F0000C0AD9ED008AF0EE680A12F057FCB5EE41
:10120000C00AF1EE10FA48BF30EE280AB6EE007AB6
:1012100084ED0C0AD9ED008AD7ED007A68EE878A52
:1012200078EEA89A78EEE77AF0EE690A37EE800A4F
:1012300012F03CFCB5EEC00AF1EE10FA48BF30EEF9
:10124000290A30EE680A6DE7B0EE478AC6E694EDEB
:101250000D8AD4ED117A94ED0C7AD4ED144A94ED04
:10126000106A94ED135A5FED235AD5ED0A6A95F88A
:1012700000A077EEC87A36EE476A67EEA47AE5EE0C
:10128000067AA7EEA58A66EEA77AA8EE257A84EDFF
:101290000D8A84ED0C7AC4ED0F7A84E65FED316A35
:1012A000D5ED067A94ED0D8A94ED117A67EEA67A63
:1012B00037EE487AF0EEE77AF1EE676AB4EE667AD6
:1012C000F1EE10FA08D4B4EEE77AF1EE10FAD4BFDA
:1012D000F0EE476AF0EE676AD5ED0A7A1FED407AC4
:1012E00095F800A067EE877A38EE268A67EEA67A30
:1012F00084ED0D8ACFE794ED118A226CA36C2263F2
:1013000084ED0D8AE3634CE643F69403EB5C012B1A
:101310006BD8494A95F800A052F82320126905F5C8
:10132000625393ED068AD2ED127A92ED137A67EE4C
:10133000887A28EE078AC4ED0C7A84ED0D8A32E6AD
:10134000B0EE680A0023A363A9E6FDEEC97A4FF464
:10135000616117EE900AFBF7C9FAB0F5616FA8BF9B
:101360004FF4616020EAE07005EB8000D0ED0E7A6A
:10137000E56878EEA78A95F800A05AE60221B9E55B
:10138000D2ED2D7A93ED117AF0EEE76AF4EEC76AAA
:10139000F1EE10FA09D517EE903AB0EEC77A002BAD
:1013A000B8BFB1EE477AF0EE477AC9EEA79ACAEE17
:1013B000A7AA33E6F0EE478AEDE601219AE5E56853
:1013C000EDE5B4EEE76AF1EE10FAC8BF36EEA77AA3
:1013D000E3E594ED100A2046FFF7BEFC002384F8F5
:1013E00054306EE6B0EE680A51E6082182E500F05E
:1013F00011FAD4E903539B6A95ED0A7AD3ED0D7A7D
:10140000DFED0E6A95F800A0C4ED0D0A21EE077A13
:1014100077EEA67A84ED0F7A84ED0C0AB0EE608A3E
:10142000B0EE409ACDED020A8DED031A8DED010A62
:10143000C3ED0D7AB7E500BF880800206F120339AD
:10144000027811430170704770B400220024C46018
:10145000046144618461C0E9092270BC416002609A
:10146000027202770262C26280F83020704700BFC9
:101470000368DFED7C1A5B6A90ED0B4A196A93ED05
:101480001A2A93ED1B7AD1ED073AD1ED052A42686D
:10149000D0ED0A5AD2ED027A92ED005ADFED726A6F
:1014A00090ED090AD0ED080AD1ED044A93ED253AF2
:1014B000D3F8903032EE476AF8EEE33A32EE077A2C
:1014C00026EE236AE7EE225A10B521EEC66AB6EE82
:1014D000002AA6EE224A044667EEA77AA4EE260A60
:1014E00025EE025AE5EEA60A85EE274AB0EE405AEE
:1014F000A6EE245AF0EE605AE7EE245A65EE052A6D
:101500002DED068BE5EEA52A92ED019A836277EE2A
:10151000E27A25EE265A64EE277A65EEA65A39EE6F
:10152000099AA7EE850AE7EEA50A69EE269AF7EE74
:10153000007A63EE233AF4EE679AF1EE10FA80ED4A
:10154000090AC0ED080AA6EE240AE7EE240AC0ED57
:101550000B3A7ED59FED457AD0ED067A9FED44AAF1
:10156000DFED43AAB0EE408A90ED040A30EE070AA0
:10157000F0EE608AA7EEA60AF0EE4A0A12F096FA9A
:10158000B5EEC00AF1EE10FA48BF30EE0A0A9FED40
:1015900037AA70EE4A7AF0EE680AC4ED047AB0EE2B
:1015A000480AFBF73DF9D4ED048A84ED030A3AEECC
:1015B00068AAF0EE6A0A3AEE000A12F077FAB5EE7F
:1015C000C00AF1EE10FA48BF30EE2A0ADFED277AA2
:1015D0009FED27AA30EE678A38EEA70AF0EE4A0A96
:1015E000A9EE880A12F062FA2368DFED225A5B6ADC
:1015F000D4ED067A1B6ADFED1D6A93ED017A9FED4B
:101600001E6A29EE099AB5EEC00A29EE259AF1EE76
:1016100010FAE9EE087A4FF00100207748BF30EE6B
:101620000A0AB8EEC77A30EE660AF7EE006AC4ED31
:10163000067AB4EEE67A67EE867AF1EE10FA58BFD3
:10164000C7EE877ABDEC068B84ED040AC4ED057AFB
:1016500010BD01210830FFF7F3FEBDEC068B002022
:10166000207710BD3ACD133F6F120339DB0F49408D
:10167000DB0FC9406F12033883F9223E0022C0E914
:101680000021704721EE015AB6EE007A25EE077A66
:1016900011EE103AC7EE227A002B10B5044670EE18
:1016A000605AF0EEE77AB8BFF1EE677A75EEE77A46
:1016B0002DED068BF5EEC07AF1EE10FAB0EE418A10
:1016C000F0EE628AB0EE40AAF0EE609A00F19380EC
:1016D000B0EE654AF0EE417AF0EE616AB0EE429A01
:1016E000F1EE628ABFEE007AF7EE00AAF4EEE71A96
:1016F000F1EE10FAF1EE667A76EEC84A84ED059ABC
:1017000048BF22EE079A87EEA87AC4EE897A27EEC0
:10171000266A78EE264AF6EE003AA7EEA46A48BF9B
:1017200084ED059A26EE236AC4ED078A66EE2A4AFE
:10173000C4ED066AF4EEC44AF1EE10FA84ED0A7ABA
:10174000C4ED087A4CDD75EEA55A38EEC90AA5EE4F
:10175000895ADFED2F0A25EE285A85EE000A12F08D
:1017600045F900236362B1EEC07A27EE2A7A77EE5C
:10177000486A84ED067AC6EE897AB1EE477AC7EEFA
:10178000286AF5EEC07AF1EE10FAF5EEC06AD8BF1D
:10179000DFED1F7AF1EE10FAD8BFDFED1D6AC4ED60
:1017A000087ACCBF37EEA67AB0EE677AC4ED0A6A43
:1017B000F6EE006A29EE269A84ED0B7AB0EE487AAE
:1017C000A9EE277A0120C4ED029AE7EE279A84ED6C
:1017D00003AA84ED048AC4ED0C9ABDEC068B10BDFF
:1017E00035EEC66A37EE877AC6EE265A37EE257A88
:1017F000C4ED095ADCE730EEC04AB1EE429AF1EE90
:10180000616AF1EE417AB7EE007AFFEE00AA6DE769
:1018100000000000B5EEC00AF1EE10FA88B03DD429
:10182000D0ED087AF4EEC07AF1EE10FA15DD90ED05
:10183000051AD0ED047A90ED027AF6EE006A61EEB8
:10184000266AF0EE670AE0EE267AE1EE000AA0EEE4
:10185000277AB0EE470A08B07047D0ED096A77EEF4
:10186000A66AF4EEC06AF1EE10FA21DCD0ED0B7A34
:10187000F4EEC07AF1EE10FA28DD90ED071A90ED43
:10188000037AF6EE006A70EE677A61EE266A61EE20
:10189000270A66EEA76AA7EEA67ADAE790ED027A43
:1018A000D0ED040A9FED0D1AB0EE470A08B070475C
:1018B00070EE677AD0ED060A90ED0C7A9FED071A6C
:1018C000A0EEA77AB0EE470A08B07047C1D89FEDE6
:1018D000031A90ED037AF0EE410ABAE70000000027
:1018E000BFF34F8F0549064BCA6802F4E062134309
:1018F000CB60BFF34F8F00BFFDE700BF00ED00E0FE
:101900000400FA0508B5FFF7EBFF00BF024B03EB3D
:10191000810191ED000A7047947E0020024B186807
:1019200008441860704700BF8408002008B5FCF721
:1019300055F8FFF7D5FF00BF89B24B1F9BB2032BB1
:1019400009D8094A023952F8230089B2074B33F803
:101950001110FBF7B5BB023989B20629044888BFCC
:101960000121F3D9FBF7ACBB94940208A4940208BC
:101970000000024008B590F83030032B00D008BDBD
:1019800090F83130042BFAD972B6024B024A1A6031
:10199000FFF7A6FF04060020EFBEADDE2DE9F04FF5
:1019A000C54E96F8953093B0002B00F062810DACD7
:1019B000002301254FF00409C048CDF8349021469A
:1019C000CDE90E354FF00808F9F730FBBB48CDF8EC
:1019D00034802146F9F72AFB10272146B8480D9795
:1019E000F9F724FB2846B74DF6F72CFF6823494644
:1019F000B2482B70F9F7ECFC2A780346002B0CBF99
:101A0000134642F001034146AC482B70F9F7E0FC65
:101A10002A78002814BF022300231343A8482B7000
:101A20003946F9F7D5FC2B78002814BF484600202A
:101A300018432870FAF748FBA34D2846F6F770F8CC
:101A4000D6F87C316B602846F6F73AF80325002279
:101A50000123214699480D93CDE90E52F9F7E6FA94
:101A60000223214695480D93F9F7E0FA0423214615
:101A700092480D93F9F7DAFA082321468F480D931F
:101A8000F9F7D4FA214610238D480D93F9F7CEFAD1
:101A90001C2011F0F2FB8D4A8D49044610F0C6FB64
:101AA0008C4B80201C6011F0E8FB8B4B8B4A8C49DF
:101AB0008146FEF781F9342011F0DFFB89490A9055
:101AC000FFF7C2FC582011F0D8FB87498046FFF78A
:101AD000CDF82C2011F0D1FB844A85490B90834628
:101AE000FEF7A0F82C2011F0C8FB82490746FEF74C
:101AF000DBF8EC2011F0C1FB7F4A774BA2F1180113
:101B00000646FDF7FDF9382011F0B7FB7B49824608
:101B1000FFF7B4FD202011F0B0FB79490546FFF72F
:101B200073F8202011F0A9FB76490446FFF76CF802
:101B3000882011F0A2FB0A9B734A0497CDE9056A3D
:101B4000CDE90093CDE90754CDE9028B6F4B00211D
:101B50008246FCF7F5F9DFF880B16D4BCBF85860A1
:101B6000674E6148C3F800A0356143F6A003654D98
:101B70005A4A40F803802C615E4B644CC2F83490A2
:101B80001F628020C4F878A011F077FB534A6149A6
:101B90000BF15C0338328146FEF70EF9342011F068
:101BA0006CFB5D490A90FFF74FFC582011F065FB74
:101BB0005A498046FFF75AF82C2011F05EFB584A2C
:101BC00058490B90FEF72EF82C2011F056FB564981
:101BD0000746FEF769F8EC2011F04FFB534A0BF172
:101BE0005C03A2F118010646FDF78AF9382011F0CE
:101BF00044FB4F498246FFF741FD202011F03DFB99
:101C00004C490546FFF700F8202011F036FB4A4901
